:020000040800F2
:1000000000000120F53F0008B1270008B3270008D1
:10001000B5270008B7270008B9270008000000002E
:10002000000000000000000000000000BB270008E6
:10003000BD27000800000000BF270008C1270008F6
:100040004540000845400008C52700084540000815
:10005000454000084540000845400008454000086C
:10006000454000084540000845400008454000085C
:100070004540000845400008D1270008DD2700085A
:10008000454000084540000845400008454000083C
:100090000000000045400008E9270008454000082E
:1000A000454000084540000845400008454000081C
:1000B000454000084540000845400008454000080C
:1000C00045400008454000084540000845400008FC
:1000D00045400008454000084540000845400008EC
:1000E0004540000845400008F12700084540000849
:1000F00045400008000000000000000045400008E6
:100100004540000845400008FD270008454000081C
:1001100045400008454000084540000845400008AB
:10012000454000084540000845400008454000089B
:080130004540000845400008AD
:1001380010B5054C237833B9044B13B10448AFF319
:1001480000800123237010BDBC08002000000000BF
:100158007839010808B5034B1BB103490348AFF3CD
:10016800008008BD00000000C008002078390108A0
:1001780014214160704714207047406A704700009E
:10018800790100087F01000883010008990100082F
:1001980010B5044604F1100000F05CFCC4F8F80047
:1001A8000148C4F87C0110BD88010008F8B5E6B024
:1001B80004460D4616461F460A4906A800F0CAFE20
:1001C80070996F9A05910492009733466E996D9ACB
:1001D800039102922A466C990191214600F060F839
:1001E80067B0F0BD94010008F8B5E6B004460D46C6
:1001F80016461F46094906A800F0ACFE6F996E9A8C
:100208000491039200976D996C9A0291019233467A
:100218002A46214600F087F867B0F0BD940100082F
:1002280038B500281CBF01680029184A23D1184B8B
:100238001C684FF6F0710C404CF24025AC421FBFD1
:100248001B6819404CF27024A14212D1114D296843
:1002580079B911490B68C3F30B03B3F58A6F1FBF54
:100268000968C1F30B0140F28343994204BF01219D
:10027800117028B905E0094B994204BF012111709A
:100288004068BDE8324001F0B9BE00BFD808002080
:1002980000ED00E0002004E00010005C000037489A
:1002A8002DE9F04104460D46216816464A681F4666
:1002B80090478046B8F5403F2ED122680A99936846
:1002C800204698478046B8F5403F25D12368089ACC
:1002D8000799D3F80CC02046E0478046B8F5403F60
:1002E8001AD12368069A39461F692046B8478046BE
:1002F800B8F5403F10D1236829465D69324620464B
:10030800A8478046B8F5403F06D123680B9A09995B
:100318009D692046A847804621680A68204690477C
:100328004046BDE8F0812DE9F04104460D462168BC
:1003380016464A681F4690478046B8F5403F2ED17A
:1003480022680A999368204698478046B8F5403F46
:1003580025D12368089A0799D3F80CC02046E047AE
:100368008046B8F5403F1AD12368069A39461F6976
:100378002046B8478046B8F5403F10D12368294643
:100388005D6932462046A8478046B8F5403F06D109
:1003980023680999DD6900222046A847804621681C
:1003A8000A68204690474046BDE8F0814FF4403047
:1003B80070470000F0B50C4685B0114600281A4673
:1003C8001CBF0568002D0B4B11D082B104B971B95F
:1003D8000D9860B10F9E0E9F0A9B0290049603979A
:1003E8000B980C9E009001962046A8470346184695
:1003F80005B0F0BD020003002DE9F04F0646D0B06D
:100408000868F56DD6F860E0726EB76EF36E00BAE4
:1004180000906C46486800BA60600DF14008886832
:1004280000BAA060C86800BAE060086900BA206134
:10043800486900BA6061886900BAA061C86900BAF1
:10044800E061086A00BA2062486A00BA6062886A95
:1004580000BAA062C86A00BAE062086B00BA2063FA
:10046800486B00BA6063886B00BAA063C86B00BAB7
:10047800E063402058F80C1C58F820CC58F838ACE9
:100488008CEA010158F840CC8AEA01018CEA01099A
:100498004FEAF979401E48F8049BEBD187EA02003D
:1004A80000EA0E00784010EBF5610098DFF824C4EC
:1004B80041186144C81882EABE032B404FEAF06134
:1004C80053405918636859186144CF194FEAB50366
:1004D80083EABE01014081EABE0111EBF765A1681C
:1004E8004D196544A91883EAB0023A404FEAF1650C
:1004F8005A405519E26855194FEAB70282EAB0071F
:1005080065440F4005EBBE0E97EAB00717EBFE6592
:1005180027697D194FEAB10782EA0701654401EAB4
:100528000E01EB18514011EBF36561694D194FEA63
:10053800BE0187EA010E65440EEA030E15EBB00012
:100548008EEA070E0EEBF065D4F818E075446544A2
:10055800AA1881EAB30505404FEAF26E4D40AE4451
:10056800E569AE44E64477444FEAB00080EAB30E4A
:100578000EEA020E8EEAB30E0EEBF765D4F820E011
:1005880075446544691880EAB2053D404FEAF16E4A
:100598004540AE44656AAE44E6440EEBB3034FEA09
:1005A800B70787EAB20E0EEA010E8EEAB20E0EEB1C
:1005B800F365D4F828E075446544281887EAB1053E
:1005C8001D404FEAF06E7D40AE44E56AAE44E64415
:1005D8000EEBB2024FEAB30383EAB10E0EEA000E45
:1005E8008EEAB10E0EEBF265D4F830E0754465443E
:1005F800EF1983EAB00515404FEAF76E5D40AE4447
:10060800656BAE44E6440EEBB1014FEAB20282EAF2
:10061800B00E0EEA070E8EEAB00E0EEBF165D4F8B6
:1006280038E075446544EB1882EAB7050D404FEA97
:10063800F36E5540AE44E56BAE44E6440EEBB000B5
:100648004FEAB10181EAB70E0EEA030E8EEAB70E41
:100658000EEBF065D4F840E07544654481EAB30ECA
:10066800AA180EEA000E4FEAF2658EEA010E7544EA
:10067800DDF844E04FEAB000754480EAB30E654403
:100688000EEA020E15EBB7078EEAB30E0EEBF7650E
:10069800DDF848E04FEAB202754480EA020E65448C
:1006A8000EEA070E69188EEA000E0EEBF165DDF80A
:1006B8004CE07544654405EBB3034FEAB70E1427C5
:1006C8000DF1500CDFF810528EEA010B82EA0B0B89
:1006D8000BEBF36A5CF804BBDA44AA44504483EA9F
:1006E800B10B4FEAF06A8EEA0B0BDA445CF804BBF4
:1006F800DA44AA44524480EAB30B4FEAF26A8BEA1E
:10070800B10BDA445CF804BBDA444FEAB000AA44FF
:1007180080EA020BD6448BEAB30B0BEBFE6A5CF85B
:1007280004BBDA444FEAB202AA4482EA0E0B0AEB8F
:10073800B10180EA0B0B0BEBF16A5CF804BBDA44FD
:100748007F1DAA44282F0AEBB3034FEABE0EBBD382
:100758003C2F61D3502F4DD204EB870CC7F15407BF
:100768005E4CA7FB04A504465D4FA8088EEA010A63
:1007780082EA0A0A5CF804BB0AEBF3655D447D195A
:100788002C1983EAB10A4FEAF4658EEA0A0A55443D
:100798005CF804AB5CF804BB55447D19AA1884EADC
:1007A800B30A4FEAF2658AEAB10A55445D444FEA52
:1007B800B4047D1984EA020AAE448AEAB30A0AEB51
:1007C800FE655CF804AB55444FEAB2027D1982EA33
:1007D8000E0A15EBB10184EA0A0A5CF804BB0AEBBD
:1007E800F1655D447D1915EBB303401E4FEABE0E5B
:1007F800BCD12046F46D1B19F365336EC9183166F8
:10080800716E71447166B36ED218B266F16E40189B
:10081800F06650B0BDE8F08F4EEA010B0EEA010A0F
:100828000BEA020B4BEA0A0A0AEBF36554F827A015
:10083800DFF8B0C0554443EAB10B654403EAB10A96
:100848000BEA0E0B28184BEA0A0A7F1C0AEBF06524
:1008580054F827A0554440EAB30B654400EAB30AAC
:100868000BEAB10BAA184BEA0A0A7F1C0AEBF265DD
:1008780054F827A055444FEAB00040EA020B6544FB
:1008880000EA020A0BEAB30BAE444BEA0A0A7F1CE1
:100898000AEBFE6554F827A055444FEAB20242EA33
:1008A8000E0B654402EA0E0A0BEA000B15EBB101C8
:1008B8004BEA0A0A7F1C0AEBF16554F827A0554455
:1008C8007F1C65443C2F05EBB3034FEABE0EA3D350
:1008D80040E700BF9979825AA1EBD96ECDCCCCCC38
:1008E800D6C162CADCBC1B8F00B581B00168074A5B
:1008F800914200D110B9064801B000BD7C2112F028
:100908009FFF4FF4003001B000BD00BFFC09000894
:10091800030002002DE9F0410B4A92E8F85188B033
:10092800694681E8F8510268084B9A4200D118B923
:10093800074808B0BDE8F0811422083000F04FFBEA
:1009480008B0BDE8F08100BFDC090008FC09000818
:1009580003000200152904D20268044B9A4200D110
:1009680008B903487047083000F048BBFC09000884
:100978000300020010B481B013460268074CA2427B
:1009880000D118B901B010BC0548704701B000F19A
:10099800240210BC083000F035BB00BFFC09000879
:1009A8000300020010B481B013460268074CA2424B
:1009B80000D118B901B010BC054870470A4601B00B
:1009C80000F1240110BC083000F070BBFC090008DD
:1009D800030002000123456789ABCDEFFEDCBA981E
:1009E80076543210F0E1D2C300000000000000008D
:1009F80000000000F10800081D0900085D09000852
:100A08007D090008AD09000801040008790F0008F5
:100A1800C50F0008810F0008F0B5A3B004460B48C5
:100A280002900D4616461F46094B0822402104A88D
:100A380000F0D1FA28980190009733462A462146BB
:100A480002A800F01BF823B0F0BD00BFFC090008A5
:100A5800100A000810B5040008BF002408D0054893
:100A6800054B20600822402104F1080000F0B3FA89
:100A7800204610BDFC090008100A00082DE9F041C5
:100A880004460E46216817464A681D469047804628
:100A9800B8F5003F19D1226806999368204698470F
:100AA8008046B8F5003F10D123683146DE683A46E3
:100AB8002046B0478046B8F5003F06D12368079A1C
:100AC80029461D692046A847804621680A682046AD
:100AD80090474046BDE8F08110B500F033FA4FF476
:100AE800403400280EBF034C4FF4C07112F0A8FE2A
:100AF800204610BD0200030010B5044600F022FA9B
:100B080008B9054810BD0021A160D0F87C21116802
:100B180088474FF4403010BD0200030070B504460A
:100B28000D4600F00FFA064E40B1D0F87C0141683E
:100B38008847A84224BF65604FF44036304670BDF0
:100B4800020003002DE9FF4715000C4600D02CB128
:100B5800064600F0F7F95FEA000801D16448C3E0EF
:100B6800D8F8F80001684A689047B0F5003F17D1F7
:100B7800D8F87C118A68404690478146B9F1810FC0
:100B880080F09E80A94508F1FC0A17D2D8F8F80031
:100B98000368D3F80CC02A462146E047B0F5003F69
:100BA80040F08E80D8F8F8000368D3F810C06A4681
:100BB8005146E047B0F5003F76D10AE0002004E056
:100BC800215C0AF800100098401C00900098A84288
:100BD800F6D34FF0000C4749474A484B01AC009800
:100BE800844558D2D3E9007001ADC5E9007010788A
:100BF80000281ABF042086464FF0000E085854F803
:100C08000E5028443E4D05600127D0F800E087606B
:100C1800019D4F681AF80C007D408EEA050585F0A5
:100C2800040E65680F687D4085F0FC05754485F005
:100C3800A30568400AF80C000CF1010CCFE7D3E9D2
:100C4800004501A8C0E9004510782E4D002814BFC2
:100C58004FF0040E4FF0000E01A8744651F80EE054
:100C68000459A6440127CEF80050DEF80040CEF81B
:100C780008704D68019F40687D406C400D68684071
:100C880084F0040480F0FC00041984F057040AF886
:100C98000C400CF1010CCC45D1D3D8F8F800016810
:100CA8004A689047B0F5003F0AD1D8F8F8000368C1
:100CB800D3F80C804A465146C047B0F5003F01D0F2
:100CC800114811E0002006E05AF8201081F06A313E
:100CD8004AF82010401CB0EB990FF5D3B06840F0EB
:100CE8000100B0604FF4403004B0BDE8F08700BFA9
:100CF80002000300103A0108D8080020240F000859
:100D0800ADBE4ED70DBE75A10100030038B50C4627
:100D1800017A1546CA0702D500F014F908B908483F
:100D280032BDD0F8F80003682146DC682A46A0479F
:100D3800B0F5003F01D0034832BD4FF4403032BD1A
:100D480002000300010003002DE9F84191B00546B7
:100D58000E461746402101A812F072FD297AC807ED
:100D680004D5284600F0EEF8040002D1DFF8A4808C
:100D78004BE0D4F8F800DFF8A0800368D3F810C07F
:100D88006A4601A9E047B0F5003F3ED1D4F8F80023
:100D980001684A689047B0F5003F36D1D4F87C1115
:100DA8008A6820469047D4F8F830024618461B68EF
:100DB800D3F80CC004F1FC01E047B0F5003F24D1A2
:100DC800D4F87C0141688847D4F8F83002461846C0
:100DD8001B68D3F80CC001A9E047B0F5003F14D157
:100DE800D4F8F8000268696893689847B0F5003F3E
:100DF8000BD1D4F8F80003681C693A463146A0477D
:100E0800B0F5003F08BF4FF44038404612B0BDE887
:100E1800F08100BF02000300010003002DE9F84142
:100E2800A5B0074688461646402115A812F008FDC9
:100E380000220492402105A812F002FD387AC10769
:100E48005ED5384600F07EF8050059D0D5F8F80090
:100E58002D4C0368D3F810C06A4605A9E047B0F5E1
:100E6800003F3CD1D5F8F80001684A689047B0F5D2
:100E7800003F34D1D5F87C118A6828469047D5F8C8
:100E8800F830024618461B68D3F80CC005F1FC017F
:100E9800E047B0F5003F22D1D5F87C01416888478A
:100EA800D5F8F830024618461B68D3F80CC005A9D7
:100EB800E047B0F5003F12D1D5F8F800026879682C
:100EC80093689847B0F5003F09D1D5F8F800036852
:100ED8001D6904AA15A9A847B0F5003F01D020460E
:100EE8000FE00A4B0A490B4A0396029101924046C9
:100EF8001C68049B009415AA796800F0E5F900E0E5
:100F0800054826B0BDE8F08101000300183A010841
:100F1800936E030026C703000200030004B001011A
:100F280000170145E10A0008010B0008250B00081D
:100F3800B50300084D0B0008150D0008510D0008F9
:100F4800250E00080168024A914218BF0020704728
:100F58002C0F000810B5040008BF002404D0034873
:100F68002060204609688847204610BD2C0F0008DD
:100F780020225C3012F062BCF0B58468A30800221D
:100F880004F0030407E000F15C0555F8226035BA67
:100F980041F82250521C9A42F5D300220BE000F18E
:100FA8005C0502EB830755F82360D500C5F11805E9
:100FB800EE40CE55521CA242F1D3F0BD30B5C46804
:100FC80003690022E31AD5188C5C0544521C082AD0
:100FD8002C77F8D330BD0360C1600261704738B523
:100FE800044615460022626023685A68904700202C
:100FF8006061A061A5604FF4003032BD81604FF49C
:10100800003070472DE9F84304462079D4F80C8065
:10101800450748BF244845D466691D46A8F1010024
:1010280000EAD60306EBC506B6EBC50F666102D229
:10103800A669761CA6611746A66906EB5576A661D1
:101048000E46E918884225D2A8EB03094A463146DC
:10105800F81812F0F3FB2268136839460FE042468D
:10106800384612F0EBFB23681A6839462046904749
:1010780007E0311811F00300F1D122681368204607
:101088009847484600EB0809A9F10101A942F0D3A5
:10109800002300E000202A1A3118F81812F0CEFBBD
:1010A8004FF40030BDE8F283040002002DE9FC4F44
:1010B800024685B0D0681369DFF86CC1DFF86C812F
:1010C800A0EB030A506840F004005060002703A812
:1010D80002900DF10C0ED8E9003403A8544DC0E974
:1010E80000342878534D00280CBF00230423994668
:1010F8005CF803305EF80940234401261D601C6833
:101108009E60DCF80430039DDCF80090DEF8046093
:101118005D406540484C654089EA0606474C664094
:101128007519474C6540D8E9006B03AC0028C4E941
:10113800006B0EBF002404200424029E5CF800000B
:10114800345920183F4C04600126046886600398CF
:10115800029E43406340384C7068634089EA00004F
:10116800364C6040034438484340280018BF0120EB
:101178005B1E9B41042F2CBFC0B2D80F02F1140391
:1011880053F8200007F00303C3F10303DB00D84042
:101198000DF807007F1C082F9DD315460C466A6979
:1011A800AB69E868D20842EA4372401E00EA0207C7
:1011B800002302409B420AD8524508D28020E055BD
:1011C8007F1C574516D2AAEB0701E01910E08020D2
:1011D800E05500E0E355E8687F1C8742FAD32A68A7
:1011E800136828469847BAF1000F03D051462046A5
:1011F80012F026FB2A68069E059F936869462846D2
:1012080098472A68D2F8009021462846C8472B6894
:10121800DA683946284690470EB1A86830604FF41E
:10122800003007B0BDE8F08F103A010854120008EA
:10123800D80800205FC5109304850012FC68017A65
:10124800C0F524FF24AF33D426AF698B04B0010165
:1012580000170145F8B501240094002300240DE08F
:10126800009D065D0F5D7E40F643761CF60F86F006
:10127800010635400095641C009DEB189442EFD39D
:101288001846F2BDF8B5002301240094002A11E0A5
:10129800009C85188F1815F8016C17F8015C6E40D2
:1012A800F643761CF60F86F0010634400094009C45
:1012B800E318521EECD11846F2BD00005D1200087A
:1012C8008D120008010000002DE9F84F1D46DDF8D9
:1012D80028900B9F0D9C4FF0FF3300930E469246CB
:1012E800D9F800B0804632465146D847834664B3A1
:1012F800D9F8043032465146404698476FEA0B0207
:10130800521C42EA0B0200996FEAD2735B1C194027
:10131800C2430091521C024300996FEAD2735B1CCE
:101328001940009186F05531484087EA000181F064
:101338005531216080F05531C943491C0843009A52
:101348006FEAD070401C82430092D9F80800012847
:1013580009D17540E943491C0D4300986FEAD572DD
:10136800521C90430AE0F11C85EA9102D243521CB8
:10137800154300986FEAD5735B1C984386F0AA362C
:10138800009086EA0B0686F0AA33F243DB430C98FA
:10139800C2F3C0725B1C42EAD3720099D243521C5A
:1013A80091430091774000998843009987F0AA37C4
:1013B8000F403843BDE8F28F034613F8012B002A8B
:1013C800FBD1181A0138704781F0004102E000BFD4
:1013D80083F0004330B54FEA41044FEA430594EAED
:1013E800050F08BF90EA020F1FBF54EA000C55EA28
:1013F800020C7FEA645C7FEA655C00F0E2804FEAF9
:101408005454D4EB5555B8BF6D420CDD2C4480EADA
:10141800020281EA030382EA000083EA010180EA0A
:10142800020281EA0303362D88BF30BD11F0004F58
:101438004FEA01314FF4801C4CEA113102D040428E
:1014480061EB410113F0004F4FEA03334CEA1333C9
:1014580002D0524263EB430394EA050F00F0A780E1
:10146800A4F10104D5F1200E0DDB02FA0EFC22FADC
:1014780005F2801841F1000103FA0EF2801843FAD0
:1014880005F359410EE0A5F120050EF1200E012AC1
:1014980003FA0EFC28BF4CF0020C43FA05F3C018FF
:1014A80051EBE37101F0004507D54FF0000EDCF178
:1014B800000C7EEB00006EEB0101B1F5801F1BD321
:1014C800B1F5001F0CD349085FEA30004FEA3C0C25
:1014D80004F101044FEA445212F5800F80F09A801B
:1014E800BCF1004F08BF5FEA500C50F1000041EB1F
:1014F800045141EA050130BD5FEA4C0C404141EB23
:101508000101013C28BFB1F5801FE9D291F0000F1D
:1015180004BF01460020B1FA81F308BF2033A3F1CC
:101528000B03B3F120020CDA0C3208DD02F1140CC3
:10153800C2F10C0201FA0CF021FA02F10CE002F1FE
:101548001402D8BFC2F1200C01FA02F120FA0CFCF7
:10155800DCBF41EA0C019040E41AA2BF01EB045140
:10156800294330BD6FEA04041F3C1CDA0C340EDC3E
:1015780004F11404C4F1200220FA04F001FA02F381
:1015880040EA030021FA04F345EA030130BDC4F13F
:101598000C04C4F1200220FA02F001FA04F340EA34
:1015A8000300294630BD21FA04F0294630BD94F0E5
:1015B800000F83F4801306BF81F480110134013DCC
:1015C8004EE77FEA645C18BF7FEA655C29D094EA3D
:1015D800050F08BF90EA020F05D054EA000C04BFBB
:1015E8001946104630BD91EA030F1EBF00210020A6
:1015F80030BD5FEA545C05D14000494128BF41F045
:10160800004130BD14F580043CBF01F5801130BDA8
:1016180001F0004545F0FE4141F470014FF0000033
:1016280030BD7FEA645C1ABF194610467FEA655CE4
:101638001CBF0B46024650EA013406BF52EA033586
:1016480091EA030F41F4002130BD00BF90F0000F74
:1016580004BF0021704730B54FF4806404F13204B0
:101668004FF000054FF0000150E700BF90F0000F69
:1016780004BF0021704730B54FF4806404F1320490
:1016880010F0004548BF40424FF000013EE700BF60
:1016980042004FEAE2014FEA31014FEA02701FBFF0
:1016A80012F07F4393F07F4F81F06051704732F022
:1016B8007F4208BF704793F07F4F04BF41F4002179
:1016C800704730B54FF4607401F0004521F00041D7
:1016D8001CE700BF50EA010208BF704730B54FF061
:1016E80000050AE050EA010208BF704730B511F062
:1016F800004502D5404261EB41014FF4806404F19A
:1017080032045FEA915C3FF4D8AE4FF003025FEA1F
:10171800DC0C18BF03325FEADC0C18BF033202EBA3
:10172800DC02C2F1200300FA03FC20FA02F001FAFD
:1017380003FE40EA0E0021FA02F11444BDE600BFA0
:101748004FF0FF3C06E000BF4FF0010C02E000BF85
:101758004FF0010C4DF804CD4FEA410C7FEA6C5C68
:101768004FEA430C18BF7FEA6C5C1BD001B050EA0B
:10177800410C0CBF52EA430C91EA030F02BF90EAF6
:10178800020F0020704710F1000F91EA030F58BFB5
:10179800994208BF90422CBFD8176FEAE37040F017
:1017A800010070474FEA410C7FEA6C5C02D150EAB5
:1017B800013C07D14FEA430C7FEA6C5CD6D152EA70
:1017C800033CD3D05DF8040B704700BF8446104635
:1017D80062468C461946634600E000BF01B5FFF734
:1017E800B7FF002848BF10F1000F01BD4DF808ED04
:1017F800FFF7F4FF0CBF012000205DF808FB00BFD5
:101808004DF808EDFFF7EAFF34BF012000205DF82E
:1018180008FB00BF4DF808EDFFF7E0FF94BF01207B
:1018280000205DF808FB00BF4DF808EDFFF7CEFF7C
:1018380094BF012000205DF808FB00BF4DF808EDBB
:10184800FFF7C4FF34BF012000205DF808FB00BF8C
:101858004FEA410212F5001215D211D56FF47873D0
:10186800B3EB625212D94FEAC12343F0004343EA73
:10187800505311F0004F23FA02F018BF404270474E
:101888004FF00000704750EA013005D111F00040D8
:1018980008BF6FF0004070474FF00000704700BF6E
:1018A80080F0004002E000BF81F0004142001FBF0D
:1018B8005FEA410392EA030F7FEA226C7FEA236C16
:1018C8006AD04FEA1262D2EB1363C1BFD21841400B
:1018D80048404140B8BF5B42192B88BF704710F0A1
:1018E800004F40F4000020F07F4018BF404211F044
:1018F800004F41F4000121F07F4118BF494292EAAC
:10190800030F3FD0A2F1010241FA03FC10EB0C00D7
:10191800C3F1200301FA03F100F0004302D5494264
:1019280060EB4000B0F5000F13D3B0F1807F06D311
:1019380040084FEA310102F10102FE2A51D2B1F109
:10194800004F40EBC25008BF20F0010040EA0300FE
:101958007047490040EB0000013A28BFB0F5000F7E
:10196800EDD2B0FA80FCACF1080CB2EB0C0200FA34
:101978000CF0AABF00EBC25052421843BCBFD04083
:101988001843704792F0000F81F4000106BF80F4FD
:1019980000000132013BB5E74FEA41037FEA226CC0
:1019A80018BF7FEA236C21D092EA030F04D092F08B
:1019B800000F08BF0846704790EA010F1CBF0020BF
:1019C800704712F07F4F04D1400028BF40F000401C
:1019D800704712F100723CBF00F50000704700F03C
:1019E800004343F0FE4040F4000070477FEA226263
:1019F80016BF08467FEA23630146420206BF5FEA34
:101A0800412390EA010F40F4800070474FF0000333
:101A180004E000BF10F0004348BF40425FEA000CFA
:101A280008BF704743F0964301464FF000001CE0A2
:101A380050EA010208BF70474FF000030AE000BFF8
:101A480050EA010208BF704711F0004302D5404236
:101A580061EB41015FEA010C02BF844601460020A8
:101A680043F0B64308BFA3F18053A3F50003BCFAC3
:101A78008CF2083AA3EBC25310DB01FA02FC634470
:101A880000FA02FCC2F12002BCF1004F20FA02F277
:101A980043EB020008BF20F00100704702F120026A
:101AA80001FA02FCC2F1200250EA4C0021FA02F2CB
:101AB80043EB020008BF20EADC7070474FEA40029F
:101AC800B2F1FE4F0FD34FF09E03B3EB12620DD964
:101AD8004FEA002343F0004310F0004F23FA02F0CE
:101AE80018BF404270474FF00000704712F1610F75
:101AF80001D1420205D110F0004008BF6FF000404C
:101B080070474FF00000704753B94AB9002908BF21
:101B180000281CBF4FF0FF314FF0FF3000F06AB9CA
:101B2800ADF1080C6DE904CE00F006F8DDF804E02C
:101B3800DDE9022304B070472DE9F047089D0C4603
:101B4800002B4ED194468C458646B2FA82F262D971
:101B58004AB1C2F12003914020FA03F30CFA02FCC7
:101B6800194300FA02FE4FEA1C471FFA8CF6B1FB34
:101B7800F7F44FEA1E4307FB141143EA014304FB41
:101B880006F199420AD91CEB030304F1FF3080F0F7
:101B98001281994240F20F81023C6344591A1FFA9C
:101BA8008EF3B1FBF7F007FB101143EA014300FB8A
:101BB80006F69E420AD91CEB030300F1FF3180F0C0
:101BC800FC809E4240F2F980634402389B1B40EA45
:101BD800044000211DB1D3400022C5E90032BDE810
:101BE800F0878B4205D90DB1C5E9000100210846EF
:101BF800F5E7B3FA83F1002946D1A34202D3904214
:101C0800C0F0F080861A64EB03030120002DE6D0B3
:101C1800C5E90063E3E7002A40F09080A1EB0C04DB
:101C28004FEA1C481FFA8CF70121B4FBF8F64FEA7B
:101C38001E4308FB164443EA044307FB06F0984298
:101C480008D91CEB030306F1FF3402D2984200F2D4
:101C5800CD8026461C1A1FFA8EF3B4FBF8F008FB59
:101C6800104443EA044300FB07F79F4208D91CEBE2
:101C7800030300F1FF3402D29F4200F2B0802046F5
:101C8800DB1B40EA0640A5E7C1F120068B4022FA9B
:101C980006F71F4320FA06FC04FA01F343EA0C0393
:101CA800F44000FA01F8380C4FEA1349B4FBF0FE8F
:101CB8001FFA87FC00FB1E4449EA04440EFB0CF99A
:101CC800A14502FA01F20AD93C190EF1FF3A80F057
:101CD8008480A14540F28180AEF1020E3C44A4EB21
:101CE80009041FFA83F9B4FBF0F300FB134449EA33
:101CF800044403FB0CFCA44507D93C1903F1FF304D
:101D080067D2A44565D9023B3C4443EA0E40A0FB98
:101D18000293A4EB0C049C42CE469C4651D34ED071
:101D280055B1B8EB0E0364EB0C0404FA06F6CB408D
:101D38001E43CC40C5E90064002150E7C2F12003EE
:101D480020FA03F10CFA02FC24FA03F394400C4342
:101D58004FEA1C4800FA02FE1FFA8CF7B3FBF8F0B2
:101D680008FB1031230C43EA014300FB07F19942B9
:101D780008D91CEB030300F1FF362CD299422AD96B
:101D8800023863445B1AA4B2B3FBF8F108FB1133C1
:101D980044EA034401FB07F3A34208D91CEB0404FB
:101DA80001F1FF3613D2A34211D902396444E41A6F
:101DB80041EA004139E70446F0E6084606E7C84527
:101DC800AED2B9EB020E63EB070C0138A8E7314637
:101DD800EDE7034699E73046D4E7D6467FE7634404
:101DE80002384DE70646234608460FE7023E63449D
:101DF80030E700BF704700BF1348144A08B54FF0DA
:101E08000043C0E900230422426101220023C26189
:101E18004FF480510722C0E90233C0E90933C0E911
:101E28000C1203610383837680F8203080F82C300D
:101E3800826380F83C30C36404F096FE18B1BDE8B4
:101E4800084000F0EFBB08BDDC080020002401407A
:101E580010B5044688B01422002103A811F0BAFC7A
:101E68002268114B9A421DD14FF0B04303A91A6E54
:101E780042F400721A661A6E02F400720292029A12
:101E8800DA6C42F00102DA64DB6C03F001030193BF
:101E9800019B4FF4004203234FF09040CDE9032308
:101EA80005F080FD08B010BD002401400268084B11
:101EB8009A420BD14FF0B0424FF40041136E23F415
:101EC800007313664FF0904005F018BE704700BFCE
:101ED8000024014030B585B000240546CDE9014411
:101EE8000394FFF789FF144805F0D2F908B100F010
:101EF80099FB1148039401A9CDE9015404F092FF1C
:101F080008B100F08FFB0C4805F0ECF808B100F0C0
:101F180089FB4FF0FF31084804F026FF064805F01A
:101F280099F9054804F07AFF0446034805F03CF99E
:101F3800204605B030BD00BFDC080020014B024A36
:101F48001A607047DC0800200024014008B50948E1
:101F5800FFF7C0FF68B1084BB3F8AA304FF6FF721D
:101F6800934216BF40F6E442044B5343B3FBF0F3ED
:101F780098B208BD002000B40075FF1FD8084C00B7
:101F880013B50023ADF80630FFF7E0FF0446194803
:101F9800FFF7A0FF184BB3F8C820B3F8A8108A427F
:101FA80004FB00F018D040F6E443B0FBF3F36420E0
:101FB8005B1A4343521A93FBF2F31E331BB2ADF87C
:101FC8000630BDF806305BB21B02ADF80630BDF82E
:101FD800060000B202B010BD4FF47A7240F6FF73EB
:101FE800B0FBF3F35343A3F53923A3F50C6340F691
:101FF800C412E0E7001000B00075FF1F4FF0B043B7
:1020080082B09A6A22F480529A629A6C42F48052A0
:102018009A649B6C03F480530193019B002002B0E7
:1020280070474FF0B04307B59A6C42F004029A64C7
:102038009A6C02F004020192019A9A6C42F0010231
:102048009A649B6C002203F00103114600930E2052
:10205800009B05F0BBF90E2005F0EAF900221146B5
:102068000F2005F0B3F90F2003B05DF804EB05F07D
:10207800DFB9000008B505F0B5FB10B16FF004003A
:1020880008BD064B9A6942F040429A614CF2FA3216
:102098001A6105F0B9FB0028F2D0EFE700400058BC
:1020A800F0B585B000230D4600930646A8B3FFF7A8
:1020B800E1FF044670BB05F095FB88BB1A481B4A34
:1020C80002230193D0F8E01506F1784302EA812152
:1020D800B3FBF1F701FB1733DB0A0293D0F8E005F5
:1020E80005F178410139314402EA8022B1FBF2F06E
:1020F80002FB1011C3EBD1230133694601A80393F6
:1021080005F002FC20B1022814BF6FF0010401247D
:1021180005F07AFB204605B0F0BD6FF00504F9E73D
:102128006FF00404F6E700BF0070FF1F00FCFF0318
:10213800014B186000207047400900202DE9F04F3E
:10214800B0F1006F89B006460F469046C0F0C080D7
:10215800DFF89091644DD9F8E03505EA832303F15F
:102168000063013B984200F2B380002900F0B3807D
:1021780040EA02035B0740F0AE80FFF77BFF0446AE
:1021880090BB05F02FFB002840F0A880D9F8E01597
:10219800009705EA812106F17842B2FBF1F301FBD1
:1021A800132208F17843013B3344B3FBF1F001FB00
:1021B8001033DB0A01334FEAD22AA3EBD222012AD9
:1021C800039388BFC6F30A050AF58037C6F10803EA
:1021D8008CBFC5F500654546FF02B3460693039BD1
:1021E8009A4505D305F010FB204609B0BDE8F08FED
:1021F800A6F10803069A1A4495421CD8009B049538
:102208000193CDF814B04FF00009059B09EB0301C9
:10221800049B99453DD3009BAB442B44A8EB050593
:10222800B5F5006F009328BF4FF400650AF1010A65
:1022380007F50067D3E753F8081F5A68B2F1FF3F64
:1022480008BFB1F1FF3FD5D0284B186810B96FF01F
:102258000504C7E727B14FF40062394610F07EFE47
:10226800DFF888900099D9F80030CBF30A001844B9
:10227800AAB210F073FE4FF400613846FFF710FF62
:1022880000BBD9F8003001934FF40063059704931D
:10229800B9E7019B07914B4402930120D3E900233E
:1022A80005F0ECFA88B90799019BD1E9000259F8C1
:1022B8000310029B5B689A4208BF884205D109F166
:1022C8000809A2E76FF001048CE76FF0030489E7BF
:1022D8004FF0FF3488E76FF0050485E76FF00404DA
:1022E80082E700BF0070FF1F00FCFF0340090020C9
:1022F800B1F1006F70B510D30B4BD3F8E0650B4B01
:1023080003EA862303F10063013B994205D838B1FB
:1023180092B210F023FE002070BD4FF0FF30FBE7B3
:102328006FF00500F8E700BF0070FF1F00FCFF0317
:10233800B0F1006F10B40DD3084BD3F8E045084B4B
:1023480003EA842303F10063013B984202D810BCDE
:10235800FFF7A6BE4FF0FF3010BC70470070FF1F9C
:1023680000FCFF034FF0B04382B0DA6C0243DA643A
:10237800DB6C03400193019B02B070472DE9F043E9
:1023880087B000240120264E0594FFF7EBFF0220BA
:10239800FFF7E8FFFFF7E6FF0120FFF7E3FF02275B
:1023A80020224FF4041301A93046CDE90123012569
:1023B8004FF008090394049705F0F4FA01A9304690
:1023C8004FF40078CDE90195CDE9037405F0EAFAF8
:1023D80001A94FF09040CDE90185CDE9037405F0DE
:1023E800E1FA142301A93046CDE90135CDE903749A
:1023F80005F0D8FA2A464946304605F0F9FB2A4640
:1024080041464FF0904005F0F3FB22462146162046
:1024180004F0DCFF162005F00BF807B0BDE8F083E8
:10242800000400481248134A08B540F61463C0E98E
:10243800002300230122C0E90232C0E90433C0E9C5
:102448000633036205F050FD08B100F0EBF80848C8
:10245800002105F0C9FE08B100F0E4F804480021A5
:1024680005F0E8FE18B1BDE8084000F0DBB808BD8B
:10247800040A00200058004070B596B005461422A2
:10248800002103A811F0A6F93822002108A811F0AC
:10249800A1F92A68304B9A425BD18023089308A897
:1024A8004FF440230E9306F021FC08B100F0BAF86F
:1024B8004FF0B0444FF4C050E36C43F00103E364C1
:1024C800E36C03F001030293029B12230026CDE97B
:1024D80003030323CDE905634FF09040042303A9C8
:1024E800079305F05FFAA36DDFF870C043F480032B
:1024F800A365A36D1A4C03F480030193019B266224
:102508000D23C4E900C320468023C4E90266C4E958
:102518000436C4E9066604F0EBFF08B100F082F85F
:10252800104AEC63A562104C0E23C4E90023102165
:10253800002380222046C4E90213C4E90423C4E925
:102548000633236204F0D4FF08B100F06BF8AC63E3
:10255800A56216B070BD00BF00580040440002409C
:10256800A4090020580002404409002000B59BB08F
:102578004822002108A811F02DF91822002102A8EC
:1025880011F028F905F07CFE4FF0B0420120D2F896
:10259800903023F01803C2F89030D2F8003423F4B6
:1025A800C06343F40073C2F80034D2F8003403F473
:1025B800C0630193019B2423089381230B93002379
:1025C800CDE91003B02208A8CDE9122305F0D0FF09
:1025D80008B172B6FEE74F23CDE90230CDE9040019
:1025E800CDE90600022102A806F05CFA08B172B62D
:1025F800FEE71BB05DF804FB08B504F07BFAFFF7B3
:10260800B5FFFFF7BBFE064807F06AF9FFF709FDBB
:10261800FFF708FF00F009FD00F00EFDFCE700BF22
:10262800340B002072B6FEE700B58DB02C220021D5
:1026380001A811F0CFF81748174B03601F238360D8
:102648004FF080420023C0E90433C0E907238361C7
:102658004FF48073436206F0CBFC08B1FFF7E2FF4A
:102668000C4806F0F1FD08B1FFF7DCFF4FF000530E
:1026780000220793074808924FF4807301A9029239
:1026880006920B9306F014FD08B1FFF7CBFF0DB0CF
:102698005DF804FB580A00200028004010B50446E5
:1026A80090B03822002102A811F094F82268194B42
:1026B8009A422CD14FF48033029302A84FF48073CE
:1026C8000F9306F013FB08B1FFF7ACFF4FF0B043D0
:1026D8000220D3F8902042F40042C3F890209A6D6B
:1026E80042F480629A659B6D002203F48063114670
:1026F8000193019B04F06AFE022004F099FE002277
:102708002A20114604F062FE2A2004F091FE10B03F
:1027180010BD00BF002800407047000010B51448E5
:10272800144C07F0DDF800F0DBFB00224FF6FF71D8
:102738004FF0904005F05CFA20464FF6FF7105F027
:10274800DDF9204600224FF6FF7105F051FA0A48DC
:1027580000224FF6FF7105F04BFA04F0E1F9074B40
:102768000120BDE81040C3F8880005F0E1BD00BFB6
:10277800340B0020000400480008004800040058FA
:1027880004F0D5B908B504F0D2F9BDE80840FFF760
:10279800F5BD08B504F0C4F9BDE8084001210020E2
:1027A80005F076BD70477047FEE7FEE7FEE7FEE7F7
:1027B800FEE770477047704770470000014806F011
:1027C80069BD00BF580A0020014804F09DBF00BF42
:1027D800A4090020014804F097BF00BF4409002065
:1027E800202005F013BA0000014806F087BB00BF9F
:1027F800580A0020014806F076BF00BFBC0A002036
:102808002DE9F04389B080460020109E0790894644
:1028180015461F46FDF704FDF0B9104CCDE90090B0
:10282800CDE9020407AB0E480593142304933A46F6
:10283800434629460068FDF7BDFD2346324604F1AC
:10284800140153F8044B42F8044B8B42F9D1079B0F
:10285800337509B0BDE8F0830120FAE7A60A002025
:102868000C3A01081FB50E4C00233C2202A8CDE902
:1028780002336275237500F0B7F8042303AA0094A5
:1028880012210848FFF7BCFF07491422204610F020
:1028980091FFB0FA80F35B09637504B010BD00BF07
:1028A800900A0020343A0108E50D0020054808B5D3
:1028B8000823036006F034FD18B1BDE80840FFF7AF
:1028C800B1BE08BDBC0A00204FF0B04307B55A6E30
:1028D80042F001025A665B6E002203F00103019385
:1028E80011463220019B04F071FD322003B05DF8DF
:1028F80004EB04F09DBD00000CB407B5054A05AB18
:102908001021019310F034FE03B05DF804EB02B01F
:10291800704700BF463A010830B585B0044602A8A2
:102928000D4610F051FCBDF90C30064A00931021F9
:10293800029B2046FFF7E0FF2046FEF73DFD28807A
:1029480005B030BD463A01084FF0B04210B5936863
:1029580023F40043936010F0BFFC0D4B01241C705E
:1029680010F08CF90B4810F0A3F90B4B4FF4004210
:102978001A61002010F0A2F9FFF7E0FA00F0B4F8AD
:1029880010F096FA21462046BDE8104010F0B0BA83
:10299800C80A0020212900080040005810F0BEBADB
:1029A80008B5FFF7D3FA40F6B83398420CD8B0F51B
:1029B800E16F0BD3FE23A0F5E16058434FF4966313
:1029C800B0FBF3F0C0B208BDFE20FCE70020FAE738
:1029D8007FB5684600F06CF80198FFF76FF800B211
:1029E80007B05DF804FB0000194A38B5D2F8803505
:1029F800591C044619D104F0A1F8054604F0AAF8B8
:102A0800054404F0A1F82B0EE3712B0CA3712B0ADB
:102A18006371030EE370C0F30742C0F30723257107
:102A2800C0B2A2706370207038BD190AC371817179
:102A3800190C1B0E41710371D2F88435C370D2F89A
:102A48008405C0F30722C0F30743000EE9E700BF7F
:102A58000070FF1F38B5094BD3F880350360013388
:102A6800054609D104F06AF8044604F06DF84440BC
:102A780004F070F844402C6038BD00BF0070FF1FA0
:102A88000121022010F01EBA0021022010F01ABA0B
:102A980000207047024B187808B100F05DB8704705
:102AA800C80A002082B00190019802B000F0F0B886
:102AB80010B50446FFF764FA074BA36040F30F20F4
:102AC800FEF7A8FF054B064A2360064B6060C4E981
:102AD8000323002010BD00BF0000484200007A44D4
:102AE8000D093E00AB03050000207047014B186834
:102AF800704700BFCC0A00200320704708B5014684
:102B08004FF47A7200238002890DFEF7FDFF08BD9D
:102B18004FF47A73A0FB0303800A40EA835070479E
:102B2800034B98689A689042FBD1C043704700BF36
:102B38000028004008B5FFF7F3FF014B186008BDF7
:102B4800CC0A002008B5FFF7EBFF024B1B68C01A40
:102B580008BD00BFCC0A0020024B187808B1FFF767
:102B6800DFBF7047D00A002010B5074B074C012281
:102B7800DA654FF48071204606F086F94FF0FF338E
:102B88002363002010BD00BF00280040580A002021
:102B980002460021014806F08EBB00BF580A0020FB
:102BA80002460121014806F086BB00BF580A0020F2
:102BB80010B58CB02C220021044601A810F00AFEA2
:102BC800FFF7D2FF0C4B0D481B681C4400230893E9
:102BD80006934FF00053E443079301224FF48073A8
:102BE80001A902940B9306F063FA08B1FFF71AFDE6
:102BF80000200CB010BD00BFCC0A0020580A0020ED
:102C080038B50546FFF78CFF02210446074806F051
:102C180059FBC4F309024FF47A71A2FB0121920A0D
:102C2800A30A2A8043EA805038BD00BF580A002012
:102C38000148002106F046BB580A0020014801213E
:102C480006F040BB580A0020F8B50F4D2E78CEB9D3
:102C58000E4C4FF0FF372763FFF7E6FCFFF784FFC2
:102C68004FF48071204606F00FF92046276306F0DE
:102C7800CDFA32462046022106F01DFBFFF75AFF27
:102C880001232B700020F8BDD00A0020580A00202C
:102C9800014610B54FF47A7200238002890DFEF7C1
:102CA80033FF0146FFF73CFF0446FFF739FF031BDC
:102CB8008B4200D310BD00BFF7E710F015BC000031
:102CC80010B5064C0221204606F0FCFA0221421CEF
:102CD8002046BDE8104006F0EEBA00BF580A0020B2
:102CE8001348144A08B54FF4E133C0E90023002320
:102CF8000C22C0E90233C0E90523C0E90733C0E963
:102D08000933036107F007FB08B1FFF78BFC08489C
:102D1800002107F075FC08B1FFF784FC044807F0B0
:102D28004FFC18B1BDE80840FFF77CBC08BD00BFE8
:102D3800340B00200044004070B596B006461422BB
:102D4800002103A810F046FD3822002108A810F041
:102D580041FD32682C4B9A4254D10223089308A8AB
:102D68002A4B0A9305F0C2FF08B1FFF75BFC4FF04E
:102D7800B04300259A6D42F400329A659A6D02F4C8
:102D880000320292029ADA6C42F00102DA64DB6CD9
:102D980003F0010301930422019B0223CDE90323DD
:102DA8000324072303A94FF09040CDE90554079366
:102DB80004F0F8FD082303A94FF09040CDE903344F
:102DC800CDE90555124C04F0EDFD12492562142396
:102DD800C4E900131023C4E9023520468023C4E95E
:102DE8000435C4E9065504F083FB08B1FFF71AFC63
:102DF8002520F46700220221A66204F0E7FA2520C4
:102E080004F016FB16B070BD0044004004000C002E
:102E1800D40A00208000024002680C4B9A4210B588
:102E2800044612D14FF0B0420C21936D23F40033C5
:102E380093654FF0904004F061FEE06F04F0CAFB28
:102E4800BDE81040252004F001BB10BD004400403F
:102E580008B50A460146024806F062FD002008BD92
:102E6800340B002013B5114B114C18604FF40013AC
:102E7800009302AB13E90600204607F045FB2368E0
:102E8800DA69D103FCD4DA695202FCD59A68084899
:102E980042F480029A6007F07DFB0649044801224B
:102EA80007F0EEFA002002B010BD00BFC80B0020EA
:102EB800340B0020D00B002008B5074B1860FFF733
:102EC800B0F8FFF70DFF054AD2F8803043F00063F1
:102ED800C2F88030002008BDCC0B00200008005844
:102EE80008B54FF0B04308489A6B42F400329A6331
:102EF8009A6B22F400329A63FFF78EFF112004F0D8
:102F0800A5FA002008BD00BF340B00200268044B5E
:102F18009A4203D1034B00201B681847704700BF33
:102F280000440040CC0B002002680B4B9A4210B5BD
:102F380004460FD1094B1B682BB1D0F8902012B969
:102F480007480121984720460549BDE8104001225D
:102F580007F096BA10BD00BF00440040C80B00201F
:102F6800D00B002010B50A4C23780BB9E37C6BB169
:102F7800FFF778FC0038074B18BF01204000187095
:102F88001B78022B02BF00232370E37410BD00BF1F
:102F9800E50D0020D80B002038B5114C2378F3B983
:102FA800E37CE3B90F4D2B68012B07D92B68042B61
:102FB80004D80D4A0421012000F00CFA2B68042BD8
:102FC8000DD9FFF74FFC0038084B18BF012040000F
:102FD80018701B78022B02BF00232370E37438BDDE
:102FE800E50D0020D40B0020A03A0108D80B0020E2
:102FF80001F0FCB802480122102104F0F9BD00BF1D
:103008000004004802480022102104F0F1BD00BF6E
:1030180000040048022803D80248102104F0EDBD3E
:10302800704700BF00040048704708B5FFF78CFCE4
:10303800BDE8084000F06EBB4FF0FF300FF0D2BF84
:103048007047704770470000014BD870704700BF49
:103058000C000020014B1874704700BF0C000020C2
:1030680008B5022000210FF085FFBDE8084001489F
:1030780010F0E8B9480D0020002101200FF07ABFB8
:1030880010B544F62063084C002818BF03460748CB
:10309800236010F089F92168044810F00DFABDE8A2
:1030A8001040024810F0CEB908000020480D00205A
:1030B80010B5094C206023680BB9084B23600848F9
:1030C80010F072F92168064810F0F6F9BDE81040D2
:1030D800034810F0B7B900BFB4000020400D03004A
:1030E800DC0B00200A460149FFF702B900F003088B
:1030F80038B50C4810F058F907F0E2FE60B90A4CF0
:103108000A480125257007F06FFD2078294607F049
:10311800C3FA044810F096F9BDE83840044810F0A6
:1031280091B900BF480D0020700000200C0000205D
:10313800300D002007F062BF1FB507F0A7FB04465B
:10314800B0B100244A4810F02FF94A4B48481B6890
:103158009C42214638BF194610F0AEF9444810F099
:1031680071F945480022042104F042FD04B010BD65
:1031780001221021404804F03BFD4FF4FA70FFF79C
:1031880091FC01F031F84FF4FA70FFF78BFC012243
:103198000421394804F02CFD01F028F8684601F0B4
:1031A80027F835482246102104F022FD32482246ED
:1031B800042104F01DFD61238DF80C302F4B3922BA
:1031C8001A702F4A596812780A7059684C705968F1
:1031D8002720887059680120C87059681E20087116
:1031E8002849087818B30C70596862F07F020A7091
:1031F8003A221A7005222449244C0978012988BFEB
:1032080000225A70637A33B107F02CFB012802D1EF
:10321800204610F0C9F81E4B1848D978002207F04C
:103228004BFB06308DD107F017FB04468AE7194A95
:103238001948117811B901780029DBD000210170F3
:1032480011705A6804215171BDF800205968100A9C
:1032580088715968CA71BDF808105A68090A11724C
:10326800BDF8081051721E2191720B22C3E700BFEE
:10327800480D00200800002000040048000000203D
:103288003C0C0020E10D0020D80B0020F40B00209E
:103298000C000020600D0020E30D002010B504464E
:1032A80080B190F906306BB9084810F07DF8084BEA
:1032B800E2791A70074B1868FFF7FAFE064B186890
:1032C800FFF7DEFEBDE81040FFF736BFF40B002025
:1032D800E20D0020B40000200800002020B103788F
:1032E80013B1024810F0AEB8704700BF240C00209C
:1032F80008B5104B0122002102201A700FF03AFE87
:103308000D4810F09FF80D4B1B788BB10C4B1A78B9
:1033180072B9DB7C63B90B4B1A68042A9EBF1A6822
:1033280001321A600021BDE8084010200FF022BECB
:1033380008BD00BFE10D0020DC0B0020E20D0020DD
:10334800E50D0020D40B0020044B1B78022B03D181
:10335800002108200FF00EBE704700BF700000204B
:1033680008B507F0B6FD80B907F07CFA01280CD142
:10337800BFF34F8F0549064BCA6802F4E062134356
:10338800CB60BFF34F8F00BFFDE708BD00ED00E045
:103398000400FA0538B504460D4607484FF40061A5
:1033A800FEF7C6FF30B92A4621460348BDE8384033
:1033B800FEF7C4BE38BD00BF00F003087047704771
:1033C80070477047202802BF014B01221A707047CE
:1033D800600E002070B505460C46164607F056FAF2
:1033E8000346002835D000241B480FF0DDFF1B4B97
:1033F80019481B689C42214638BF194610F05CF8F2
:10340800BDE87040144810F01DB84A68F05CD0540C
:103418000133DAB29442F8D8114B0D701B78012BA6
:1034280088BF00244C700F4C637A33B107F01AFA46
:10343800012802D120460FF0B7FF0B4B0B48D97873
:10344800002207F039FA0630CDD107F005FA044614
:10345800CAE70649DDE700BF480D00200800002044
:10346800D80B0020F40B00200C00002000000020E6
:10347800044B1B7823B9044A05210120FFF7AABF92
:10348800704700BFD80B0020A53A010810B50024EA
:1034980090B03C22214601A8009410F09BF92F4BD4
:1034A8002022DA7219788DF8001059788DF80110F9
:1034B80099788DF80210D9788DF8031019798DF85C
:1034C800041059798DF8051099798DF80610D97975
:1034D8008DF80710197A8DF80810597A8DF80910A7
:1034E800997A8DF80A108DF80B2021460DF10B0200
:1034F80058180131007B02F8010F1C29F8D193F804
:1035080028208DF8282093F829208DF8292093F871
:103518002A208DF82A2093F82B208DF82B2093F859
:103528002C206AB193F83F2052B10DF12B010022F3
:103538009818013290F82C0001F8010F142AF7D1DD
:1035480007484FF40061FEF7F3FE20B90448402213
:103558006946FEF7F3FD10B010BD00BF71000020F2
:1035680000F80308014940220FF0F8BC00F80308EE
:1035780070B52A4D28796B794D2BC0B233D1C0EB89
:10358800001080000A2838BF0A204FF47A73584385
:10359800234BAC791860EB794D2BE4B22BD1C4EBFB
:1035A8000414A40095F82C301E4E63BB95F83F30E8
:1035B8004BBB44F62060FFF763FD3068FFF778FDEA
:1035C8002B7A194A1949DBB213706B7A184ADBB2A5
:1035D80013700023EA1892F82C20D2B2CA5401338F
:1035E800142BF7D170BD6B79482B0ABF4FF4616378
:1035F8006B795843C6E7EB79482B0ABF4FF46163F0
:10360800EB795C43CEE7FFF73BFD012C38BF012483
:103618004FF47A735C433460CFE700BF7100002039
:1036280008000020B4000020E40D0020E50D002073
:10363800D80B002010B590B000213C2201A80091C1
:1036480010F0C8F84022314968460FF087FC9DF811
:1036580000203AB99DF80100272803D19DF80210EF
:10366800012909D0FFF712FF4FF47A70FFF71AFA11
:10367800FFF77EFF10B010BD254B1A705870997077
:103688009DF80310D9709DF8041019719DF8051064
:1036980059719DF8061099719DF80710D9719DF818
:1036A800081019729DF8091059729DF80A1099723C
:1036B8009DF80B1001F03F01D972D87AD1B2884237
:1036C8001BD89DF8282083F828209DF8292083F806
:1036D80029209DF82A2083F82A209DF82B2083F89A
:1036E8002B200DF12B0100229818013211F8014FFF
:1036F80080F82C40142AF7D1BAE701F14000684459
:10370800194410F8340C08730132D6E700F803089E
:10371800710000201FB5002403A92046039407F078
:10372800BDFB03A9012007F0B9FB384B38480094CA
:1037380022464FF4FA710FF0D9FD364B3648009403
:1037480022464FF4FA710FF0D1FD344B34480094FF
:1037580001224FF4FA710FF0C9FD2046FEF7E8FC8C
:1037680008B1FEF75FFF2F4B009400224FF4FA6177
:103778002D480FF0BBFD2D4A002101200FF0B6FCAB
:103788002B4A002102200FF0B1FC2A4A0021042014
:103798000FF0ACFC284A002108200FF0A7FC00F02D
:1037A800A9FB2649264807F02FFB264807F01CFAF4
:1037B8001B480FF047FE244B0021187806F06CFFD9
:1037C80022490094224B0968224800220FF08EFDFE
:1037D80020480FF037FEFFF72DFF1F4A0021102069
:1037E8000FF084FC1D4A00214FF480700FF07EFC1E
:1037F8001B4B1C4819681C4B009400220FF076FDE7
:1038080018480FF01FFE04B010BD00BFC9330008F0
:10381800240C0020CB3300080C0C0020C533000812
:10382800F40B002051330008300D0020F5A90008E2
:10383800413100083D310008F9300008000003015B
:10384800240000200C000020700000200800002048
:1038580069300008480D0020A12F0008F92F000842
:10386800B4000020DC0B0020F932000808B500F095
:10387800BBFCBDE8084000F0B9BC000010B500244E
:10388800A2B07C22214603A802940FF0A3FF532381
:103898008DF8083040F22713ADF80A3001238DF86F
:1038A8000C30ADF80440FFF77BF800B200EB4000A5
:1038B80000EB4010FE23B0FBF3F08DF80D0001A8DB
:1038C80000F0A6FCA0B958238DF80E3007248022FA
:1038D800002113480FF07EFF224602A910480FF07E
:1038E800B2FF0F4A21460120FFF774FD22B010BD38
:1038F8008DF80E0000F078FC00F090FD094B1A6876
:1039080012128DF80F201A688DF810205A685B681B
:103918008DF8123012128DF811200B24D7E700BF52
:10392800610D0020640E002030B50378592B91B04A
:10393800044640F0FB8105295AD84378443B162BAE
:1039480056D8DFE813F03F0155002F015500370125
:1039580055005500550055009A0055001A015500AC
:1039680055005500A30155005500B70055005500F6
:10397800550017008578482D11D1BC4A1421012023
:10398800FFF728FD41F28830FFF78CF840F6B83091
:10399800FFF788F811B0BDE83040FFF7E1BC532DC0
:1039A8000ED180220021B2480FF014FFFFF766FF06
:1039B80041F28830FFF776F8AD4A152101208EE0F4
:1039C800432D17D1002468468DF8004007F084F88D
:1039D800A74A4C2313702723547093709DF8003026
:1039E80041330120DBB2D07005211371FFF7F2FCDF
:1039F80011B030BD442DFBD19D4C592323705A235F
:103A08006370A570FFF732FF8022002120460FF077
:103A1800E1FE00232570637001252723A370E5705C
:103A28002571FEF7BDFFFE23B0FBF3F000EB40006D
:103A380000EB40108F49C0B260710B6864229BB2E2
:103A4800B3FBF2F3DBB2A3710B689BB2B3FBF2F0EA
:103A580002FB1033DBB2E3714B689BB2B3FBF2F3AA
:103A6800DBB223724B689BB2B3FBF2F102FB11335A
:103A7800DBB2637222460A21A0E78378303BDBB2CF
:103A8800092BB5D87C497D4A0B700B78DBB2537291
:103A9800774A592313704D2353700B783033DBB2B8
:103AA800032101209370FFF795FC11B0BDE8304069
:103AB800FFF7ECBC8578482D16D16D4A5623137054
:103AC800002353702723937001200323D0701371B0
:103AD80018235371072393711023D371082111B050
:103AE800BDE83040FFF776BC432D81D100243C224D
:103AF800214601A800940FF06DFE6846FFF732FDDD
:103B08005B4B8022214618460FF064FE9DF800208A
:103B1800057042709DF8012082709DF80220C270E5
:103B28009DF8032002719DF8042042719DF805203C
:103B380082719DF80620C2719DF8072002729DF8D7
:103B4800082042729DF8092082729DF80B109DF89A
:103B58000A20C272034601730DF10B02E0B28142E2
:103B680004D80D31424AC9B201203FE704F10D00E3
:103B780012F8015F1D540134F0E7807839280CD819
:103B88003038C0B2FFF736FA394A237813706378B1
:103B98005370A3789370032110E711B0BDE830404B
:103BA800FFF766BC80783928F7D83038C0B2FFF7FD
:103BB80029FAE9E780783928EFD83038C0B2FFF71A
:103BC80029FAE1E78378303BDAB2092AE5D8C078E8
:103BD8003038C2B2092AE0D82179A1F14802D2B21C
:103BE8000B2ADAD8264D45FA02F2D507D5D40A228F
:103BF8004D2902FB030034D13C2358434FF47A7318
:103C08005843204B1860FFF73BFA194A2378137082
:103C180063785370A3789370E378D3700521237980
:103C280013710120FFF7D6FB144B00221A702722CC
:103C38005A7001229A70DA70A278303A02EB820147
:103C4800E278303A02EB4102D2B21A7122795A7103
:103C58000D4A1278D2B21A72074A1278D2B25A7240
:103C680023E74829CAD14FF46163C6E7AB3A010894
:103C7800610D0020640E0020D80B00207100002088
:103C8800DEF7FFFF08000020E40D00208278303ABC
:103C9800D3B2092B81D8C378303BD9B209293FF672
:103CA8007CAF0079A0F14801C9B20B293FF675AF86
:103CB8005F4D45FA01F1C9073FF56FAF0A214D285D
:103CC80001FB02332DD13C2253434FF47A72534304
:103CD800584A13601068FFF7EBF9574A23781370B6
:103CE80063785370A3789370E378D37005212379B0
:103CF80013710120FFF76EFB504B00221A70272228
:103D08005A7001229A70DA70A278303A02EB820176
:103D1800E278303A02EB4102D2B29A712279DA7132
:103D280096E74828D1D14FF46162CDE7502B47D1AF
:103D380002297FF65DAE4378303B012B3FF658AE43
:103D48008378312B7FF454AE0B2904D8FFF790FB0E
:103D58000021394A32E6394D0234002214F8013F75
:103D6800A918303B0132DBB20C2A0B73F6D1FFF7EE
:103D78005BF9314A50231370272100235370917047
:103D88000121D1701171E918581D097B01333031B7
:103D9800C9B20C2B1154F6D100222A7027226A705E
:103DA8000122AA70EA70264A1278D2B22A72254AEB
:103DB8001278D2B26A72EB72FFF768FB1121C8E77A
:103DC800412B7FF415AE4378432B7FF411AE1629AF
:103DD8007FF40EAE1C4D421C002312F8011FE9545B
:103DE8000133142BF9D1FFF7BDF8184B5B7D012B7C
:103DF80019D112490023EA5CC8180133D2B2142B36
:103E080080F82C20F7D10F4B00221A701B78DBB2F8
:103E18004B72FFF73BFB084B0021625C5A5401319F
:103E28001629FAD195E7074B02221A70F3E700BF6B
:103E3800DEF7FFFFB4000020610D002071000020B4
:103E4800E40D0020D80B0020E50D0020900A00208A
:103E580037B504460D4600293AD023480FF0F2FA48
:103E68002B78ABB3A4B36068237888B3032B0DD049
:103E7800392B2FD0022B2BD16178012928D00B06A2
:103E880026D403B0BDE83040FFF74EBD6378012B60
:103E980007D10078012802D0022800D008B906F01E
:103EA800D5FD00240DF107008DF8074006F014FE3B
:103EB8000E4A4C2313702723547093709DF80730D3
:103EC80041330120DBB20521D0701371FFF782FA6C
:103ED80003B030BD6378012BFAD10378044A03F0AC
:103EE80001031370F4E700BF0C0C0020610D0020E3
:103EF8003C0C0020034B0022C3E902220122C3E943
:103F080000227047FC0D002000487047FC0D00207F
:103F18004FF0B04382B0DA6C0243DA64DB6C0340E2
:103F28000193019B02B070472DE9F04186B000244F
:103F38000220154D0594FFF7EBFF0420FFF7E8FF7B
:103F4800124F03944FF4807601230DEB0001CDE965
:103F580001632846032304934FF4005803F022FD1D
:103F680001A93846CDF8048003F01CFD22464146DD
:103F7800384603F03DFE28462246314603F038FE17
:103F8800204606B0BDE8F08100040048000800485B
:103F9800032810B50ED8012810D868B902460B4876
:103FA8004FF4807103F024FE002209484FF40051B9
:103FB80003F01EFE002010BD0122F0E70022034896
:103FC8004FF4807103F014FE0122EEE7000400486C
:103FD8000008004802207047002070470120704701
:103FE800002814BF16200F20704700000D48854692
:103FF80002F07EFD0C480D490D4A002302E0D4581A
:10400800C4500433C4188C42F9D30A4A0A4C00231A
:1040180001E013600432A242FBD30FF0E3FBFEF78A
:10402800EBFAFEE70000012000000020BC08002099
:10403800B4450108BC080020602C0020FEE74FF0C2
:10404800B04382B0DA6C42F00102DA64DB6C03F050
:1040580001030193019B02B07047000070B5012273
:1040680086B05248102103F0C3FDFFF7E8FF4FF474
:10407800805101224FF0904003F0BAFD01224FF425
:1040880000614FF0904003F0B3FD4FF4C05011238E
:10409800CDE9010301A901234FF09040039303F0F8
:1040A80081FC08240A2500224FF480514FF09040EB
:1040B80003F09EFD0120FEF7F5FC01224FF480512C
:1040C8004FF0904003F094FD0120FEF7EBFC013D1A
:1040D800E9D14FF400614FF0904003F083FD08B937
:1040E800013CDFD14FF400614FF0904003F07AFDBE
:1040F800044660BB0425FFF7A2FF012603900DEBE1
:1041080005012A48CDE9015603F04CFC3246294600
:10411800264803F06DFD2120FEF7C4FC22462946FF
:10412800224803F065FD2120FEF7BCFC32462946F3
:104138001E4803F05DFD2120FEF7B4FC1B48224613
:10414800294603F055FD4FF42570FEF7ABFCFFF749
:1041580076FF4FF0B04300249A6D42F480029A65CE
:104168009B6D03F4800300934FF4C052009B12230D
:10417800CDE901230323CDE9034304230DEB030118
:104188004FF09040059303F00DFC094809498460FD
:1041980040F61463C0E900130123C0E90334C0E901
:1041A8000744446103F0A0FE06B070BD0004004857
:1041B8000C0E002000580040FFF750BF10B1012836
:1041C80009D0704701394A424A414FF090404FF4B4
:1041D800007103F00DBD4B1E5A4202485A41082196
:1041E800F7E700BF00040048FFF7E6BF00F016B984
:1041F800054B1A6802805A689B684381034B028109
:1042080001221A70704700BF640E0020E30D0020E1
:1042180010B5044600F008F810F0FF001CBFEE23AC
:104228002370AA23637010BD2DE9F74300242D4E97
:104238002D4D346021462046FFF7C0FF214601205E
:10424800FFF7BCFF21460220FFF7B8FF5227A04620
:10425800012195F8640185F86071C5F86881FFF758
:10426800ADFF0320FEF71EFC0DF10602C021284613
:1042780002F0FCFB80BBBDF806204EF6AA639A420A
:104288002AD14FEA440909F154095FFA89F94946E4
:10429800284600F025F9F8B985F860910DF1060275
:1042A800C021284602F0E2FB284600F0D5FA98B96A
:1042B800326801231A4432600C4AC5F86831116823
:1042C800A3400B4313600134032C05F5C875BFD117
:1042D800306803B0BDE8F0830021E0B2FFF76EFF5D
:1042E800F1E700BF780E0020B8000020740E00200F
:1042F8002DE9F74F344C054604F5966B4FF00A0A42
:104308004FF00E0948F2E8084FF490174FF4804632
:10431800D4F86831002B50D0204600F08DFD0DF107
:1043280002020DF10101204600F04EFB0DF10302DF
:1043380001A9204600F082FE0021204600F0D4F8B2
:1043480001220021204600F094F90122114620465E
:1043580000F08FF9022D0ED81C4B33F815601C4B5A
:1043680053F825701B4B53F825801B4B13F8059009
:104378001A4B13F805A032460121204600F0C2F975
:104388003A460021204600F0BDF94146204600F09B
:10439800C5F84A460021204600F0C2F852460121DD
:1043A800204600F0BDF80DF102020DF10101204692
:1043B80000F00AFB0123C4F87C3104F5C874A34556
:1043C800A6D103B0BDE8F08FB8000020E03A01089C
:1043D800D43A0108C83A0108C33A0108C03A0108AA
:1043E80010B50B7E9BB9D0F87C21098912B1C0E9C0
:1043F8005E1310BD084BD0F878411A68C2F5807377
:104408004B4304FB02331B12C0F87831F1E7012358
:10441800C0F87C31EDE700BF680500202DE9F047C2
:10442800DFF8A480294FFFF7C7FED8F800300BB19A
:104438003B6813B9FFF7F8FE38603B68002B3BDD9B
:10444800DFF88C90234D02200024FFF751FF89F8F4
:104458000040D5F86861012E1ED1DFF87CA02846FF
:10446800514600F049FCB8B951462846FFF7B8FF55
:104478009AF8183083B9194BD5F8782143F82420D5
:10448800D8F80030A6401E4399F80030C8F80060FC
:1044980043F0010389F800301E200134FEF702FBC7
:1044A800032C05F5C875D4D199F800300023C8F855
:1044B80000303B60BDE8F087084B4FF47A721A6011
:1044C8005A609A60F2E700BF740E0020700E002058
:1044D800E30D0020B80000207C0E0020640E0020B0
:1044E8004A088A2102F072BA152906D8044BCB4033
:1044F800DB0702D50174002070476FF00700704792
:104508000B00300010B50A460C46092102F080FA6B
:1045180018B9237803F00103237010BD01F051BED0
:1045280001F02EBD01F033BEF7B500230F46144647
:1045380001210DF1070206468DF8073002F068FAEE
:104548000546D0B9012C9DF8073025D1042F39D85C
:10455800DFE807F00316191C1F0043F010049C4203
:104568000BD022460121304602F030FA68BB71694F
:1045780086F830413046FFF7D1FF284603B0F0BD3A
:1045880043F02804EBE743F00404E8E743F0400471
:10459800E5E743F08004E2E7042F13D8DFE807F0EB
:1045A8000306090C0F0003F0EF04D8E703F0D70463
:1045B800D5E703F0FB04D2E703F0BF04CFE703F02D
:1045C8007F04CCE76FF00305D7E70546D5E713B5B9
:1045D80000230C460DF1070201218DF8073002F087
:1045E80017FA78B99DF80730C3F300122270C3F3A5
:1045F800C002A270C3F380026270C3F38012DB09A9
:10460800E270237102B010BD37B50D460DF10202FC
:10461800F821044602F02AFA70B901AA04212046BA
:1046280002F042FA40B9BDF802201AB1019BB3FB6F
:10463800F2F32B602B68A36103B030BD037F0B70CE
:104648000020704737B50D460DF1060220210446BB
:1046580002F00CFA28B9BDF8063023B9236A2B609A
:10466800207703B030BDDB002B6023620123237762
:10467800F7E70529F8B504460E46154633D862B162
:1046880000EB810301215A6B0023701E042807D810
:10469800DFE800F010191C1F260011460123F4E77B
:1046A80084F82810003D344418BF012584F82850A8
:1046B800002007E0C2F34F224421204602F096F979
:1046C8000028EFD0F8BD84F82A10EBE784F82B1007
:1046D800E8E75B00FE226021204602F0B0F9EFE730
:1046E8001B01EF22F7E76FF00300EBE7052996BF00
:1046F8004018002390F82830137094BF00206FF002
:104708000300704770B54318044693F828300E46E6
:1047180015463BB105291BD8DFE801F0030912143F
:104728001616426304EB86040020656307E0C2F3B3
:104738004F224421204602F059F90028F2D070BDDA
:10474800C263EFE70264EDE7C2F34F226421F1E7A9
:104758006FF00300F3E737B50446154605292AD854
:10476800DFE801F0030614161818436B2B601FE0EE
:104778000DF10602442102F079F9D0B9BDF80620FE
:1047880053028AB12B60A36301230FE0C36BEDE7EB
:10479800036CEBE70DF10602642102F067F940B9FA
:1047A800BDF806305B02E1E7A26B2A6084F8293085
:1047B800002003B030BD6FF00300FAE737B50D46AF
:1047C8000DF107020121044602F022F938B99DF8DB
:1047D800073084F83031DB092B7084F84C3003B093
:1047E80030BD2DE9F843037C0C4601F8083B05462B
:1047F800FFF70AFF40BB207304F110012846FFF7BA
:1048080021FF08BB04F11401284600F019FCD8B9AF
:1048180004F1240705F1270904F1170806463A466A
:10482800B1B22846FFF797FF70B9013619F8013F72
:1048380008F8013F062E07F10407F0D104F13C0106
:104848002846FFF7BBFF08B1BDE8F883211D2846BD
:10485800BDE8F84301F01DBDF0B50022054693B050
:10486800882102F0B3F84FF47A72A5F852214FF478
:10487800C872A5F85421514AC5F858210023504A56
:1048880085F8F030C5F8D4202B6202A92846FFF736
:10489800A8FF044670B9ADF8080002AE0FCE05F1C6
:1048A80010070FC70FCE0FC70FCE0FC796E80F0020
:1048B80087E80F00434BC5F834314FF4FA730126EB
:1048C800A5F838314FF42063A5F83C3132468021F1
:1048D80085F85061284602F079F832460746FF21EC
:1048E800284602F073F8002211460743284602F0D2
:1048F8006DF83C4364B204430DF107029121284648
:1049080002F086F864B29DF8073085F83A3104431E
:1049180032460021284602F059F864B204430022C6
:10492800FF21284602F052F864B204430022802195
:10493800284602F04BF864B2204340B200283BD02E
:1049480013B0F0BD0028FBD1A1B2012228460134E2
:10495800FFF78FFE062CF5D10028F1D104466885B3
:10496800024604212846FFF784FE0028E8D10246C3
:1049780005212846FFF77DFE0028E1D14FF490136A
:104988006B634FF4804201212846FFF7BBFE0028E5
:10499800D6D14FF40C13FF22C5E90F3085F830212A
:1049A8000121284602F012F8012385F83231002847
:1049B800C6D185F81541C3E70446C5E7856B0100F4
:1049C800A470090064008403012300F069BD2DE987
:1049D800F0428EB00C460C2304AA1421054601F0BF
:1049E800DDFF8446002860D1BDF81620BDF81830D8
:1049F800A075BDF81210206052BA5BBA6060BDF8AD
:104A08001A60B5F8520192B29BB249BA5B025202DF
:104A18002361A18276BAE260B0F57A7F8BB295F80D
:104A280031719DF81010B6B20AD0704300F5FA70D3
:104A38004FF47A76B0FBF6F02E7F002E39D186B28D
:104A4800002F40D0B001C0B2B608E0750DF10F00DC
:104A58002681CDE90040284601F072FE844620BB3D
:104A68009DF80FE084F818E005F150060FCE07AF67
:104A78000FC796E80700E37D87E80700D4E903013C
:104A8800A28AADF83020D4E90149CDE90A01CDE97F
:104A9800084907AC8DF833308DF834E00FCC503529
:104AA8000FC597E8070086E8070060460EB0BDE826
:104AB800F0822E8C5E43B2EB262F4FEA262C04D1CF
:104AC80057B948F6E0260020BFE780B25043A2EB72
:104AD8000C06B0FBF6F0B2E742F2B826B2E70000E7
:104AE800F7B517460E210DF106021D460B4C06467A
:104AF80001F0BCFFBDF8063004EA43433B6050B9FF
:104B08000DF106020C21304601F0B0FFBDF8063069
:104B180004EA43442C6003B0F0BD00BF0000FE1F50
:104B280073B590F8DA30013B022B06460C4634D8B0
:104B380001AB6A460121FFF7D3FF009BB3F57F0F56
:104B4800054603D8019BB3F57F0F23D915BB34B1B4
:104B58001349304602B0BDE8704001F0FFBB0422A3
:104B6800FF21304601F032FF2A46044670213046C4
:104B780001F02CFF2A460443FF21304601F026FFAE
:104B880064B204432A468021304601F01FFF64B214
:104B9800044365B2284602B070BD0025FAE700BF9D
:104BA8006C05002037B5044601228021057C01F000
:104BB8000DFF0122FF21204601F008FF00221146C7
:104BC800204601F003FF94F83A219121204601F094
:104BD800FDFE01220021204601F0F8FE0022FF21FF
:104BE800204601F0F3FE00228021204601F0EEFE6F
:104BF800012D24D0032D32D0C5BB012229462046E1
:104C080001F0E4FE01238DF80730B0B905469DF8A0
:104C18000730DB0705F101050AD548B9B5F5FA6F84
:104C280027D001460DF10702204601F0F1FEEEE71C
:104C3800B5F5FA6F08BF6FF0060003B030BD18B9BC
:104C480029462046FFF76CFF02220021204601F08A
:104C5800BDFE0028F1D1042384F83231EDE718B9FC
:104C680001212046FFF75CFF0422EEE76FF0070002
:104C7800E3E76FF00600E0E738B5057C044625B1A8
:104C8800204600F03BFD28B138BDFFF78BFF002818
:104C9800F6D0F9E7002DF7D1032384F83231F3E792
:104CA80073B50646002501220B21304601F08EFE21
:104CB800002204460B21304601F088FE0DF1070260
:104CC80004431321304601F0A3FE9DF8073064B277
:104CD800044301355B0760B2EDB205D0032D08D05F
:104CE8000028E0D002B070BD032D08BF6FF00B00A4
:104CF800F8E76FF00B00F5E738B5002303740446B6
:104D08000D46FFF7B9FF50B929462046FFF75FFE69
:104D180028B901462046BDE83840FFF7C1BF38BD75
:104D2800152970B5054616461C4667D10122FF2194
:104D380001F04CFE002211460446284601F046FECA
:104D480000220443FF21284601F040FE64B20443D8
:104D580001228021284601F039FE64B20443022270
:104D68008521284601F032FE64B204430422FF2163
:104D7800284601F02BFE64B204430022CD212846C8
:104D880001F024FE64B204431122CC21284601F02C
:104D98001DFE64B204430722FF21284601F016FED7
:104DA80064B204430022BE21284601F00FFE64B21B
:104DB80004430622FF21284601F008FE64B204439A
:104DC8000922CC21284601F001FE64B204430022E6
:104DD800FF21284601F0FAFD64B204430122FF21B5
:104DE800284601F0F3FD64B2002204431146284628
:104DF80001F0ECFD64B2204340B270BD042A17D81C
:104E08000A2101F0E3FD0028F7D1231E18BF012372
:104E18001B01EF228421284601F011FE0028ECD165
:104E280085F8DA6001462846BDE87040FFF738BFCC
:104E38006FF00A00E1E7000070B594B00546402223
:104E4800002104A80EF0C6FC002301212846ADF875
:104E580006308DF803308DF80430029300F0A0FC82
:104E680095F8142195F81311012A04D840F0AD8063
:104E7800202940F2AC8001AA02A9284600F02BFBA9
:104E88000446002840F09E8095F85031002B40F0F1
:104E9800A280D5F84C11284601F060FA0446002893
:104EA80040F090800346014604222846FFF738FF69
:104EB8000446002840F086800122FF21284601F0A0
:104EC80085FD0DF1060206468421284601F0CEFD37
:104ED80022460643FF21284601F078FD76B20643B4
:104EE80074B2002C6ED1BDF806301B01C5F8D43061
:104EF80004A92846FFF775FC0446002862D10DF185
:104F080003012846FFF7FEFA044600285AD19DF807
:104F1800033085F8313104AC0FCC05F110060FC60B
:104F28000FCC0FC60FCC0FC694E80F0086E80F0011
:104F38000DF103020121284601F06AFD044600280C
:104F480040D19DF8033085F83031024601462846A5
:104F5800FFF7EAFA0446A8BB024602212846FFF7F3
:104F6800E3FA044670BB0323014685F832310DF19C
:104F78000502284601F00BF9044618BB9DF80530D8
:104F880085F8E8300DF105020121284601F0FFF807
:104F98000446B8B99DF8053085F8E03003AA032126
:104FA800284600F0E7FE044660B9039BC5F8E430E4
:104FB80003AA0421284600F0DDFE044610B9039B2D
:104FC800C5F8DC30204614B070BD0C2951E72846DE
:104FD80000F013F954E701495DE700BF22070020FC
:104FE80013B50C460DF10702132101F011FD9DF8D0
:104FF800073013F0180F03F0070218BF6FF0050011
:10500800226002B010BD13B590F8DA30042B0C46BC
:1050180009D101A9FFF7E4FF019B1A1F534253412D
:10502800237002B010BD01AA142101F0F1FC002880
:10503800F7D19DF8043003F00103F1E700F04BBA13
:1050480013B50C460DF10602282101F00FFD78B9C1
:10505800BDF80620C2F30B0312F4006F18BFA3F5C6
:1050680080534FF0FA0214BF13FB02F3534323603B
:1050780002B010BDF0B54FEAD20C4FF0FF341C60FF
:1050880002F00702664600278E4200D207B1F0BD43
:10509800845D664503BF1441E4B215463D4614F0ED
:1050A800010705D005EBC6051D6001270136EBE7B2
:1050B8000135082D4FEA5404F8D014F0010FF0E739
:1050C800034B800953F82000003818BF01207047AF
:1050D8001808002010B5B1EBD20F4FEAD20402F045
:1050E800070381BF01229A40035D13438ABF03551A
:1050F8006FF03100002010BD0A460623B02101F0F0
:105108002FBC0A460623B02101F048BC2DE9F04F18
:1051180085B00546109F0E9E01978A4693461C4609
:105128004FF00009119B994508D10023129A176086
:1051380013B36FF0310005B0BDE8F08F01AB3A460C
:1051480031465846FFF796FFDDF80480B8F1FF3F77
:105158000FD00F9B08EB0300FFF7B2FF504508D1B3
:1051680042462046FFF7B6FF08F1010709F1010999
:10517800D8E76FF03103D9E721462846FFF7BCFF8F
:105188000028D8D102A92846FFF7BBFF02ABA21915
:105198009442D0D014F8015B13F8011B8D42F7D06C
:1051A800C7E770B5C02288B00E46012190F830518B
:1051B800044601F00BFCF0B901A92046FFF79CFD5D
:1051C800C8B90122FF21204601F000FC98B93246F7
:1051D800B621204601F04AFC68B90246FF21204664
:1051E80001F0F4FB38B92A460121204601F0EEFB14
:1051F80008B984F8305108B070BDF0B50F4689B0D1
:105208001646FF210122044601F0E0FB0246A8B938
:105218004F21204601F0DAFB80B92C224E2120468E
:1052280001F0D4FB024648B9FF21204601F0CEFB2D
:1052380020B9B422B621204601F0C8FB0025C4F8E5
:105248002451A4F82851DEB9354607ABB422CDE97C
:1052580003730623CDE90032029504F5927304F531
:10526800957231462046FFF751FF30B9012384F883
:10527800153184F8137184F8146109B0F0BD013553
:1052880005F1B400FFF71CFF0028DED12C2DF6D164
:10529800DBE710B541F001020021044601F096FB5E
:1052A80078B9204600F02AFA58B901462046FFF797
:1052B800F7FC30B9024601462046BDE8104001F02F
:1052C80085BB10BD2DE9F74F4FF0000B88461746F8
:1052D800FF21012205461E469DF838A09DF83C9006
:1052E8008DF807B001F072FB5A4604465946284625
:1052F80001F06CFB5A460443FF21284601F066FB87
:1053080064B2044364B2B8F1000F32D0BAF1000FAE
:1053180006D00C9ACB21284601F07AFB204344B2F0
:10532800B9F1000F07D00DF10702EE21284601F070
:105338006FFB204344B20122FF21284601F046FBBF
:10534800012204430021284601F040FB64B20443D3
:105358000022FF21284601F039FB64B29DF807308E
:105368000D9A204323F0100340B2137003B0BDE838
:10537800F08FBAF1000F06D03A46CB21284601F04B
:1053880025FB204344B2B9F1000FD4D03346802224
:10539800EE21284601F053FBCBE72DE9F04387B017
:1053A8009146002205460E468DF817201F4653B336
:1053B80090F8308101221146284601F007FB044687
:1053C80048BB40212846FFF764FFF0B9B9F1010F47
:1053D80024D10DF11703CDE90294CDE900632246EB
:1053E800234649462846FFF76DFF044678B947B17A
:1053F80042460121284601F0E9FA044638B985F801
:105408003081002403E09846D4E7347004462046EF
:1054180007B0BDE8F08300233370F8E73070E6E7A3
:105428002DE9F043054687B00E4691461F4653B313
:1054380090F8308102220121284601F0C7FA04467B
:1054480048BB01462846FFF724FFF0B9B9F1010F20
:1054580024D10DF11703CDE90249009322462346D2
:10546800019649462846FFF72DFF044678B947B10B
:1054780042460121284601F0A9FA044638B985F8C0
:105488003081002403E09846D4E73470044620466F
:1054980007B0BDE8F08300233370F8E73070E6E723
:1054A800F8B51D46164600232A4690F83071044682
:1054B800FFF773FF70B903462A4631462046FFF7C7
:1054C800AFFF38B93A460121204601F07FFA08B902
:1054D80084F83071F8BD2DE9F04F002393B0CDE981
:1054E8000A12C0F82431A0F828310122FF21CDE9A1
:1054F8000E33B0F83C818DF8343004468DF83530E1
:1055080001F064FA002840F0F08002464F2120465E
:1055180001F05CFA002840F0E8802C224E21204659
:1055280001F054FA002840F0E0800246FF212046AE
:1055380001F04CFA002840F0D880B422B621204669
:1055480001F044FA002840F0D0800246802120462D
:1055580001F03CFA002840F0C88003460DF13502FE
:105568000DA92046FFF79CFF002840F0BE8004F5F7
:10557800957307930323CDE90203B421062304F5A9
:1055880092790EAECDE90031049601464B4604F5FA
:1055980095722046FFF7BAFD002840F0A6800DF16D
:1055A800360120460E9DFFF7FCFD002840F09D8047
:1055B800BDF83630434541D9C4F82401A4F8280180
:1055C80005F1B400FFF77CFD08B92B2D1FD9062380
:1055D800B42204960326CDE90032CDE90256079A93
:1055E8004B4601212046FFF791FD00287DD10DF1A2
:1055F800360120460E9DFFF7D4FD002875D1BDF871
:105608003630434574D901274FF0010A19E00135B6
:10561800D6E7089E099324E0089E0A9B1E600B9B10
:105628001F70012384F815310A9B1B6884F8133115
:105638000B9B1B7884F81431002056E000273E4667
:10564800BA46BDF836304345E7D2A3EB080383EAF0
:10565800E372A2EBE3725FFA8AF70992032604F574
:10566800927BDBF80000BBF804301090ADF84430B2
:105678002A460FAB07980621FFF7FCFC0F9D6B1C11
:1056880039D005F1B400FFF71BFD5045C5D1731C97
:105698002A4648460893FFF71DFD30BB4946204679
:1056A8000135FFF729FD00BB0DF136012046FFF754
:1056B80078FDD0B9BDF83620A2EB0803002BB8BF9F
:1056C8005B424245A5D9099A9342A5D910A920461B
:1056D800FFF712FDBDF8442003461098C4F82401D2
:1056E800ABF804201846002B97D013B0BDE8F08F14
:1056F8000746064688E76FF03100F6E737B500231E
:1057080004468DF807304FF4FA650DF1070120467D
:10571800FFF779FC58B99DF80730012B07D0013DF8
:1057280003D0204601F0DEF9EFE76FF0060003B082
:1057380030BD02464FF08043934202D8002013B98F
:1057480070479B08F8E7C11891424FEA50009CBF88
:10575800C018521A9B08F2E773B500228321054648
:1057680001F034F9044690B906460DF10702832189
:10577800284601F04DF99DF807300343DBB2044693
:105788002BB90136B6F5FA6FEFD16FF00604012296
:105798008321284601F01AF9204340B202B070BDB7
:1057A8002DE9F04F90F8F06091B04FF00009072E06
:1057B800CDE9079904460F4600F0A2820122802114
:1057C80001F004F901228046FF21204601F0FEF88D
:1057D8004A4648EA00084946204601F0F7F84FFAD9
:1057E80088F848EA00080622FF21204601F0EEF872
:1057F8004FFA88F848EA00080DF11502832120467F
:1058080001F006F99DF815204FFA88F848EA0008D3
:1058180042F004028321204601F0D8F84FFA88F8B4
:1058280048EA00080722FF21204601F0CFF84FFA86
:1058380088F80122812148EA0008204601F0C6F8CC
:105848004FFA88F848EA0008204601F04BF94FFA69
:1058580088F848EA000801228021204601F0B6F8BD
:105868004FFA88F848EA000517F0010B6DB200F00E
:105878001E82F20700F11E826B229421204601F05D
:10588800A5F880462046FFF767FF06AA48EA000801
:105898009021204601F008F945EA0805069B6DB2FB
:1058A8002422942105432046C3F3062AC3F3C039B2
:1058B80001F08CF86DB205432046FFF74DFF6DB23D
:1058C800054306AA9021204601F0EEF8069B6DB22A
:1058D8001BBA2522942105432046099301F076F846
:1058E8006DB205432046FFF737FF6DB2054306AAA0
:1058F8009021204601F0D8F8069B6DB21A0E054398
:105908001B0C6DB28DF828208DF8293017F0020392
:10591800029300F0DB8016F0020840F0D7800222E4
:105928009421204601F052F801902046FFF714FF19
:10593800019B0DF116020343902120461D4301F0FF
:1059480067F86DB27B2294210543204601F03EF8AA
:105958006DB205432046FFF7FFFE6DB205430DF11A
:1059680017029021204601F053F86DB27722942156
:105978000543204601F02AF86DB205432046FFF79B
:10598800EBFE6DB2054306AA9021204601F08CF883
:10599800069B5A0E8DF82C20C3F386428DF82D20D5
:1059A800C3F3C6228DF82E206DB2C3F30612DB00B6
:1059B80003F07803942105438DF82F2020467822A0
:1059C8008DF8153001F002F86DB205432046FFF757
:1059D800C3FE6DB2054306AA9021204601F064F883
:1059E800069B9DF8152002EB53728DF83020C3F307
:1059F80086528DF83120C3F3C6328DF83220C3F3B6
:105A080006228DF833206DB2C3F346029B0103F0E2
:105A18004003942105438DF83420204679228DF8DF
:105A2800153000F0D3FF6DB205432046FFF794FE12
:105A38006DB2054306AA9021204601F035F8069B71
:105A48009DF8152002EB93628DF83520C3F3C6420A
:105A58008DF83620C3F306328DF837206DB2C3F3C4
:105A680046129B0003F07C03942105438DF83820EF
:105A780020467A228DF8153000F0A8FF6DB2054354
:105A88002046FFF769FE6DB2054306AA902120461D
:105A980001F00AF8069B9DF815208DF83E8002EB70
:105AA80093728DF83920C3F3C6526DB28DF83A203F
:105AB800C3F3064205438DF83B20C3F34622C3F3E4
:105AC80086036DB28DF83C208DF83D3017F0040345
:105AD800019300F0F180730700F1EE807B2294219E
:105AE800204600F073FF80462046FFF735FE07AAE0
:105AF80048EA00089021204600F0D6FF45EA080849
:105B08004FFA88F848EA00057C229421204600F0E4
:105B18005DFF6DB205432046FFF71EFE6DB20543DB
:105B280008AA9021204600F0BFFF6DB2732294218D
:105B38000543204600F04AFF6DB205432046FFF7B3
:105B48000BFE6DB2054306AA9021204600F0ACFF7B
:105B5800069B6DB21B0274229421054320461FFA4E
:105B680083F800F033FF6DB205432046FFF7F4FDDC
:105B78006DB2054306AA9021204600F095FF6DB24C
:105B88009DF81B30752294210543204643EA0808F6
:105B980000F01CFF6DB205432046FFF7DDFD6DB236
:105BA800054306AA9021204600F07EFF069B6DB2B1
:105BB8001B029BB27622942105432046039300F0F2
:105BC80005FF6DB205432046FFF7C6FD6DB20543DC
:105BD80006AA9021204600F067FF6DB29DF81B20B1
:105BE800039B05436DB21343002281212046039392
:105BF80000F0ECFE06220543FF21204600F0E6FEF9
:105C08006DB205430DF115028321204600F000FF17
:105C18009DF815206DB2054302F0FB028321204652
:105C280000F0D4FE6DB205430122FF21204600F0AA
:105C3800CDFE6DB2054301220021204600F0C6FECC
:105C48006DB205430022FF21204600F0BFFE6DB271
:105C5800054300228021204600F0B8FE6DB20543BE
:105C68006DB2039BFDB9BBF1000F29D1029AAABB03
:105C7800019AAAB1720713D4079AC4F81821089A8E
:105C8800C4F81C214FEA4822C4F820213BB1A3F5EF
:105C9800C8534FF47A7253431B095B421BB2E3604B
:105CA8003E4384F8F060284611B0BDE8F08FD9462D
:105CB800DA462BE6CA4629E64FF00008434693E742
:105CC800F007D3D40998BDF8282084F813A184F8E4
:105CD8001491C4F82A01A4F82E21C7E7B107C7D444
:105CE8009DF8162084F8F1209DF8172084F8F220FA
:105CF8000BA904F1F30002930DF098FD029BB7E79E
:105D08004D46D0E740B101380023FF2803F10102D6
:105D180003D800EB032080B2704740081346F4E72D
:105D2800C3B2000A03FA00F001307047084B5A4327
:105D38004FF47A7302F5FA724FF4FA60B2FBF0F09E
:105D4800B2FBF3F203FB0100B0FBF2F0704700BFB7
:105D5800002F3A00064B5A434FF47A7002F5FA7254
:105D6800B2FBF0F24A4302F5FA72B2FBF0F0704768
:105D7800002F3A002DE9FF4102294FF000050746A0
:105D880016468DF80350ADF804501CD80DF10202E8
:105D98002946FEF7C7FB044630B90DF10302462138
:105DA800384600F035FE04469DF80300FFF7B8FFBB
:105DB80081B29DF802203846FFF7CCFF30602046BC
:105DC80004B0BDE8F081032918D10DF1020229467B
:105DD800FEF7A8FB0446002846D101460DF1020251
:105DE8003846FEF79FFB044628B901AA51213846D8
:105DF80000F03CFE0446BDF80400D7E7042935D17D
:105E080002A9FEF7E4FB9DF80B304BB30DF102023B
:105E180029463846FEF786FB044618BB01AA5121DD
:105E2800384600F023FE0446BDF80400FFF778FF6B
:105E380085B2BCB90DF1020201213846FEF772FBAA
:105E4800044678B90DF106027121384600F00EFEBD
:105E58000446BDF80600FFF763FF80B2401BA7E7C2
:105E68001D46E7E70020F9E72846A7E728462C461D
:105E7800A4E7F0B5022985B0054616461ED80DF1EF
:105E880005020021FEF74EFB0446A0B99DF8052047
:105E980031462846FFF74AFF83B2B3F5807F9ABFA1
:105EA80000F1FF32D2B2FF22A5F8D82046212846B9
:105EB80000F08CFD0446204605B0F0BD032920D132
:105EC8000DF105020021FEF72DFB9DF80520044683
:105ED80031462846FFF72AFF80B2FFF713FF024634
:105EE800ADF80600A5F8D800002CE4D151212846C9
:105EF80000F07CFD04460028DDD1C5F8E4600024EC
:105F0800D9E7042939D102A9FEF761FB9DF80B7086
:105F1800B7B10DF1050200212846FEF703FB044640
:105F28000028C8D10DF106025121284600F09EFD37
:105F380004460028BFD1BDF80600FFF7F1FE87B27E
:105F48000DF1050201212846FEF7ECFA0446002867
:105F5800B1D19DF8052031462846FFF7E7FE3844C1
:105F6800FFF7D0FE71210246284600F03FFD0446A7
:105F78000028A0D1C5F8DC60C1E76FF003049AE7F8
:105F8800F0B585B000238DF80330D30705460F46DA
:105F9800164605D441B9A2F10C03DAB2062A12D981
:105FA8006FF0030005B0F0BD012920D1A2F108036C
:105FB800DAB2062AF4D8062B19D8DFE803F0371826
:105FC800651886189900062B11D8DFE803F004102D
:105FD80029102B102D0018225721284600F0F6FC16
:105FE80008225621284600F0F1FC0028DAD174086E
:105FF800013CE4B2002F00F08E80012FD0D101AA1D
:1060080004212846FFF7B6FE38B9224670212846F3
:1060180000F0DCFC002800F0B28085F8E060C1E701
:106028003022D9E74022D7E75022D5E7102248216D
:1060380000F0CCFC08224721284600F0C7FC0222C9
:1060480004463221284600F0C1FC0C2204433021CA
:10605800284600F0BBFC64B204430122FF21284615
:1060680000F0B4FC64B2044364B230223021284604
:1060780000F0ACFC00220443FF21284600F0A6FCF7
:1060880064B2204340B2B0E72822482100F09EFCC9
:1060980008224721284600F099FC032204463221B1
:1060A800284600F093FC044364B2092230212846B4
:1060B80000F08CFC01220443FF21284600F086FCF6
:1060C80064B2044364B22022D0E73822482100F0A9
:1060D8007DFC08224721284600F078FC032204466C
:1060E8003221284600F072FC044364B20822DDE73E
:1060F8004822114600F06AFC08224721284600F091
:1061080065FC032204463221284600F05FFC044364
:1061180064B20722CAE702AA03212846FFF72AFE2B
:1061280088B903AA02212846FFF724FE58B9224657
:106138005021284600F04AFC28B9029A0321284633
:10614800FFF797FE10B185F8E8602BE7039A022164
:106158002846FFF78EFE85F8E86000287FF422AF16
:1061680069692846FEF7DAF900287FF41BAF024672
:1061780001230DF103012846FFF752F912E7019AAE
:1061880004212846FFF775FE85F8E060E5E713B5BA
:10619800144629B1012910D06FF0030002B010BDD8
:1061A8000DF10702502100F033FC0028F6D19DF8CC
:1061B800073001335B002370F0E70DF1070270210F
:1061C800F1E7F0B5002385B04FF4FA62CDE900237A
:1061D80044F61F63994206460F4604D86FF003053C
:1061E800284605B0F0BD02A9FEF7F1F905460028DA
:1061F800F6D19DF809209DF8083013439DF80A2030
:106208001343A7F636341BD06A4602213046FFF7FF
:10621800B1FD00283BD19DF808302BB1009B03F25B
:106228004E239C42DAD9E41A9DF80A3023B3009B26
:1062380003F2B223B4EB430F4FEA4302CED9A41AB8
:106248009DF80B305BB101AA03213046FFF792FDA0
:10625800019B03F525739C42C0D9C0B9E41A9DF887
:106268000C30002BBCD0A4F2262204213046FFF7C4
:1062780000FE77610546B3E79DF80930002BDFD0B3
:10628800009B03F525739C42A8D9E41AD8E7054674
:10629800A6E770B54FF4FA6286B00023CDE9022371
:1062A80040F636330B600C4604A90646FEF78FF914
:1062B8000546002836D19DF811209DF8103013436B
:1062C8009DF81220134319D002AA02213046FFF785
:1062D80051FD002840D19DF810302BB1029B03F2EC
:1062E8004E222368134423609DF81230EBB1029BC1
:1062F80003F2B222236803EB420323609DF81330B4
:10630800EBB99DF814305BB101AA04213046FFF7C0
:1063180031FD019B03F22622236813442360D8B978
:1063280023687361284606B070BD9DF81130002BB4
:10633800E4D0029B03F5257223681344DDE703AA22
:1063480003213046FFF716FD039B03F525722368EA
:10635800134423600028D4D00546E3E72DE9F7432A
:10636800002406460D46204615F80480B8F1000FB3
:1063780000D010B103B0BDE8F083671CB8F1FF0F7F
:1063880015F8079029D1A71CEB5DB9F1030F36D892
:10639800DFE809F0020B131B271D2C44E27802EBFF
:1063A8000323A6F834313C46DEE7271D2C44E27867
:1063B80002EB0323A6F83631F5E7271D2C44E278D3
:1063C80002EB0323A6F83831EDE7271D2C44E278C9
:1063D80002EB0323A6F83C31E5E7B8F1040F0ED829
:1063E80002344246291901A80DF02DFA434601AAA4
:1063F8004946304604EB080700F0B2FAD3E76FF0DD
:106408000300D0E773B500230E4613600DF10701B2
:1064180005461446FEF712F940B99DF807302BB12E
:10642800B38A2A6A534380331B0A236002B070BDC3
:1064380013B5CB681360144601AAFFF7E3FF18B938
:106448002368019A1344236002B010BDF8B5B0F870
:106458005451D0F8580168438030000A0E4645432D
:10646800DDE90717144652B1B60206EB5202B2FB39
:10647800F4F202EB4202524302F50042140C069A6F
:10648800534301F50042120C06200332B2FBF0F22E
:10649800C2EBC202B2F5803F38BF033103F50043B7
:1064A8003EBFB1FBF0F1C1EBC10101F500414FEA7C
:1064B800134334BF090C1B4903FB03F338BF49439B
:1064C80003EB57030B44B3FBF7F39B03FE2205F1E1
:1064D80020007F33B3FBF2F35C434FF47A7704F583
:1064E800FA748009B4FBF7F42401FFF722F904F5E4
:1064F800FA74BC4228BF4FF4FA63064629BFB4FBBE
:10650800F3F300205B19B4FBF7F428BFB3FBF4F0F6
:10651800FFF70FF9099B864294BF1E6018600020A0
:10652800F8BD00BF0000F0FF2DE9F04F91B005461F
:1065380007930B6908930F46CB680B9393460FAAF2
:10654800FFF776FF0EAA39462846FFF75BFF48BBE0
:106558000F9C95F8E0A0D5F8DC3005934FF47A76D7
:1065680006FB04F101F50041049180340E9909916C
:1065780024F0FF010A910F910499D5F8E4300693AD
:10658800BAF1080F0CBF02230323090C95F8E82081
:10659800DFF898810C9108D1079BCBF80080C5F8EB
:1065A8004081186011B0BDE8F08F06990D93284618
:1065B800FFF7BCFB5246059981462846FFF7B6FB14
:1065C8000D9B5B490C9A814403FB09F94FEAC929E1
:1065D80040F2776309F5FA79240AB9FBF6F903FB67
:1065E80009F909F5FA79B9FBF6F909FB04F404F19C
:1065F8008003089C74430C40B4FBF2F44D4A1B0A18
:10660800944228BF1446012B38BF01230C204FF4B5
:10661800167258435443FFF78CF83B7E3A894FEA89
:10662800400A002B7FD14249049B0B4003F5FA71C5
:10663800414B5A4341F25C23B2FBF3F2099B73438B
:10664800B3F5481F28BF4FF44813A1EB4303B1FB30
:10665800F6F1B3FBF6F31B02B3FBF1F63602C6F50F
:106668008036564306F50046360C06F58036760821
:106678007643B60B4FF44873734303F5004304F5B0
:1066880000401B0C5B43000C00FB0030FFF751F887
:1066980003046422323341F28837B3FBF2F340F645
:1066A800B532B3FBFAF302FB0377244B9F429CBF3E
:1066B80042F21073B7FBF3F7DDE90532134403F533
:1066C800FA734FF47A7A4FF4FA62B3FBFAF0B3FB39
:1066D800F2F202F5C812B2FBF0F088BF4FF470472F
:1066E800FFF727F8000200F5FA70B0FBFAF0404314
:1066F80007FB0700FFF71DF80AFB00F0079B404562
:1067080028BF4046CBF80000C5F84001CDE9029308
:106718004FF448730093DDE90A1201943346284682
:10672800FFF794FE3EE74FF48036A3E7AE878F026B
:106738000000FFFF666666009A9906000F279F24EF
:106748002DE9F04F11F0780F8BB018BF4FF2A00968
:10675800C1F3C30B18BF29FA0BF990469A460DF1FD
:106768000E024FF000034FF00001159F8DF80E3018
:1067780004468DF80F308DF810308DF81130ADF8D3
:106788001230099314BF09F001094FF00109FDF710
:10679800ADFF9DF80E500646D5B1002840F09A800E
:1067A800149909AB05AA2046FFF7BEFE002840F061
:1067B8009380149A099B5381014606AA2046FDF747
:1067C800CAFF069D25B1059B9D422CBF00250125CA
:1067D80020B904AA02212046FDF788FF9DF8106021
:1067E80026B300287AD107AA02212046FDF7B3FF75
:1067F80088B90122FF21204600F0E8F858B90DF1C8
:106808001202B621204600F031F920B90246FF21D4
:10681800204600F0DBF8BDF81230079E5B02C4F892
:1068280048311EB19E422CBF0026012628B90DF121
:10683800110203212046FDF759FF9DF8113093B14D
:1068480000286CD1BAF1000F03D04FEA0828B8FB32
:10685800FAFA08AA03212046FDF77DFF089B534555
:1068680094BF0023012320B9B9F1000F38D0FF22CB
:106878003A703A780AB914994A810DF10F02012148
:1068880020460193FDF732FF08BB9DF80E20019BBF
:10689800002A08BF0125BBF1040F18BF9DF80F207F
:1068A80084F82E501ABFB2FA82F25209012284F8F3
:1068B8002F209DF81020002A9DF8112008BF0126DE
:1068C800002A08BF012384F8306084F831300BB007
:1068D800BDE8F08F002581E735467FE70026ACE765
:1068E8000BF1FF32092A0AD8DFE802F0050505098D
:1068F8000907090B070B0522BAE70422B8E7012E9E
:1069080001D10322B4E7BBF1040F01D0012B01D15F
:106918000222ADE7012D16BF00233D703B70002316
:10692800A7E707B502F10A03009393B20A4690F865
:106938006011D0F85C0101F029FB03B05DF804FB9D
:1069480013B502F10A0390F860410093D0F85C0196
:1069580093B20A4644F0010101F0AEFB02B010BD4B
:106968003F2BF8B50E46054611461C4611D80A4F6E
:1069780038461A4600F8016B0CF065FF621C394670
:106988002846FFF7CEFF002814BF6FF01300002041
:10699800F8BD6FF00300FBE7980E002073B51546AD
:1069A8008DF8071001220DF1070104461E46FFF776
:1069B800B8FF18B16FF0130002B070BD3246294617
:1069C8002046FFF7BDFF0028F6D0F3E708B5064BD1
:1069D80019705A7019460222FFF7A3FF002814BF46
:1069E8006FF01300002008BD980E002008B5074B73
:1069F8001970110A59709A7019460322FFF791FF0E
:106A0800002814BF6FF01300002008BD980E002066
:106A180037B515468DF8071001220DF10701044618
:106A2800FFF77FFF18B16FF0130003B030BD0122EC
:106A380029462046FFF784FF0028F6D0F3E7F7B58C
:106A480015460DF1070206460F461C46FFF7E0FF04
:106A580050B99DF807301D4044EA050239463046D2
:106A68008DF80720FFF7B2FF03B0F0BD73B51446E9
:106A78008DF8071001220DF107010546FFF751FFB8
:106A880018B16FF0130002B070BD064E02223146F5
:106A98002846FFF755FF0028F3D133885BBA2380D7
:106AA800F1E700BF980E002073B514468DF8071063
:106AB80001220DF107010546FFF733FF18B16FF00A
:106AC800130002B070BD064E042231462846FFF777
:106AD80037FF0028F3D133681BBA2360F1E700BF02
:106AE800980E002008B50220FBF7DCFF002008BD47
:106AF8007047000010B5032000F056FC01F028FD97
:106B0800064B18600F20FBF7C3FF044618B9FBF7C4
:106B18004AFE204610BD0124FBE700BF28080020DC
:106B28004FF0E022136923F00203136170474FF01E
:106B3800E022136943F0020313617047014BD3F855
:106B4800900570470070FF1F014BD3F894057047FC
:106B58000070FF1F014BD3F8980570470070FF1FA6
:106B68008068C0F380007047F7B50023019304469E
:106B7800002800F0E980856D25B9FBF769F9E5651E
:106B880084F8545023689A68D00040F1A1809A682C
:106B9800D10000F1B480A26D42F01002A265E26D4E
:106BA80042F00102E26501251846FFF7D9FFA26D00
:106BB80002F01002024340F0C980A26D206922F45D
:106BC800817242F00202A2659A68D2075DD4226BF4
:106BD800A67E94F82CC0003A18BF01221703D4E906
:106BE80002120A43217E42EA8132617E42EAC132C0
:106BF80042EA4632002842EA4C02B4BF20F0004183
:106C08004FF400113A430A4394F82010012903D1A4
:106C1800002E76D142F48032616A21B1A66A01F46D
:106C2800E07131430A43D968E66C21F4FE3121F45E
:106C3800FF711143D96094F83C206168012A01F082
:106C4800404C4CEA060609D1D4E910273A433243AE
:106C5800A66C324342EA0C0242F001061F693E4A22
:106C68003A4032431A6121F00042B2F1804F0CD011
:106C7800B1F1004F09D0394ED6F8082701F4701148
:106C880022F470120A43C6F808275A69666BA16B8A
:106C980022F0070232435A615A6922F0700242EA2E
:106CA80001125A61002835D19A6A62F00F029A627D
:106CB8005B6903F007039E423CD10023E365A36DA3
:106CC80023F0030343F00103A365284603B0F0BD96
:106CD8009A68234922F0104222F0170242F08052AB
:106CE8009A60204A1268B2FBF1F201325200019216
:106CF800019A002A3FF44BAF019A013AF7E70025C1
:106D080052E7A16D41F02001A165E16D41F001015B
:106D1800E16581E7B0F5001FCAD19A6AE269013AD4
:106D280092006FF00F0102F01C0201FA02F2216ECC
:106D38000A43BCE7A36D23F0120343F01003A365D5
:106D4800E36D43F00103E3650125BEE7A36D43F05E
:106D58001003A365F8E700BF02FCFF1F00200140F5
:106D6800400D030028080020F8B54569082D0446A1
:106D78000E460AD00368DB68D80705D5A36D43F033
:106D88002003A3650120F8BD0425FBF783FE074611
:106D980023681A682A4220D0A26D42F40072A265C4
:106DA800DA6812F4406F14D1A27E92B91A681207F9
:106DB8000FD51846FFF7D4FE20BB5A6822F00C0204
:106DC8005A60A26D22F4807222F0010242F00102A0
:106DD800A265227EFAB10020D5E7711CD9D0FBF755
:106DE80059FEC01BB04201D8002ED1D123681B68C0
:106DF8002B40CDD1A26D84F8543042F00402A26534
:106E08000320C0E7A26D42F02002A265E26D42F0C5
:106E18000102E265DDE70C221A60DCE70368186C02
:106E280070470000F7B50023019390F85430012B08
:106E3800044600F0C08005680269012380F85430D8
:106E48002846FFF78DFE002840F0AF80D1E90030DA
:106E5800022822F004027ED0B2F1004FC3F3110ED3
:106E680035D1AA6A42EA0E02AA628A68686902EA09
:106E7800032222F07C4222F0FF0220EA03210A4387
:106E8800002B6A611DDA4D4A4D4DD2F80817AB4206
:106E980001F0E07043D10D0213D4D2F8083723F083
:106EA800E073034343F40003C2F80837454B1A68FC
:106EB800454BB2FBF3F20C2302FB03330193019B16
:106EC80053BB0020002384F8543003B0F0BD226E79
:106ED80000F01F074FF00F0C0CFA07FC6FEA0C06C6
:106EE80022EA0C0CBEF1000F11D1C3F38462BA4040
:106EF80042EA0C0222668008E26901309042B4D866
:106F0800A86AC3F38362BA4006403243ACE793FAF7
:106F1800A3F2B2FA82F2EAE7019B013BCEE72B4DDE
:106F2800AB420BD1C901CCD4D2F8083723F0E073B7
:106F3800034343F08073C2F80837C2E7244DAB42DD
:106F4800BFD14B02BDD4D2F8083723F0E073034316
:106F580043F48003EFE7B2F1004F01BFAA6AC3F31D
:106F680011018A43AA62002BABDA15481349834200
:106F7800D1F8082709D1D1F8083702F0A07223F018
:106F8800E0731A43C1F808279BE71048834204D1ED
:106F9800D1F8083702F44002F1E70D48834290D156
:106FA800D1F8083702F0C072E9E7A26D42F020027A
:106FB800A265184686E7022087E700BF0020014047
:106FC800001000B028080020400D0300004000B861
:106FD800002000B4026838B504461046FFF7C0FD2B
:106FE80008B9002038BD9368990707D4936823F03F
:106FF800004323F0170343F010039360FBF74AFDA7
:10700800054623689B685B07EBD5FBF743FD401BF0
:107018000228F6D923689B685A07F2D5A36D43F076
:107028001003A365E36D43F00103E3650120D9E78D
:1070380073B50023026801939368DD07044602D5FF
:10704800002002B070BD9168214B194209D0A36D90
:1070580043F01003A365E36D43F00103E3650120EA
:10706800EFE7936823F0004323F0170343F001038D
:107078009360184BD3F8083718021CD4637E012B91
:10708800DED0FBF707FD144E054622681368DB07C0
:10709800D6D49368D9075FBF9368334043F00103A0
:1070A8009360FBF7F7FC401B0228EED923681B68A6
:1070B800DA07EAD4CBE7094B094A1B68B3FBF2F3BA
:1070C80001330193019B002BD8D0019B013BF8E7CA
:1070D8001700008000200140E8FFFF7F28080020FB
:1070E800400D030038B504460068FFF739FD054632
:1070F80020BB94F85430012B20D0012384F854305D
:107108002046FFF795FFB0B9A36D226823F470639A
:1071180023F0010343F48073A3651C23E065136027
:1071280084F85400936823F0004323F0170343F0D6
:107138000403936038BD84F85450FBE70220F9E754
:10714800026838B5936891680446C80701D40020DE
:1071580038BD9907FBD4936803F00503012B19D1B7
:10716800936823F0004323F0170343F0020393606E
:1071780003231360FBF78EFC054623689B68DB0737
:10718800E5D5FBF787FC401B0228F6D923689B68E6
:10719800DA07F2D5A36D43F01003A365E36D43F05E
:1071A8000103E3650120D3E770B5044600284BD0FE
:1071B800836D43F002038365FFF70CFF054668B94A
:1071C8002046FFF7BDFF054608B90123A3652268DD
:1071D800936823F0104323F01703936023685A68D9
:1071E80022F4677222F003025A6040F29F321A605A
:1071F800D968164A0A40DA601A6922F040421A61D0
:107208005A6922F007025A611A6A02F0F0221A62D9
:107218005A6A02F0F0225A62DA6A02F0F022DA625E
:107228009A6A0B4A00269E62D2F8083723F0FE734A
:10723800C2F808372046FAF739FEE6652666A665DD
:1072480084F85460284670BD0125FBE700023E83A0
:107258000020014010B590F85430012B044615D099
:10726800012380F85430FFF7B5FE58B92046FFF7E0
:1072780067FF38B9A36D23F4807323F0010343F04B
:107288000103A365002384F8543010BD0220FCE7F5
:10729800F7B50023019390F85430012B04467FD0B2
:1072A800012380F85430FFF74BFF23689A6812F0E7
:1072B8000102054607D0A36D43F01003A365002320
:1072C80084F854302DE0A16D364F21F4817141F0DE
:1072D8000201A165DE68D96826F4FF4626F07C061F
:1072E80021F40041360421F00301360CD96008204E
:1072F8009968394041F0004199609968002913DA8A
:107308000199013101910199B1F52E3FF5D3A36D92
:1073180023F0120343F01003A365002384F85430CC
:107328000125284603B0F0BDD3F8B410013801F0A8
:107338007F010A44DCD199681A48014041F00101F3
:107348009960D3F8B41021F07F0141EAD202C3F862
:10735800B4209A68024042F002029A60FBF79AFB56
:10736800074623689A68D20708D4DA683243DA6095
:10737800A36D23F0030343F001039FE7FBF78AFBA8
:10738800C01B0228EDD923689B68D907E9D5A36DEE
:1073980043F01003A365E36D43F00103E365BFE722
:1073A8000225BEE7E8FFFF7F0749CA6822F4E062CA
:1073B8000302120403F4E063120C134343F0BF63A7
:1073C80043F40033CB60704700ED00E0164B30B556
:1073D800DC68C4F30224C4F10703251D042B28BF6D
:1073E8000423062D4FF0FF358CBF033C002405FA1B
:1073F80003F321EA0303A54022EA0502A34000287B
:1074080043EA0203ACBF00F16040084A4FEA0313A5
:10741800B8BF00F00F00DBB2AABF00F561401354FB
:1074280080F8003330BD00BF00ED00E014ED00E04F
:10743800002807DB044A4109012300F01F008340AC
:1074480042F82130704700BF00E100E000280CDB63
:107458004309064900F01F0020330122824041F809
:107468002320BFF34F8FBFF36F8F704700E100E019
:1074780070B5D0E913456560446D14B1D0E916457F
:107488006560D0E9105404F01C060124B4406C6017
:10749800046863608368102B0BBFA260A160E16081
:1074A800E26070BD0268416CD3B210B5083B142489
:1074B800B3FBF4F30B4CA24288BF0B4A21F0030143
:1074C80099BF01F1804202F50232521807338264F3
:1074D800064AC26403F01F03012202FA03F303659C
:1074E80010BD00BF070402401C080240800802408B
:1074F80038B500285CD002682E4B9A424FF0140130
:107508004AD82D4B1344B3FBF1F32C499B00C0E937
:107518001013022380F825301368056923F4FF430C
:1075280023F070031360D0E9024323432B434569DA
:1075380011682B4385692B43C5692B43056A2B4387
:107548000B431360FFF7AEFFB4F5804F04BF002371
:1075580043604368816C03F07F020A60D0E913142A
:10756800013B032B4C601ED8154B1649816513440B
:107578009B000121013A01FA02F200214365C2652C
:107588001960114B5A6400230122C36380F8243028
:1075980080F82520184638BD0C4B1344B3FBF1F393
:1075A8000B499B00B3E70023C0E91533C365EAE73D
:1075B8000120F0E707040240F8FFFDBF0000024089
:1075C8003F8200104009024000090240F8FBFDBF5D
:1075D8000004024038B5002841D00268136823F03F
:1075E800010313601F4B9A424FF0140130D81E4B11
:1075F8001344B3FBF1F31D499B00C0E910130124A8
:1076080003F01C0304FA03F3002515604B60FFF731
:1076180049FF836C41681D60D0E913325A604A1EE5
:10762800032A06D8124B0B449B0094401D60114B53
:107638005C640023C363C0E91533C0E90B33C0E9B8
:107648000D33C36580F8253080F82430184638BDDE
:10765800094B1344B3FBF1F308499B00CDE7012024
:10766800F5E700BF07040240F8FFFDBF0000024035
:107678003F82001000090240F8FBFDBF00040240F1
:1076880070B590F82450012D04463BD090F8256041
:107698000125AE4280F824504FF000062CD1022577
:1076A80080F825500568C6632E6826F001062E600E
:1076B800FFF7DEFE036BBBB12B6843F00E032B60B4
:1076C800A36C1A68D20342BF1A6842F480721A6027
:1076D800636D1BB11A6842F480721A602B6843F01C
:1076E80001032B60002070BD2B6823F004032B607E
:1076F8002B6843F00A03E2E78023C36380F8246021
:107708002846F0E70220EEE770B4426C046C036888
:1077180026681D6802F01C020421914031420FD0F6
:1077280015F0040F0CD01A6892065EBF1A6822F092
:1077380004021A60036B6160002B33D070BC1847D9
:1077480002219140314217D015F0020F14D01A6867
:10775800940606D41A6822F00A021A60012280F8F8
:107768002520114A93428CBF104B114B59600023BE
:1077780080F82430C36ADFE708219140314211D0F4
:1077880029070FD5196821F00E011960012303FAA2
:1077980002F26260C36380F82530002380F8243049
:1077A800436BC9E770BC7047800002400004024088
:1077B800000002400A4A536943F4802330B55361FC
:1077C800EFF3108472B60023CD58C5500433B3F5D7
:1077D800807FF9D11369DB03FCD484F3108830BDB2
:1077E80000400058064B5A69002ABFBF054A9A60F4
:1077F80002F188329A60BABF5869C00F00207047FA
:107808000040005823016745044B5A6942F0004282
:107818005A615869C043C00F704700BF0040005804
:1078280070B50546FBF736F9124E04463369D9039D
:1078380013D43369DA0744BF012232614CF2FA32B9
:10784800134011D10B4E306910F480200BD0FBF798
:1078580021F9001BA842F6D304E0FBF71BF9001B33
:10786800A842E3D3032070BD024A1361024A0120F3
:107878005360F8E700400058D80E00202DE9F04189
:10788800184D98462B78012B06460C46174626D0ED
:1078980001232B704FF47A7000236B60FFF7C0FF51
:1078A800A0B9012E16D1104A536943F00103536160
:1078B8002760BFF36F8FC4F804804FF47A70FFF726
:1078C800AFFF094A536923EA0603536100232B706B
:1078D800BDE8F08139462046FFF76CFFEDE702204E
:1078E800F6E700BFD80E002000400058054A53694B
:1078F80023F47E7343EAC00040F4803040F0020075
:1079080050617047004000582DE9F041234F3B7803
:10791800012B054688463FD001233B704FF47A700F
:1079280000237B60FFF77CFF044688B92B68042B93
:1079380013D11B4A536943F4803343F00403536162
:107948004FF47A70FFF76CFF0446154B1A681B68F2
:1079580000233B702046BDE8F0814FF0FF33C8F8A4
:1079680000306E68D5E901321344B3420AD9304673
:10797800FFF7BCFF4FF47A70FFF752FF50B1C8F819
:1079880000600446064A536923F47E7323F0020319
:107998005361DAE70136E5E70224DBE7D80E002079
:1079A800004000582DE9F04F524C00234FF00F09CA
:1079B8000A6832FA03F501D1BDE8F08F012505FA0E
:1079C80003F818EA020200F08E804E68032706F0DA
:1079D80003054FEA430E07FA0EFC6F1E012F6FEAEC
:1079E8000C0C32D8876807EA0C0ACF6807FA0EF73A
:1079F80047EA0A078760476827EA0808C6F30017B6
:107A08009F4047EA08074760C76807EA0C088F687D
:107A180007FA0EF747EA0807022DC76017D14FEAA1
:107A2800D30800EB880803F0070AD8F820704FEA5B
:107A38008A0A09FA0AFB27EA0B0B0F6907FA0AF701
:107A480047EA0B07C8F8207001E0032DDCD107686E
:107A580005FA0EF507EA0C073D4316F4403F0560AA
:107A680041D023F0030707F1804707F5803703F07B
:107A7800030CBD684FEA8C0C4FF0070E0EFA0CFE93
:107A8800B0F1904F25EA0E0E2FD01B4DA8422ED0F4
:107A980005F58065A84214BF0725022505FA0CF5EF
:107AA80045EA0E05BD602568D74316F4801F0CBF54
:107AB8003D4015432560656816F4001F0CBF3D4026
:107AC80015436560D4F8805016F4803F0CBF3D40E4
:107AD8001543C4F88050D4F88450B60354BF3D40D1
:107AE8001543C4F88450013362E70025D6E7012521
:107AF800D4E700BF0008005800040048374A2DE9C1
:107B0800F04F00234FF0010A4FF0070B4FF00F0919
:107B180031FA03F401D1BDE8F08F0AFA03FC1CEA3C
:107B2800010654D023F0030404F1804404F58034A2
:107B380003F00307A568BF000BFA07F8B0F1904FF0
:107B480008EA050E45D0264DA84244D005F58065C3
:107B5800A8420CBF02250725BD40754517D1D2F8AC
:107B6800805025EA0605C2F88050D2F8845025EAEC
:107B78000605C2F88450156825EA0605156055689B
:107B880025EA06055560A56825EA0805A560056883
:107B980003265C0006FA04F423FA06F6254300EBF4
:107BA8008606056003F00705376AAD0009FA05F592
:107BB80027EA05073762856825EA04058560456870
:107BC80025EA0C054560C56825EA0404C46001334C
:107BD8009EE70025C0E70125BEE700BF0008005862
:107BE800000400480369194214BF012000207047AF
:107BF8000AB18161704781627047436901EA0302F3
:107C080021EA030141EA024181617047044AD168CF
:107C1800014208B502D0D060FBF7D4FB08BD00BF15
:107C28000008005803689A69910744BF00229A62C5
:107C38009A69D2075EBF9A6942F001029A61704759
:107C480030B5039D04682B4343EA0243064A606843
:107C5800C1F309010B4342EA555223F0004320EADD
:107C680002000343636030BDFF63FF0303682DE92F
:107C7800F0419C6914F0100405460F4616466FD073
:107C880010220024DA61A0462B689A69900661D414
:107C9800B8F1000F35D044F0040401202E68B36910
:107CA800D90541BF4FF48072F26144F0010401200C
:107CB8005A0541BF4FF4806244F00804F261012084
:107CC8009B054FD54FF4007344F00204F361284636
:107CD800FFF7A8FF736823F0FF7323F48B3323F4B3
:107CE800FF7323F0010373606B6C23436B642023E1
:107CF80085F84130002385F8423085F8403001206E
:107D080032E07A1CC1D0FAF7C5FE801BB84201D810
:107D1800002FB9D12B68596895F84220986900045A
:107D2800D2B20AD5490408D4202A06D05A6842F4A7
:107D380080425A60FAF7AEFE06462B689B699B069E
:107D4800A2D4FAF7A7FE801B1928F6D920244FF0F1
:107D5800010899E7B8F1000F9DD12022DA619AE76E
:107D680020469BE70028B2D1BDE8F08170B50446F3
:107D78000D46164623689B699B0701D500201BE02A
:107D8800324629462046FFF771FFA0B96A1CF1D098
:107D9800FAF780FE801BA84201D8002DEAD1636C57
:107DA80043F020036364202384F84130002384F8DF
:107DB800423084F84030012070BD70B504460D464D
:107DC800164623689B699B0601D5002019E03246B8
:107DD80029462046FFF74AFF90B9FAF75BFE801B59
:107DE800A84201D8002DECD1636C43F020036364F2
:107DF800202384F84130002384F8423084F840304E
:107E0800012070BD70B504460D46164623689B696F
:107E18005B070ED4324629462046FFF727FF38BBBA
:107E280023689A69910625D59A69520703D5228D48
:107E38000AB1002070BD9A6912F010021CBF10220E
:107E4800DA614FF0200118BF04226264D9615A68D0
:107E580022F0FF7222F48B3222F4FF7222F0010228
:107E68005A60002384F8411084F8423084F8403086
:107E78000120DFE7FAF70EFE801BA84201D8002D8B
:107E8800C4D1636C43F020036364202384F8413039
:107E98000023EBE72DE9F041069F04468846164685
:107EA8001D462268936938EA03030CBF01230023A7
:107EB800B34201D0002015E06B1CF3D0FAF7EAFDBD
:107EC800C01BA84201D8002DEBD1636C43F02003FE
:107ED8006364202384F84130002384F8423084F816
:107EE80040300120BDE8F08110B5044600284AD092
:107EF80090F8413003F0FF021BB980F84020FAF7F0
:107F0800BBFA242384F8413023681A6822F001025E
:107F18001A60626822F070621A619A6822F400425C
:107F28009A60D4E90221012924D142F400429A60DE
:107F38005A6842F0007242F400425A60DA6822F449
:107F48000042DA60D4E904210A43A16942EA012225
:107F5800DA60D4E907210A431A601A6842F001027C
:107F68001A6000202023606484F84130206384F87C
:107F7800420010BD42F4044202299A6004BF4FF443
:107F880000625A60D4E70120F3E700002DE9F347C7
:107F9800984690F841300A9F202B04460E46914699
:107FA80040F0868090F84030012B00F081804FF03F
:107FB800010A80F840A0FAF76DFD192305460090E4
:107FC80052464FF400412046FFF764FF18B10120E4
:107FD80002B0BDE8F087212384F84130102384F8EB
:107FE80042306064A4F82A80638DC4F824909BB260
:107FF800FF2B60632F4B26D9FF22228500934FF079
:10800800807331462046FFF71BFE638D9BB22A46DC
:1080180039462046FBB9FFF7D0FE0028D7D12368A0
:108028002021D9615A6822F0FF7222F48B3222F49F
:10803800FF7222F001025A6084F8411084F840006F
:1080480084F84200C4E7628D92B2228500934FF013
:108058000073D2B2D5E7FFF789FE0028B7D1636A6B
:10806800226813F8011B91626362638D228D013BC4
:108078009BB26385638D013A92B29BB22285002B35
:10808800C3D0002AC1D100953B4680212046FFF786
:1080980001FF00289BD1638D9BB2FF2B03D9FF22E0
:1080A80022850090ABE7628D92B222850090CEE7E0
:1080B80002208DE7002000802DE9F347984690F8CC
:1080C80041300A9F202B04460E46914640F0878097
:1080D80090F84030012B00F082804FF0010A80F8C0
:1080E80040A0FAF7D7FC19230546009052464FF4F2
:1080F80000412046FFF7CEFE18B1012002B0BDE8CE
:10810800F087222384F84130102384F842306064D9
:10811800A4F82A80638DC4F824909BB2FF2B606377
:10812800304B26D9FF22228500934FF080733146C9
:108138002046FFF785FD638D9BB22A4639462046C7
:10814800FBB9FFF73AFE0028D7D123682021D9616F
:108158005A6822F0FF7222F48B3222F4FF7222F066
:1081680001025A6084F8411084F8400084F8420003
:10817800C4E7628D92B2228500934FF00073D2B2A9
:10818800D5E7FFF73FFE0028B7D123685A6A636A2C
:108198001A70636A228D01336362638D013B9BB25F
:1081A8006385638D013A92B29BB22285002BC2D0BF
:1081B800002AC0D100953B4680212046FFF76AFE81
:1081C80000289AD1638D9BB2FF2B03D9FF22228509
:1081D8000090AAE7628D92B222850090CDE7022036
:1081E8008CE700BF0024008010B590F84120202AB9
:1081F8000346D4B21CD190F84020012A18D024227A
:1082080080F841200268106820F0010010601068B2
:1082180020F480501060106801431160116800203C
:1082280041F00101116083F8414083F8400010BD1E
:108238000220FCE710B590F84120202A0346D4B26A
:108248001BD190F84020012A17D0242280F8412021
:108258000268106820F001001060106820F4706057
:1082680040EA012111601168002041F0010111600C
:1082780083F8414083F8400010BD0220FCE700006D
:10828800024A136843F4807313607047000400586F
:108298000D4B10B55B690C4628B99A0507D500F057
:1082A80027F820B110BD9B0501D400F019F8074A42
:1082B8001369012C23F00403136101D130BFF1E7E6
:1082C80040BF20BF20BFEDE70004005800ED00E0EC
:1082D800024B186800F4C060704700BF00040058E3
:1082E800024A136843F4804313607047000400583F
:1082F8000C4A136823F4804313600B4B1B6832212C
:108308004B430A49B3FBF1F35169890500D533B9E9
:10831800536913F4007F14BF032000207047013B0A
:10832800F2E700BF000400582808002040420F0070
:108338000B4A136823F0070343F002031360094B49
:108348001A69012842F004021A6105D130BF1A697E
:1083580022F004021A61704740BF20BF20BFF6E731
:108368000004005800ED00E04FF0B0431868C0F377
:10837800404070474FF0B0431868C0F34000704762
:108388004FF0B042536823F47F4343EA002353601D
:1083980070474FF0B0431868C0F340607047000062
:1083A8007FB54FF0B0432C4AD3F80831C0F303101F
:1083B80003F00F0352F82040284A52F82330B4FB48
:1083C800F3F4FFF785FF264B054693E80700B5F55C
:1083D800007F04AB03E9070010D0224B9C4218D35E
:1083E80003F5B70303F67F539C4229D903F57413A9
:1083F80003F510639C4225D802230BE01A4B9C42DC
:1084080007D91A4B9C421BD903F5370303F5D853F8
:10841800F0E7002304AA02EB830353F80C4C144D35
:108428002B6823F0070323432B60FAF733FB064638
:108438002B6803F007039C4206D1002004B070BDEE
:108448000123E7E70024EAE7FAF724FB801B022868
:10845800EED90320F2E700BFE83A0108483B0108DB
:1084680090390108C0CF6A00BFEA21013F93340266
:10847800004000584FF0B04310B59A68D96812F020
:108488000C0205D00C2A4AD101F00303012B51D16B
:108498004FF0B0412B480B6813F0080306D00B6867
:1084A80013F0080337D1D1F8941007E00C682407BB
:1084B80056BFD1F894300968C3F3032350F823302A
:1084C800002A0CBF184600204FF0B0418A6802F01D
:1084D8000C020C2A1ED1CA6802F00302022A2ED00E
:1084E800032A06D10B68184A13F4801F174B18BFCC
:1084F80013464FF0B042D068D168D268C0F3062066
:108508005843C1F302130133B0FBF3F0530F0133A7
:10851800B0FBF3F010BD0B68C3F30313CEE7042AD6
:1085280005D0082A06D11B6813F4801305D0064825
:108538000023C9E700231846C6E70448C4E7024BEE
:10854800D7E700BFE83A01080024F4000048E80132
:1085580008B5FFF78FFF4FF0B043044A9B68C3F399
:10856800031352F82330B0FBF3F008BD483B010871
:108578002DE9F0410446002853D04FF0B0439D68E0
:10858800DE6803689B0605F00C0506F0030668D54F
:10859800026A1DB10C2D46D1012E44D1002A40D0CB
:1085A8004FF0B043A16A1A68170756BFD3F8943042
:1085B8001B681B0903F0F00399421FD90846FFF70F
:1085C800EFFE00282DD14FF0B042136843F00803A6
:1085D80013601368A16A23F0F0030B431360606A09
:1085E800FFF7CEFEFFF7B4FFAB4B1860AB4B186834
:1085F800FAF74EFA002834D0BDE8F0814FF0B042C7
:10860800136843F008031360136823F0F0030B4367
:108618001360606AFFF7B4FE0846FFF7C1FE002842
:10862800E0D00120E8E74FF0B043002A54D01A68A0
:1086380042F001021A60FAF72DFA0746FFF79AFE90
:10864800002842D04FF0B042136843F0080313608B
:108658001368A16A23F0F0030B431360606AFFF705
:108668008FFE2368D80748D42368990700F18C80C7
:1086780023681E0740F1FA80A3694FF0B046002B2B
:1086880000F0E180D6F89430E16903F010029142DD
:1086980000F0C48003F00302022AC2D0D80740F1D8
:1086A800B380D6F8943023F00103C6F89430FAF773
:1086B800F1F90746D6F89430990740F1A580FAF702
:1086C800E9F9C31B112BF5D904E0FAF7E3F9C01B4C
:1086D8000228B3D903208FE71A6822F001021A6032
:1086E800FAF7D8F90746FFF745FE0028B9D0FAF798
:1086F800D1F9C01B0228F6D9ECE7082D03D00C2DC0
:1087080005D1032E03D16368002BADD189E74FF063
:10871800B043A1681A6822F480120A431A6062689A
:10872800B2F5803F10D11A6842F480321A60FAF725
:10873800B1F90746FFF718FE002895D1FAF7AAF90C
:10874800C01B6428F6D9C5E7B2F5041F04D11A681E
:1087580042F400121A60E6E7196821F480311960C2
:10876800196821F400111960002AE0D1FAF792F98A
:108778000746FFF7F9FD00283FF476AFFAF78AF9C4
:10878800C01B6428F5D9A5E7042D236903D00C2D57
:108798000ED1022E0CD1002B3FF443AF4FF0B04264
:1087A8006169536823F0FE4343EA016353605FE75E
:1087B8004FF0B046BBB1336843F480733360FAF7C7
:1087C80069F9074633685A0505D4FAF763F9C31BF4
:1087D800022BF7D97EE77368626923F0FE4343EA08
:1087E8000263736044E7336823F480733360FAF7F5
:1087F80051F9074633685B057FF53AAFFAF74AF94E
:10880800C31B022BF6D965E74FF0B042E169D2F8F5
:10881800943023F010030B43C2F894304FF0B04764
:10882800D7F8943043F00103C7F89430FAF732F9D7
:108838000646D7F894309A0718D4FAF72BF9831B11
:10884800112BF6D946E7D6F8943023F00103C6F881
:108858009430FAF71FF90746D6F894309B0705D5E8
:10886800FAF718F9C31B112BF6D933E72368580711
:1088780054D50B4F3B68D90514D4FFF701FDFAF71F
:1088880009F906463B68DA050CD4FAF703F9831BA5
:10889800022BF7D91EE700BF280800202C0800206B
:1088A80000040058E3684FF0B046002B58D023F07E
:1088B8008003052B02BFD6F8903043F00403C6F8B6
:1088C80090304FF0B046FAF7E5F8D6F8903043F01C
:1088D80001030746C6F8903041F28838D6F8903040
:1088E8009B0705D4FAF7D6F8C31B4345F6D9F1E63A
:1088F800E36823F00403812B1BD1FAF7CBF8D6F8F1
:10890800903043F08003C6F8903007464FF0B046E9
:1089180041F28838D6F89030180504D5E36A002B60
:108928004AD1002068E6FAF7B5F8C01B4045F1D9EE
:10893800D0E6FAF7AFF8D6F8903023F08003C6F8FF
:10894800903007464FF0B04641F28838D6F890305C
:108958001905E3D5FAF79EF8C01B4045F6D9B9E6E4
:10896800FAF798F8D6F8903023F080030746C6F84F
:10897800903041F28838D6F890301A0516D4FAF7B4
:1089880089F8D6F8903023F00103C6F890300746EE
:108998004FF0B04841F28836D8F890309B07BDD5E3
:1089A800FAF778F8C31BB342F6D993E6FAF772F8E8
:1089B800C01B4045DFD98DE60C2D4ED0022B4FF061
:1089C800B0431A6822F080721A6033D1FAF762F85D
:1089D8000546FFF7DEFC38BBD4E90C314FF0B04256
:1089E8000B43D0682D4901400B43E16B0B43216CCD
:1089F8000B43616C0B43A16B43EA0123D3601368FB
:108A080043F080731360D36843F08053D360FAF760
:108A180041F80446FFF7BDFC002882D1FAF73AF87E
:108A2800001B0A28F6D955E6FAF734F8401B0A283D
:108A3800CFD94FE6FAF72EF80446FFF7AAFC30B96B
:108A48004FF0B042164BD1680B40D36069E7FAF794
:108A580021F8001B0A28F0D93CE6012B3FF4E1ADD0
:108A68004FF0B043D868236B00F003029A427FF4BA
:108A7800D8AD626B00F0700393427FF4D2ADA26B65
:108A880000F4FE43B3EB022F7FF4CBAD636C00F030
:108A98006040C01A18BF0120AEE500BF8C80C1112C
:108AA800FCFFFEEE2DE9F0410D46044610B9012009
:108AB800BDE8F081684E336803F007038B4216D394
:108AC80023689A0727D54FF0B047A268BB6823F000
:108AD800F0031343BB60F9F7DDFF0646BB68DB0311
:108AE80019D4F9F7D7FF831B022BF7D911E03368A4
:108AF80023F007030B433360F9F7CCFF07463368CD
:108B080003F00703AB42DBD0F9F7C4FFC01B022810
:108B1800F5D90320CCE72368580617D54FF0B0479E
:108B28006269D7F8083123F00F0343EA1213C7F834
:108B38000831F9F7AFFF0646D7F80831D90305D44D
:108B4800F9F7A8FF831B022BF6D9E2E723685A0737
:108B580013D54FF0B047E268BB6823F4E0631343D2
:108B6800BB60F9F797FF0646BB689B0305D4F9F786
:108B780091FF831B022BF7D9CBE72368180714D57D
:108B88004FF0B0472269BB6823F4605343EAC2033D
:108B9800BB60F9F77FFF0646BB68590305D4F9F7B0
:108BA80079FF831B022BF7D9B3E72368DA070FD4C1
:108BB800294C236803F00703AB4239D8FFF7C8FCF8
:108BC800264B1860264BBDE8F0411868F9F760BFDE
:108BD8006268022A1DD1FFF7C7FB00283FF467AF80
:108BE8004FF0B04641F28838B36823F003031343CB
:108BF800B360F9F74FFF0746B368626803F00C03E8
:108C0800B3EB820FD4D0F9F745FFC01B4045F3D929
:108C18007FE7032A02D1FFF7BCFBDEE712B9FFF7B3
:108C2800A9FBDAE74FF0B0431B685B05D8D43EE7F1
:108C3800236823F007032B432360F9F72BFF06462D
:108C4800236803F00703AB42B8D0F9F723FF801B72
:108C58000228F5D95DE700BF004000582808002029
:108C68002C08002008B5FFF773FC4FF0B043044A06
:108C78009B68C3F3022352F82330D84008BD00BFD5
:108C8800283B010808B5FFF763FC4FF0B043044ADE
:108C98009B68C3F3C22352F82330D84008BD00BFF5
:108CA800283B01084FF0B043D3F89000C0F34000D0
:108CB80070474FF0B0410209D1F8883002F47F22A2
:108CC800000123EA020300F47F200343C1F888303F
:108CD80070474FF0B041020CD1F88830120423EAF3
:108CE800020343EA0040C1F8880070470368DA03CA
:108CF80070B5044639D5FFF7C3FAF9F7CBFE614ED4
:108D080005463368DB0532D54FF0B043616BD3F8C5
:108D1800902002F4407291421DD0D3F89010D3F8FD
:108D2800902042F48032C3F89020D3F8902021F4A8
:108D3800407022F480328D07C3F89020C3F8900069
:108D480009D5F9F7A7FE41F288360546FFF7AAFFCD
:108D5800012840F090804FF0B042616BD2F890301B
:108D680023F440730B43C2F89030002605E0F9F76E
:108D780091FE401B0228C4D903262568E8070AD5B6
:108D88004FF0B0416268D1F8883023EA124392B2BA
:108D98001343C1F88830A9070AD54FF0B041A2683B
:108DA800D1F8883023EA124392B21343C1F88830CD
:108DB800AA0609D54FF0B0422169D2F8883023F4C9
:108DC80040630B43C2F88830AB0502D5206AFFF731
:108DD80080FF680502D5606AFFF77BFF290502D589
:108DE800A06AFFF776FF6A0602D56069FFF761FFA0
:108DF8002B0602D5A069FFF75CFFE80502D5E069FC
:108E0800FFF757FFE90610D54FF0B042E168D2F8F6
:108E1800883023F440730B43C2F88830B1F5807F63
:108E280002BFD36843F08073D3602A040ED54FF095
:108E3800B042216BD2F8883023F040430B43C2F88C
:108E4800883019B9D36843F08073D3606B0410D5A8
:108E58004FF0B042E16AD2F8883023F040530B4318
:108E6800B1F1005FC2F8883003D1D36843F480338E
:108E7800D360304670BDF9F70DFE401BB0427FF657
:108E880065AF79E70004005830B590F82C30012B15
:108E980002464FF0020022D0174B82F82D00CA2458
:108EA800012582F82C505C6253245C62B1F5807F06
:108EB800146B996914D121F488519961596C24F083
:108EC800010421F0004159641463DD650A4BFF2158
:108ED80059620020012382F82D3082F82C0030BD21
:108EE80021F408519961D96C24F0020421F0004161
:108EF800D9641463D865E9E70028004070B50B4EC3
:108F0800036B756D1D40EA07044603D50123F3651D
:108F1800F9F7D3FEAB0704D50223F365204600F02A
:108F2800C9F9012384F82D3070BD00BF0028004026
:108F380038B50A4CE36823F02003E360F9F7AAFD8B
:108F48000546E3689B0601D5002038BDF9F7A2FD68
:108F5800401BB0F57A7FF4D90320F6E700280040DB
:108F6800F8B5114DEC6814F0400406461AD1EB68C8
:108F780043F08003EB60F9F78DFD23460746EC6864
:108F880014F0400401D1032B01D11846F8BDF9F7BC
:108F980081FDC01BB0F57A7F234684BF032386F882
:108FA8002D30ECE70023F0E70028004038B50F4CDF
:108FB800E36823F08003E360A3699B06054606D4B3
:108FC800FFF7B6FF10B1032085F82D0038BDA3695F
:108FD80023F02003A361FFF7ABFF10B1032085F84E
:108FE8002D00A36943F02003A361EFE700280040A8
:108FF80038B5044600284BD090F82D3003F0FF0216
:109008001BB980F82C20F9F749FB0223214D84F87D
:109018002D30EB68DB0636D4CA236B6253236B62B0
:109028002046FFF79DFF10B1FF236B6238BDAB6987
:1090380023F08E6323F04003AB6121696368AA695A
:109048000B431343A2691343AB61D4E9022343EAF8
:1090580002432B61D4E90931EA680B4322F4F85240
:109068001343EB602046FFF7A1FF0028DCD1D4E9C9
:109078000713AA690B4322F0604213436269134342
:10908800AB61FF236B62012384F82D300020CDE70C
:109098000120CBE7002800400023092803D840EA34
:1090A8000310C0B270470A380133C0B2F5E70000B8
:1090B8002DE9F04790F82C30012B05464FF00200BF
:1090C80069D0012385F82C304E4B85F82D00DE68D9
:1090D80006F44076B6F5807F78D04C69087891F828
:1090E800019091F802A091F82470002A55D19B694B
:1090F80013F0400308BFCB70FFF7CEFF8046484609
:10910800FFF7CAFF02465046FFF7C6FF81463846BA
:10911800FFF7C2FF0B6ACF78234343EA875343EA3A
:10912800090343EA084343EA022343EA0063354A52
:10913800CA205062532050628C6A8869B4F5807FD7
:10914800946945D124F4885494610124D465B6F512
:10915800807F09BFCB6913640343536418BF50640D
:10916800284B4A681A672A6B42F001022A639A69F7
:1091780042F488529A61244AD2F8803043F400338A
:10918800C2F880301F4BFF225A620020012385F865
:109198002D3085F82C00BDE8F087B4F1803F07D06A
:1091A800B4F5000F04D09B6913F0400308BFCB70DF
:1091B8000B6ACA781C4344EA0A0444EA004343EAB7
:1091C800092343EA825343EA0763B0E70023AEE783
:1091D80024F4085494610224D465B6F5807F09BF4D
:1091E800CB6993640343D36418BFD064054B4A68C2
:1091F8005A672A6B42F002022A639A6942F40852BB
:10920800B8E700BF002800400008005890F82C205C
:10921800012A03464FF0020012D00A4A83F82D00B3
:10922800CA21516253215162916941F02001916133
:10923800FF2151620020012283F82D2083F82C00A1
:10924800704700BF0028004090F82C20012A0346F0
:109258004FF0020019D00D4A83F82D00CA2151623F
:109268005321516291690A4841F080019161D0F817
:10927800801041F48021C0F88010FF215162002045
:10928800012283F82D2083F82C0070470028004025
:1092980000080058064B5A6D520610B5044603D50F
:1092A8004022DA65F9F70CFD012384F82D3010BD52
:1092B800002800407047890001F1804101F53141E3
:1092C8000A607047890001F1804101F53141086861
:1092D80070470000034AD2F8903043F40043C2F8C4
:1092E8009030704700040058034AD2F8903023F4B5
:1092F8000043C2F89030704700040058074B1A68C2
:1093080022F040021A6040F441704FF4B8521860DD
:109318005A601A6842F040021A607047000001580B
:1093280037B5054600284ED0837903F0FF046BB1AA
:10933800032C0BD0254B4FF400629A612868FFF785
:10934800DDFF002401232B71AC602FE000236B713B
:109358002846F9F7B9FA1E4AD2F8903043F48053F8
:10936800C2F89030002CE5D102234FF0B042AB7127
:10937800D2F8943023F40043C2F89430154B1B689C
:109388001C214B43DB0C64214B430193019B93B994
:109398000124AC60FFF79EFF0C4B9A6842F4006210
:1093A8009A604FF400629A61002CC7D00123AB7118
:1093B800204603B030BD019B013B0193D2F89430A5
:1093C8005B04E3D4E6E70124F2E700BF0004005899
:1093D800000800582808002037B5174D2B680246AA
:1093E8001C204343DB0C6420434314480193019B36
:1093F80093B901209060114C21732B681C214B43B9
:10940800DB0C64214B430193019B6BB901209060F5
:109418000A4BDB6803B030BD019B013B01938368B5
:109428009C07E4D50020E6E7019B013B0193A36874
:10943800DB07E9D5ECE700BF280800200000015849
:1094480037B5184D2B6802461C204343DB0C6420BB
:10945800434315480193019BA3B901209060124C26
:10946800FF2323732B681C256B43DB0C64256B439C
:109478000193019B73B9012090600B4BDB680B7063
:1094880003B030BD019B013B019383689C07E2D583
:109498000020E4E7019B013B0193A368DB07E8D5C3
:1094A800EBE700BF28080020000001580E4B0F49C9
:1094B8001B681822534382B01B0D64225343019347
:1094C8004B69019AC3F3800322B902238360012008
:1094D80002B07047019A013A01924A69920701D590
:1094E800002BEDD10020F3E72808002000040058E5
:1094F80007B50379012B0FD10A4B1B681822534378
:109508001B0C0193FFF7F0FE019B013B0193019BAC
:10951800002BF9D1FFF7DEFE03B05DF804EBFFF78F
:10952800C5BF00BF28080020F8B51E468379012B67
:10953800154604460F46DAB22DD14379012B2AD0BD
:10954800022342718371FFF7D3FF0D212046FFF7F5
:10955800CBFEFFF741FF390A2046FFF73DFFF9B27E
:109568002046FFF739FF2E44B5420ED12046FFF7BB
:10957800B1FEFFF79BFFA06801230038A3714FF0ED
:10958800000318BF01206371F8BD15F8011B2046C0
:10959800FFF722FFE8E70220F6E7F8B51E468379D1
:1095A800012B154604460F46DAB22FD14379012B19
:1095B8002CD04271FFF79CFF1D212046FFF794FE37
:1095C800FFF70AFF390A2046FFF706FFF9B22046DF
:1095D800FFF702FF00212046FFF7FEFE2E44B542AA
:1095E8000ED12046FFF776FEFFF760FFA068012343
:1095F8000038A3714FF0000318BF01206371F8BD54
:1096080029462046FFF71CFF0135E8E70220F6E768
:10961800F8B51F468379012B154604460E46DAB283
:109628002CD14379012B29D04271FFF761FF06F055
:10963800EF03A3F18402534253412371314620467C
:10964800FFF752FEFFF7C8FE2F44AF4210D1FFF7D5
:1096580041FE842E02D02046FFF728FFA068012390
:109668000038A3714FF0000318BF01206371F8BDE3
:1096780015F8011B2046FFF7AFFEE6E70220F6E7E4
:10968800F8B51E468379012B154604460F46DAB213
:1096980027D14379012B24D04271FFF729FF39469E
:1096A8002046FFF721FEFFF797FE00212046FFF72F
:1096B80093FE2E44B5420ED12046FFF70BFEFFF76E
:1096C800F5FEA06801230038A3714FF0000318BF0E
:1096D80001206371F8BD29462046FFF7B1FE013528
:1096E800E8E70220F6E737B50023ADF8043001AA11
:1096F800022312210546FFF7C3FFBDF804400223E9
:1097080064BA01AAA4B219462846FFF781FFE20706
:1097180002D5284609F0B4F9A30702D5284609F06E
:10972800B5F9600702D5284609F0DAF9210702D50C
:10973800284609F0DBF9E20602D5284609F0DCF9EB
:10974800A30602D5284609F0C5F9600602D52846C1
:1097580009F0A2F9210606D514F4807118BF012179
:10976800284609F09FF9A20502D5284609F0AAF96A
:10977800630402D5284609F0C5F903B030BDF8B531
:109788001E468379012B154604460F46DAB227D1C7
:109798004379012B24D04271FFF7AAFE0E212046FF
:1097A800FFF7A2FDFFF718FE39462046FFF714FE23
:1097B8002E44B5420ED12046FFF78CFDFFF776FE0A
:1097C800A06801230038A3714FF0000318BF0120DF
:1097D8006371F8BD15F8011B2046FFF7FDFDE8E7AA
:1097E8000220F6E7F8B51E468379012B1546044694
:1097F8000F46DAB22BD14379012B28D04271FFF7FB
:1098080077FE1E212046FFF76FFDFFF7E5FD39467D
:109818002046FFF7E1FD00212046FFF7DDFD2E443D
:10982800B5420ED12046FFF755FDFFF73FFEA06871
:1098380001230038A3714FF0000318BF01206371A2
:10984800F8BD29462046FFF7FBFD0135E8E7022071
:10985800F6E7026852E8003F23F0C00342E800310F
:1098680002680029F5D102F1080353E8003F23F408
:10987800000302F1080C4CE800310029F3D1202341
:10988800C0F888307047000010B5026852E8003F01
:1098980023F4907342E8003102680029F5D10F4C97
:1098A80002F1080353E8003F234002F1080C4CE89A
:1098B80000310029F4D1C36E012B07D152E8003FD3
:1098C80023F0100342E800310029F7D12023C0F823
:1098D8008C300023C366436710BD00BFFEFFFFEF57
:1098E80038B50546C8B12423C0F8883003681A681B
:1098F800002422F001021A601C605C609C60F9F789
:109908008BFAC5F8904085F88440C5F88840204611
:10991800C5F88C40EC662C6738BD0120FCE70000D8
:10992800F8B504461346D4F88850202D32D1F1B149
:10993800EAB1E06FA4F85620A4F8542000262122AA
:10994800C4F890602165C4F88820226888B1124F55
:10995800C762124F0763124F2832C0E90D76FDF730
:109968008FFE30B11023C4F89030C4F8885001201D
:10997800F8BD236840221A62226802F1080353E8FE
:10998800003F43F0800302F1080141E8003000285D
:10999800F3D1EDE70220EBE7AD990008F59900084F
:1099A800019A000808B50346806A1B681B6813F013
:1099B800200317D1A0F85630026802F1080353E8D3
:1099C800003F23F08003083242E800310268002992
:1099D800F2D152E8003F43F0400342E80031002949
:1099E800F7D108BDF9F792FAFBE7704708B5806A26
:1099F800FFF7FBFF08BD7047806A38B50468D0F8E8
:109A08008830D0F88C50A268120606D5212B04D1D4
:109A18000023A0F85630FFF71CFFA3685B0606D5A5
:109A2800222D04D10023A0F85E30FFF72DFFD0F8D7
:109A3800903043F01003C0F89030FFF7DCFF38BDDA
:109A480070470000D0F88C20B0F86010222A08B5C2
:109A5800036855D15B6A826D0B401370836D0133C7
:109A68008365B0F85E30013B9BB2A0F85E30B0F879
:109A78005E309BB2002B42D1026852E8003F23F4CB
:109A8800907342E8003103680029F5D103F1080218
:109A980052E8002F22F0010203F1080C4CE80021E3
:109AA8000029F3D12022C0F88C20184A416793423C
:109AB800016705D1C26E012A0ED0F9F735FA1EE00A
:109AC8005A681102F6D553E8002F22F0806243E865
:109AD80000210029F7D1EDE70022C26653E8002FE4
:109AE80022F0100243E800210029F7D1DA69B0F822
:109AF8005C10D20644BF10221A62FFF7A1FF08BD0E
:109B08009A6942F008029A61F9E700BF00800040B4
:109B1800D0F88C20B0F86010222A08B5036852D11A
:109B28005A6A1140826D22F8021B8265B0F85E20E5
:109B3800013A92B2A0F85E20B0F85E2092B2002AF4
:109B480040D153E8002F22F4907243E80021002905
:109B5800F7D103F1080252E8002F22F0010203F1C5
:109B6800080C4CE800210029F3D12022C0F88C20F1
:109B7800174A41679342016705D1C26E012A0ED088
:109B8800F9F7D2F91EE05A681102F6D553E8002F0A
:109B980022F0806243E800210029F7D1EDE7002296
:109BA800C26653E8002F22F0100243E80021002982
:109BB800F7D1DA69B0F85C10D20644BF10221A62F5
:109BC800FFF73EFF08BD9A6942F008029A61F9E77B
:109BD800008000402DE9F84F0368B0F86060D3F8C2
:109BE8001CB01F689D68D0F88C20222A044640F0DB
:109BF800B980B0F8683043B1DFF87491DFF874A128
:109C08004FF000081BF0200F20D1B4F85E309BB253
:109C1800D3B1B4F868209A4216D9226802F1080331
:109C280053E8003F23F08053083242E800312268AD
:109C38000029F2D1504B636752E8003F43F02003FC
:109C480042E800310029F7D1BDE8F88F2368A26DFA
:109C58005B6A33401370A36D0133A365B4F85E30BB
:109C6800013B9BB2A4F85E302368D3F81CB01BF00C
:109C7800070F2ED01BF0010F09D0F90507D50122D7
:109C88001A62D4F8902042F00102C4F890201BF028
:109C9800020F09D0EA0707D502221A62D4F89020E9
:109CA80042F00402C4F890201BF0040F09D0E80722
:109CB80007D504221A62D4F8903043F00203C4F89E
:109CC8009030D4F8903023B12046FFF794FEC4F8C2
:109CD8009080B4F85E309BB2002B93D1226852E892
:109CE800003F23F4807342E8003123680029F5D14E
:109CF80003F1080252E8002F02EA090203F1080002
:109D080040E800210029F3D120225345C4F88C20D3
:109D1800616721670AD05A68110207D553E8002FF6
:109D280022F0806243E800210029F7D1E26E012A7F
:109D380014D10022E26653E8002F22F0100243E813
:109D480000210029F7D1DA69B4F85C10D20644BFC3
:109D580010221A622046FFF773FE53E72046F9F7F0
:109D6800E3F84FE79A6942F008029A616CE700BF8E
:109D7800FEFFFFEF008000404D9A00082DE9F84FE4
:109D88000368B0F86060D3F81CB01F689D68D0F80D
:109D98008C20222A044640F0B780B0F8683043B1DE
:109DA800DFF87091DFF870A14FF000081BF0200F6A
:109DB80020D1B4F85E309BB2D3B1B4F868209A428F
:109DC80016D9226802F1080353E8003F23F08053B4
:109DD800083242E8003122680029F2D14F4B63670C
:109DE80052E8003F43F0200342E800310029F7D150
:109DF800BDE8F88F2368A26D596A314022F8021B2A
:109E0800A265B4F85E20013A92B2A4F85E20D3F8B5
:109E18001CB01BF0070F2ED01BF0010F09D0F9055D
:109E280007D501221A62D4F8902042F00102C4F842
:109E380090201BF0020F09D0EA0707D502221A6208
:109E4800D4F8902042F00402C4F890201BF0040FCC
:109E580009D0E80707D504221A62D4F8903043F0F5
:109E68000203C4F89030D4F8903023B12046FFF7AD
:109E7800C2FDC4F89080B4F85E309BB2002B95D137
:109E8800226852E8003F23F4807342E800312368D7
:109E98000029F5D103F1080252E8002F02EA09026D
:109EA80003F1080040E800210029F3D1202253459E
:109EB800C4F88C20616721670AD05A68110207D557
:109EC80053E8002F22F0806243E800210029F7D1EF
:109ED800E26E012A14D10022E26653E8002F22F034
:109EE800100243E800210029F7D1DA69B4F85C10C0
:109EF800D20644BF10221A622046FFF7A1FD55E79B
:109F08002046F9F711F851E79A6942F008029A6178
:109F18006EE700BFFEFFFFEF00800040199B0008BE
:109F280038B5044603682169A2681D68C0690A43F8
:109F380061690A437749024329400A431A605A680B
:109F4800E16822F440520A435A60734AA169934275
:109F58001CBF226A11439A6822F06E4222F43062D2
:109F68000A439A60DA6A616A22F00F020A43DA62E7
:109F78006A4A934219D14FF0B043694AD3F88830FE
:109F880003F0030343F44033934200F0B480B3F189
:109F9800031F24D0013A934240F0B580B0F5004F3A
:109FA80040F08F80FEF766FA6EE05E4A93421CD15D
:109FB8004FF0B0435C49D3F8883003F00C0343F406
:109FC80040228A4200F0978006D8002B7CD0574B5D
:109FD8009A42E3D0012026E0B2F10C1FFAD1B0F585
:109FE800004F53D04FF4004075E04B4A9342F1D1F3
:109FF8004FF0B043D3F8883003F44063B3F5006FF3
:10A0080018D006D85BB1B3F5806FE3D1FEF732FA0A
:10A0180007E0B3F5406FDDD14FF400400BE0FEF7E9
:10A0280021FE40B900204FF00113A3660023C4E9C4
:10A038001D3338BD3E4865683E4B626A05EB4501F5
:10A0480033F81220B0FBF2F39942C3D8B3EB053FC3
:10A05800C0D800231946F7F757FD090241EA1061F5
:10A068006B080002C0182A464FF0000341F10001B6
:10A07800F7F74AFD304BA0F540729A42AAD82368F8
:10A08800D860CFE7FEF7EEFD0028CBD06168294BFA
:10A09800626A33F81220B0FBF2F24B0803EB42037A
:10A0A8004FF6EF72B3FBF1F3A3F11001914291D88F
:10A0B80023F00F02216892B2C3F342031343CB602B
:10A0C800B0E7FEF7D7F904E0B0F5004FDAD0FEF7B5
:10A0D800C9FD0028A6D06368616A164A32F81120C3
:10A0E800B0FBF2F000EB5300B0FBF3F04FF6EF7368
:10A0F800A0F11002C1E7B0F5004F0D48EBD1C5E75C
:10A10800FEF7C0FDC0E7B0F5004FF9D0FEF7BAFD85
:10A11800DFE700BFF369FFCF00800040003801404F
:10A12800020003000044004008000C0004000C007A
:10A138000024F400883B0108FFFC0F00836ADA075B
:10A1480010B506D50168C46A4A6822F40032224371
:10A158004A609C0706D50168046B4A6822F480327D
:10A1680022434A60590706D50168446B4A6822F4BD
:10A17800802222434A601A0706D50168846B4A6820
:10A1880022F4004222434A60DC0606D50168C46B0B
:10A198008A6822F4805222438A60990606D50168AB
:10A1A800046C8A6822F4005222438A605A060FD54A
:10A1B8000168446C4A6822F480122243B4F5801F77
:10A1C8004A6005D14A68846C22F4C00222434A607E
:10A1D8001B0606D50268C16C536823F400230B43A1
:10A1E800536010BD2DE9F843DDF8209005460F4671
:10A1F800164698462A68D36937EA03030CBF012339
:10A208000023B34201D0002029E0B9F1FF3FF2D08A
:10A21800F8F740FCA0EB080048452C6802D8B9F1D3
:10A22800000F1ED154E8003F23F4D07344E80032F5
:10A23800002AF7D104F1080353E8003F23F0010393
:10A2480004F1080141E80032002AF3D12023C5F8BF
:10A258008830C5F88C30002385F884300320BDE8A9
:10A26800F88323685A07C5D5E3691B05C2D54FF49F
:10A278000063236254E8003F23F4D07344E80032BB
:10A28800002AF7D104F1080353E8003F23F0010343
:10A2980004F1080141E80032002AF3D12023C5F86F
:10A2A8008830C5F88C30C5F89030D4E773B50446CB
:10A2B8000026C0F89060F8F7EDFB23681B681A07C2
:10A2C800054619D423681B685B070AD56FF07E43DF
:10A2D800009300222B464FF480012046FFF782FFAF
:10A2E800B0B900202023C4F8883084F88400C4F86A
:10A2F8008C30E06620670CE06FF07E4300933246B6
:10A3080003464FF400112046FFF76CFF0028D9D010
:10A31800032002B070BD10B5044650B3D0F88830A1
:10A328001BB980F88430F8F707FD22682423C4F8A5
:10A338008830136823F0010313602046FFF7F0FD0F
:10A34800012816D0A36A13B12046FFF7F7FE236849
:10A358005A6822F490425A609A6822F02A029A6057
:10A368001A6842F0010220461A60BDE81040FFF763
:10A378009DBF012010BD000030B581658168A0F83F
:10A388005C200023B1F5805FA0F85E20436735D1DB
:10A398000369002B40F2FF1318BFFF23A0F86030B9
:10A3A8000023C0F890302223C0F88C30016801F1F6
:10A3B800080353E8003F43F00103083141E8003443
:10A3C8000368002CF2D1456E84680169B5F1005F1D
:10A3D80032D1B0F8685095422ED8B4F5805F244A3F
:10A3E80003D1244C002908BF22464267B1B153E883
:10A3F800002F42F4807243E80021F7E729B9036986
:10A40800002B14BF7F23FF23C8E7B1F1805FC5D1BC
:10A418000369002B14BF3F237F23BFE703F1080222
:10A4280052E8002F42F0805203F1080040E8002172
:10A438000029F3D1002030BDB4F5805F0E4A03D166
:10A448000E4C002908BF2246426741B153E8002F4D
:10A4580042F4907243E800210029F7D1EAE753E873
:10A46800002F42F0200243E800210029F7D1E1E75C
:10A47800DD9B0008859D00084D9A0008199B00087F
:10A48800D0F88C30202B30B415D1B9B1B2B100233B
:10A498000468C3660A4B9C420AD063681B0207D54E
:10A4A80054E8003F43F0806344E80035002DF7D1BD
:10A4B80030BCFFF761BF022030BC70470120FBE7CA
:10A4C80000800040436E30B52BB90123A0F86A30F4
:10A4D800A0F8683030BD0368094D9A689968094C3E
:10A4E800490FC2F342626B5C615CDB00B3FBF1F3C2
:10A4F800A0F86A30AB5CA25CDB00B3FBF2F3E7E7E1
:10A50800A83B0108A03B01081FB504AB03E90600FE
:10A5180090F88430012B04463AD0012380F8843027
:10A528002423C0F8883003681A6822F001021A60F0
:10A538009A6822F440120A439A6071B95A68BDF8C1
:10A548000C009DF80E1022F0100202435A605A685F
:10A5580022F07F4242EA01625A601A6842F0010220
:10A568001A60F8F797FA6FF07E42034600924FF4AC
:10A57800800100222046FFF735FE38B92023C4F8B1
:10A588008830002384F8843004B010BD0320F8E735
:10A598000220F9E790F88430012B0FD0012380F8CE
:10A5A8008430016851E8002F42F0020241E800239C
:10A5B800002BF6D180F88430184670470220704787
:10A5C80010B590F88430012B044617D02423C0F826
:10A5D800883003681A68196821F00101196042F08F
:10A5E80000524FF0005141661A60FFF76BFF2023BD
:10A5F800C0F88830002084F8840010BD0220FCE7F1
:10A6080070B590F88430012B044617D005682423D0
:10A61800C0F888302E682B6823F001032B60AB68E4
:10A6280023F060431943A960FFF74CFF20232E60F5
:10A63800C0F88830002084F8840070BD0220FCE750
:10A6480038B5084D052455F8043B2BB9013C14F0E6
:10A65800FF04F8D1204638BDDB6898470028F5D0BC
:10A66800F9E700BF2C100020034BD870034B1B6880
:10A678001B6C03B1184770471410002010100020FD
:10A68800034B1874034B1B685B6C03B11847704786
:10A698001410002010100020F0B5314D314B95F901
:10A6A8000420314E91B00C46012795F905108DF81C
:10A6B800047002288DF809208DF80A1010D18DF841
:10A6C8000800D8711C7202F063FD337803B114B12D
:10A6D80001A803F0C1F9254B059A1A6011B0F0BD25
:10A6E80059714FF480711A71D9801C7233788DF8C2
:10A6F800087053BB1F2306A88DF81C208DF818304E
:10A7080002F024FF20238DF8183006A82B798DF845
:10A718001C3002F01BFF22238DF8183006A86B7935
:10A728008DF81C3002F012FF21238DF8183006A88E
:10A738006B798DF81C3002F009FF29238DF8183049
:10A7480006A80B4B079302F001FF02F021FD01233D
:10A7580006A88DF818308DF81C3002F0F7FEB4E723
:10A768001410002060080020F00E0020E40F0020E4
:10A77800000400017FB5092301A88DF8043003F017
:10A788006BF90038044B059A1A6018BF0120404243
:10A7980007B05DF804FB00BFE40F002070B5044665
:10A7A8000B46144962784A700020A2780A72087031
:10A7B8001A884A729A788A72DB780B746368CB605D
:10A7C8000D4B1B68DA6A2AB1237803F0FB030A2BC6
:10A7D80000D09047094E002556F8043B1BB15B6A30
:10A7E8000BB1204698470135EBB2052B6DB2F3D17A
:10A7F80070BD00BF30080020101000202C10002071
:10A8080070B5044611480123037063784370A37838
:10A818008372E368C360E378037623694376237918
:10A8280043720B4B1B689B6A03B19847094E00257E
:10A8380056F8043B1BB19B690BB12046984701357C
:10A84800EBB2052B6DB2F3D170BD00BF44080020F8
:10A85800101000202C100020014B1868704700BF12
:10A86800E40F002000B58BB0012368468DF8003056
:10A8780002F046FD38B99DF80400003818BF0120E1
:10A888000BB05DF804FB0020FAE7000008B501F002
:10A8980037FE40B9FFF7E6FF012806D0054B197AC5
:10A8A800D879FFF7F9FE012008BDBDE80840FFF799
:10A8B800C7BE00BF600800202DE9F04186B00546FC
:10A8C8000E46174601F01CFE002873D101F030FE39
:10A8D800044640B9FFF7C6FF01280AD03D4B197A54
:10A8E800D879FFF7D9FE6FF00204204606B0BDE81C
:10A8F800F081DFF8E48088F80860003E18BF012680
:10A908008DF80460354E687833798DF812306946D1
:10A9180002F094FC00283FD08DF804400394ADF871
:10A9280010406FF0060495E803002D4B83E8030000
:10A93800337988F80A30394601A803F091F9294B90
:10A94800059A1A6011283FD801A353F820F000BFD8
:10A95800C3A90008BDA90008D1A90008D1A9000809
:10A96800D1A90008D1A90008D1A90008EFA80008BA
:10A97800D1A90008D1A90008D1A90008B7A90008E1
:10A98800D1A90008D1A90008BDA90008BDA90008DF
:10A99800BDA90008D7A900082B788DF808306B7876
:10A9A800ADF810306B6803934FF0FF34BBE76FF0DE
:10A9B80005049AE76FF0010497E70B4B00221A7021
:10A9C800E31D18BF144690E74FF0FF348DE76FF092
:10A9D80004048AE7600800204408002014100020BE
:10A9E80054080020E40F0020E30F002037B501F0E1
:10A9F800A9FD134D052455F8043B4BB11A693AB12A
:10AA08009B682BB1984718B155F8043C1B699847C7
:10AA1800013C14F0FF04EED1FFF712FE68B9094DAE
:10AA28002B7853B1084BADF80040D97801942246F1
:10AA38006846FFF741FF00B92C7003B030BD00BF76
:10AA48002C100020E30F00201410002030B58BB02C
:10AA5800044601F055FD0546002835D1FFF702FFF1
:10AA6800012834D168468DF8005002F049FC40BBFB
:10AA78009DF80430A34204D0012C22D0022C12D01D
:10AA880014B100200BB030BD002BFAD068468DF809
:10AA9800044002F05BFDA0B90E4B1B681B6B002B3A
:10AAA800EFD09847EDE763B968468DF8044002F0A7
:10AAB8004DFD30B9074B1B681B6B002BE1D02046BE
:10AAC800EFE74FF0FF30DDE76FF00100DAE76FF0F6
:10AAD8000200D7E71010002010B504468AB018B954
:10AAE8004FF0FF300AB010BD002368468DF80030E3
:10AAF80002F006FC0028F3D19DF804302370F1E73A
:10AB08007FB500220B4620498DF8072001220A70E4
:10AB180042784A700446002A33D102790A721A88A8
:10AB28004A729A788A72DB780B740369CB60C378AF
:10AB3800164D8DF80830037B8DF809308368039330
:10AB48002B68DB6A0BB102A898472B689B6B13B183
:10AB5800227E02B198470E4E052556F8043B1BB1DC
:10AB6800DB690BB120469847013D15F0FF05F4D18C
:10AB78000DF10700FFF7B0FF637913B1054B012210
:10AB88001A7004B070BD00BF3008002010100020FB
:10AB98002C100020E30F002010B504468AB018B925
:10ABA8004FF0FF300AB010BD202368468DF8003002
:10ABB80002F0A6FB0028F3D1024A9DF90430237065
:10ABC8001371EFE71410002000B58BB02323019018
:10ABD80068468DF8003002F0B9FC003818BF012033
:10ABE80040420BB05DF804FB70B5654C01468EB071
:10ABF8001822204606F0C0F8624B00221A70F9F7B6
:10AC080083F923784068012202FA03F1014004D154
:10AC18005D4B084608F09CF8FEE75C495C481A461C
:10AC280002F0F8F818B14FF0FF300EB070BD2723CE
:10AC380004A88DF8103002F089FC564E564D0028B5
:10AC480070D1012333702B68DB690BB10020984762
:10AC5800272304A88DF8103002F052FB059B93F8C7
:10AC68004820227093F8182193F81A316270A37063
:10AC7800464BD3E9020105F06FFF05460028D2D103
:10AC8800464E062304A88DF8103002F039FB059BC8
:10AC9800736104A802F05AFC022304A88DF810304E
:10ACA800059602F02DFB0836032304A88DF8103012
:10ACB800059602F025FB0F2606F014F8012304A8D8
:10ACC8008DF814308DF8106002F040FC10230DEB65
:10ACD80003008DF810308DF8145002F037FC04236F
:10ACE8008DF8103004A8A3788DF8143002F02EFCEB
:10ACF8003A238DF8103004A86369059302F026FC06
:10AD080002A920788DF8086004F09CF8003818BF74
:10AD18000120E0711420FFF757FFE07903F062F992
:10AD2800284682E728238DF810302B681B6943B129
:10AD380004A802F0E5FA2B6805981B6940F2C45193
:10AD48009847272304A88DF8103002F0FFFB50B96C
:10AD5800012304A88DF8103002F0D2FA9DF81430BF
:10AD6800002B7FF46EAF3378002B7FF46CAF052295
:10AD780004A88DF81020059302F0E8FB78E700BFDF
:10AD880014100020E30F0020B03B0108E80F00205A
:10AD980000100020F00E002010100020501000209D
:10ADA80037B500230D4601930446D0B900F0A8FB3F
:10ADB8000190019BD3B10F4A42F824300E4A9A629F
:10ADC8000E4A1268916B1963916C596392690C4928
:10ADD800D9625A6128465B680A49F22298470020DE
:10ADE80006E001A900F092FB0028E2D04FF0FF3006
:10ADF80003B030BD2C100020A1A6000810100020C0
:10AE08007DA70008F10E0020194B07B51860194BF3
:10AE1800194A1A60194A5A60194A9A60194ADA6036
:10AE2800194B02681A6042685A6082689A60C26860
:10AE3800DA60164A1A6182695A61154BC26B5A6008
:10AE4800144A019119609A601946134ADA60002081
:10AE5800FFF7A6FF48B901A800F056FB003818BF55
:10AE68000120404203B05DF804FB4FF0FF30F9E7E2
:10AE7800101000200010002009A8000809AB0008E5
:10AE88001DAF0008A5A70008E80F0020FDED000889
:10AE98004010002071A6000889A6000849B118B121
:10AEA800012804D000207047034B0B60FAE7034BDE
:10AEB800FBE74FF0FF30704700040001010001027A
:10AEC80008B503F0ABF8002814BF6FF001000020AC
:10AED80008BD08B502F084F9002814BF6FF001001E
:10AEE800002008BD10B504468AB018B94FF0FF30ED
:10AEF8000AB010BD212368468DF8003002F000FA30
:10AF08000028F3D1024A9DF9043023705371EFE70A
:10AF1800141000202DE9F0412F4D304F00232B70E5
:10AF280043786B703B689B6A8AB004460BB128462D
:10AF38009847DFF8AC80002658F8043B1BB11B6A21
:10AF48000BB1204698470136F3B2052B76B2F3D100
:10AF58002378052B2FD00B2B35D0012B25D1214C55
:10AF6800062368468DF8003002F0CAF90199E079A5
:10AF780005F038FE10B91C4B019A5A611B48FFF7BF
:10AF88000BFE1B48FFF7AEFF6B788BB9A371194B0B
:10AF98005878FFF75BFD3B685B6A0BB1114898472F
:10AFA8006B7813B9E07905F0AFFE0AB0BDE8F0811F
:10AFB800FF23A371EFE7104B01225A74227A9A7487
:10AFC800627ADA74F1E76378002BEED00AB0BDE854
:10AFD800F041FFF7CFBB00BF44080020101000204D
:10AFE8002C10002060080020501000206408002069
:10AFF80065080020141000203008002030B58BB000
:10B00800FFF767FF0446F0B903F0FCFE831C1DD070
:10B01800F8B9134D2B685B69DBB1272368468DF8B7
:10B02800003002F06DF92B6801985B694FF4B96143
:10B03800984703F0F9FE78B92CB9094B1B68DB690E
:10B048000BB10120984720460BB030BD6FF00704C4
:10B05800EFE74FF0FF34ECE74FF0FF34F3E700BFC2
:10B0680010100020014B1878704700BF8410002092
:10B07800014B5878704700BF8410002070470000CB
:10B08800044B9A7A0AB101225A70034B5B6903B1E7
:10B0980018477047841000206C08002073B5224CB4
:10B0A8006378002B33D008F03BF966680546FFF754
:10B0B800D3FB0644AE4214D2A37A93B1E0228DF8B2
:10B0C80000208DF80130217AE36801930122684657
:10B0D800FFF7F2FB08B1073010D100236370A372A9
:10B0E800656094F83430EBB1002384F834300F4BAA
:10B0F8005B6BBBB102B0BDE87040184740F2DC5151
:10B108000B4808F0D9F90A4808F09CF9E8E794F8E0
:10B118003520002AE5D094F8360084F83530FFF75A
:10B1280095FCDEE702B070BD841000206C0800209A
:10B138006810002037B5104D104CC8B1C1B162720B
:10B14800012300222860E16023700D480D4B009216
:10B158004FF0FF3108F0CAF800250B48258220225D
:10B16800294605F01DFE6570A574A58603B030BD9F
:10B1780000232B602370EFE780100020841000204C
:10B188006810002089B00008981000202DE9F047C9
:10B198008E4C23788CB0002B56D0C2780AB9837BAA
:10B1A80013B1238A01332382437B002B4CD0E02A3E
:10B1B8004AD10023A372876897F80080B8F1220F5C
:10B1C80027D8B8F1220F30D8DFE818F04100FB008B
:10B1D80052005A0061006E0075008E009D00B40098
:10B1E800C7002F002F002F002F002F002F002F0047
:10B1F8002F002F002F002F002F002F002F002F00CF
:10B208002F002F002F002F002F002F00C900D00083
:10B21800D400B8F17E0F00F0CC80B8F17F0F00F0B9
:10B22800DF80B8F17D0F00F0AB80A57A002D00F02B
:10B238005B81674C637A3BB94FF47A71204608F01A
:10B248003BF9204608F0FEF80CB0BDE8F087E3684B
:10B2580001220021A2721970A37AE1689818A072DD
:10B268000620C854A37AE1689818A072CA54DCE78B
:10B27800584B9B6A002BD8D0012102209847D4E76D
:10B288007B7884F83630012384F83530CDE7042301
:10B298008DF804307B78003B18BF012301A88DF896
:10B2A800083002F053F9C0E77878003818BF012059
:10B2B80002F098FEB9E7484E0FCE01AD0FC50FCE8C
:10B2C8000FC596E8070085E807007B780A2BACD8FD
:10B2D800424A12685268002AA7D00CA901EB8303DE
:10B2E80053F82C0C9047A0E77878431E012B9CD884
:10B2F8003A4B01381B6818BF012020729B68002B4D
:10B3080093D0984791E7E26801230821A37211704E
:10B31800627A057BA17AAA4228BF2A46934284D240
:10B3280085685A1CEB5CE56801334E1CA6726B54A9
:10B33800D3B2EDE7E3680122A27209221A70A37A58
:10B34800E268218A581CA072D154A27A238AE16843
:10B358001B0A501CA0728B5467E7238265E70523FC
:10B368008DF8043001A802F077FB5EE7194BDB6A21
:10B3780098475AE7194B78781B686075DB68BEE711
:10B38800037B072B7FF451AF06238DF80430B7F801
:10B398000130ADF808307B793A791B0443EA02237F
:10B3A800FA781343642253430393BB798DF8103022
:10B3B800D8E73B2201A88DF804208DF8083002F068
:10B3C800C5F8012384F834302FE700BF841000202B
:10B3D800681000206C0800209C39010880100020AB
:10B3E8002A2301A88DF8043001F08AFF94F80A9006
:10B3F800E6689DF808009DF809509DF80A709DF8C8
:10B408000BC09DF80D309DF80E209DF80F109DF88B
:10B418000CE009F1010A84F80AA006F80980354E03
:10B4280094F80A903668D4F80C8009F1010A84F877
:10B438000AA096F803A008F809A094F80A90D4F88E
:10B448000C8009F1010A84F80AA096F802A008F80D
:10B4580009A094F80A90D4F80C8009F1010A84F83C
:10B468000AA096F801A008F809A094F80A9009F132
:10B47800010A84F80AA096F80080E66806F80980B0
:10B4880094F80A80E66808F1010984F80A9006F839
:10B4980008C094F80AC0E6680CF1010884F80A802C
:10B4A80006F80C70A77AE66807F1010C84F80AC060
:10B4B800F555A57AE6686F1CA7727055A07AE568FD
:10B4C800461CA6722954A17AE0684D1CA572425404
:10B4D800A27AE168501CA0728B54A37AE268591CC6
:10B4E800A17202F803E0A0E6034807F05DFF65706B
:10B4F800AAE600BF801000206810002070470000F6
:10B50800004870476C080020002070474FF0FF305B
:10B5180070470000044B054A93F81831022B18BFF6
:10B52800062382F89034704728170020EC1C00206E
:10B53800034BD3F8483313B15B6903B1184770471D
:10B54800EC1C0020034A137843F004031370FFF740
:10B55800EFBF00BFD01000201FB50A4B8DF80900BF
:10B5680093F87C208DF80A2093F88C2093F84800F3
:10B578000D3202A98DF8082003F064FCC0B205B0B2
:10B588005DF804FB2817002008B5074807F00CFFF2
:10B59800064B93F81A2412B1012283F81924BDE846
:10B5A8000840FFF7C5BF00BFEC200020EC1C0020BE
:10B5B80010B50C4CD4F8403343F08003C4F8403342
:10B5C80094F81A3413B10020FFF7DEFF94F8913491
:10B5D80023F0120343F0120384F89134BDE81040BD
:10B5E800FFF798BFEC1C00202DE9F041DFF8AC8094
:10B5F80098F81831022B06460D4602D0284BDB6A14
:10B60800984702F0A6FD044628B1022002F097FDF3
:10B61800002002F099FD98F81831012B17D102F09B
:10B628009AFD074630B1002002F08AFD002002F0A2
:10B638008CFD3C4602F091FD48B1002002F081FDEE
:10B64800002002F083FDBDE8F041FFF763BF002C46
:10B65800F9D1144C94F8902494F81A34BAB90BB16F
:10B6680084F84164304602F017FFD8F82C0007F040
:10B6780061FED4F8B4339842E5D30B4807F094FE42
:10B6880094F8913443F0100384F89134DBE70BB15C
:10B6980084F84154284602F0FFFEF1E728170020FD
:10B6A8002C430108EC1C002084200020074A10B518
:10B6B800137843F002031370FFF73AFFBDE8104018
:10B6C800034B01220021022007F042BBD0100020CA
:10B6D800F93B0108074A10B5137843F008031370C3
:10B6E800FFF726FFBDE81040034B0122002102208E
:10B6F80007F02EBBD0100020093C01082DE9F041CD
:10B708000F4616461D46804607F00AFE0B4A0C4CAB
:10B718001378278123F0110343F01103C4E90008CB
:10B72800137066812573FFF703FFBDE8F041054BF1
:10B7380001220021022007F00BBB00BFD01000201F
:10B74800BC100020193C010813B507F0E9FD0D4BAA
:10B758006C461860204607F037FD94E803000A4A53
:10B768000A4B83E80300137843F020031370FFF7B4
:10B77800DFFE074B01220021022002B0BDE8104085
:10B7880007F0E6BACC100020D010002024200020BA
:10B79800263C01082DE9F04192B0064602F0D9FC9A
:10B7A800002840F05881AD4D95F81831012B09D08B
:10B7B8002B6BAB4C93B194F80431BBB1042B6FD015
:10B7C800032003E002F0C7FC18B10F2012B0BDE857
:10B7D800F08102F0C2FC0028EAD0F6E7B5F8203183
:10B7E800D4F81C24013B53432B63E4E79D4803F042
:10B7F80060FA002840F0128194F80C3123802B6BFA
:10B808000C930DF1180895F839308DF8383040460A
:10B8180095F81C318DF83A3007F0FCFCD5F8283142
:10B82800009302AF98E80600D5F82431384607F0AF
:10B8380088FC97E803000FAB83E80300EB6A0D93DD
:10B8480000238DF844302388ADF8463095F8303120
:10B8580001228DF839201BB98DF844208DF8393034
:10B86800814B0093814B95F84800A3F179020CA90C
:10B8780003F05DFBC0B10B28A8D1D4F8941499B19A
:10B88800002EA3D0D4F84033794843F02003C4F8FD
:10B89800403307F011FE764807F0D4FD002095E705
:10B8A800704803F03AFAA4E795F8487095F96930BA
:10B8B80095F9392095F87D106E4E384603F044FB13
:10B8C800009641B2EB6C95F850203846183603F0D4
:10B8D800DFFA0096EB6C95F8502095F9701095F802
:10B8E800480003F0D5FAD4F8C413AB6DD4F8DC23C0
:10B8F8000B44C4F8B033EB6D1344C4F8B43394F874
:10B908000431042B07D02B6E0B44C4F8B0336B6E94
:10B918001344C4F8B4330023089395F83031002B4E
:10B9280040D100238DF8133095F839308DF8213047
:10B9380095F838308DF82230D5F880300993D5F84D
:10B9480084300A932388ADF82C3095F8303194F878
:10B958001B648DF82E3095F84800474B8DF8206011
:10B968000DF1130208A903F0A7FA012384F8413462
:10B9780095F8393084F842349DF8133084F843340C
:10B98800D4F81C34C4F85064C4F84834C4F85834A3
:10B9980002F0E5FBC8B1D4F81C0402F0F2FBA0B138
:10B9A800102013E708A802F0A7FC60B995F9390040
:10B9B80094F837629DF82070FFF7CEFD3E44B04200
:10B9C800AFD2082002E7132000E795F81831012BC1
:10B9D80001D102F0D8FB02F0C5FB0023059394F8CF
:10B9E800043195F9395094F81B649BB1042B7FF40A
:10B9F800E7AE05A802F0B4FE58BB94F8183413B1AA
:10BA0800059B013B0593174B05983246E9B202F0B6
:10BA18000DFF02E0134802F0DDFE08B11120D5E663
:10BA2800D4F8403394F80C11218043F00203C4F891
:10BA3800403394F8183411480133DBB284F81834D1
:10BA480084F845340E4B00259B6AC4F898549847EF
:10BA580024E71220BAE60E20B8E600BF2817002017
:10BA6800EC1C0020F41D0020581700208021002025
:10BA780054200020A420002008210020EE1C0020D3
:10BA88002C43010873B5134D134E0096EB6C95F8D3
:10BA9800502095F9781095F8480003F0F9F995F8D1
:10BAA8003031337595F8480040F2012306F13C0225
:10BAB8003146738203F0F8F950B196F83C3086F8B5
:10BAC8008230064B00205B6B9847F37C86F8A830E1
:10BAD80002B070BD28170020D42000202C43010894
:10BAE800F8B5324C94F81831012B05460ED0022BCC
:10BAF8004ED0002B57D138B9D4E91B0104F1740397
:10BB080083E803000020F8BD012806D102F02CFBD1
:10BB18000028F8D184F81851F5E7022843D1244EBB
:10BB280084F8180106F5747CBCE80F0006F57A77EE
:10BB38000FC79CE8030094F8E92094F8003187E8DF
:10BB4800030086F8FB53D2B1022B18D1D4F8043184
:10BB58006367C6F8EC3394F87D3094F8082186F8CA
:10BB6800F83394F88C3084F8782086F8F93396F80E
:10BB78001B2486F8E82340F20133A6F8FA330023A1
:10BB880086F81A340B4BDB6A9847FFF77BFFB9E757
:10BB980048B9074B84F81801062283F89024054B0E
:10BBA800DB6A9847AEE70320ADE700BF28170020FF
:10BBB800EC1C00202C430108F0B5504C504EB4F852
:10BBC800DC202287D4E92D0194F8B12084F869207B
:10BBD80004F16C0282E80300D4E92F0104F1740235
:10BBE80082E80300B4F8C420A4F87C2091B0D4F80B
:10BBF800CC20D4F8C810C4F884200025D4F8D0206C
:10BC0800C4F888200123A4F82031C4F8801084F8EF
:10BC18003051A56284F81B5184F83A5084F81D51BC
:10BC280084F81E51C4F83451C6F89854A6F818542C
:10BC380086F81A54A4F838518DF8183004F50973A9
:10BC4800039304F50A7394F84800049303A92D4B51
:10BC580084F84551C4E94F55A4F84651059303F0BB
:10BC6800FFF8E36EC6F8D43394F87D3086F8E033F5
:10BC780094F88C3086F8E1334FF48073A6F8E233F9
:10BC880086F8D05394F8303186F8E43306F57477A3
:10BC98000FCF06F57A740FC497E8030040F201232A
:10BCA80084E80300A6F8FA33D6F8483386F81B541C
:10BCB800CDE901551BB15A685B6901920293124B99
:10BCC8000793A3F148020892A3F1140209920F4ABC
:10BCD8000B9229330A93A2F19C030C93A2F19803C7
:10BCE8000D93131D0E9301A902F14C0307A802F549
:10BCF80099620F9302F022FA11B0F0BD28170020C4
:10BD0800EC1C0020D4100020542100200C18002026
:10BD1800F8B50D4F0D4E0C4607F046FB3B6B9847A8
:10BD28000B4A96F84800214603F0BEF850B1094D79
:10BD3800706D95F8243485F86A347B6B9847E37CFA
:10BD480085F89034F8BD00BF2C430108281700205F
:10BD580010210020EC1C00200F4890F81B3480F8BC
:10BD6800B8330E4B93F8692080F8BB2393F87D20F5
:10BD780080F8C82393F88C2080F8C92393F83031D1
:10BD880080F8CC330022A0F8CA2300F56E7100F5C4
:10BD98006070FFF7BDBF00BFEC1C00202817002013
:10BDA800114890F89034EBB190F81B3480F8D033F8
:10BDB8000E4BDA6EC0F8D42393F87D2080F8E02388
:10BDC80093F88C2080F8E12393F8303180F8E4333D
:10BDD8004FF48072A0F8E22300F5747100F56670E4
:10BDE800FFF796BF704700BFEC1C00202817002003
:10BDF80070B5344C2421204604F0D4FF636A98427D
:10BE080018BF60624FF01C012F4814BF01250025A0
:10BE180004F0C8FF636C984218BF60644FF48071E7
:10BE28002A4818BF45F0020504F0BCFFD4F8483191
:10BE3800984218BFC4F848014FF0D401244818BFED
:10BE480045F0040504F0AEFFD4F82032984218BF3C
:10BE5800C4F820024FF000011E4818BF45F008053D
:10BE680004F0A0FFD4F82432984218BFC4F8240282
:10BE78004FF46071184818BF45F0100504F092FFA0
:10BE8800D4F8A835984218BFC4F8A8054FF0140193
:10BE9800124818BF45F0200504F084FFD4F8C035D7
:10BEA80098420F4B18BFC4F8C005D3F8483318BFE1
:10BEB80045F040052BB11B691BB12846BDE8704011
:10BEC800184770BD28170020501700207017002051
:10BED800741800204C19002050190020D41C002090
:10BEE800EC1C00202DE9F04F8FB04FF00009012B1A
:10BEF80006460F4690468DF80D90ADF8109002D882
:10BF08004C46BC4202D30FB0BDE8F08F305D02F062
:10BF180033FA2044B842F6DC335D651C023BEDB2CF
:10BF2800112BF0D801A252F823F000BF7DBF000802
:10BF3800A7BF0008A5C00008CDC000084BC1000875
:10BF480071C10008D7C10008FFC1000885C20008F8
:10BF58000FBF00080FBF0008D9C200080FBF0008B4
:10BF68000FBF000881C30008A9C30008E1C3000887
:10BF780015C40008052002F0A7FA70B105210020B9
:10BF880002F068FA725DBA4BE51C0234E4B283F839
:10BF98005C24325D83F85D24EDB22C46B1E70023C2
:10BFA8008DF80E308DF80F308DF814308DF818306C
:10BFB800B9F1000F6DD1AF4C4FF0050994F87C2012
:10BFC8008DF831206B1E94F839208DF833203344D6
:10BFD80094F838200B938DF8342094F81A3194F89B
:10BFE80068208DF83520D4F82C218DF832300A924B
:10BFF80073B37B1C5B1BDBB28DF8303006AB01934F
:10C0080005AB009394F848000DF10F030DF10E02F3
:10C018000AA902F05DFF8DF80D0000F0070007285F
:10C0280013D194F939209DF90E3084F839309A42A9
:10C038009DF80F3084F83830B8BF01229DF81430CD
:10C04800B8BF84F81D2184F868304FF0000A09E071
:10C058000523D1E701220DF10D01032002F0A4F818
:10C068000AF1010A5FFA8AF29DF81830B3FBF9F178
:10C078009142EFD82B44DDB26B1EDBB29F420BD945
:10C08800F25C032A9AD0AF4288BF1D464FF00109DF
:10C0980083E70534E5B2F9E71D46F7E7735D7549AF
:10C0A80003F00F03012281F81B31023402FA03F373
:10C0B800A1F82031E4B2002204A9042002F074F8A7
:10C0C80025466AE707238DF80D30735DC3F3021226
:10C0D80003F00F038DF82830E31CDBB28DF829201C
:10C0E800F25C231DDBB2651DF35C0234E4B21B0471
:10C0F80043EA0223325D5F4C13436422534394F8AE
:10C1080048000B930AA902F0F2FE00F00703072B80
:10C11800EDB28DF80D000CD19DF8283084F8703000
:10C1280084F878300B9BE36663679DF8293084F8C0
:10C1380069308DF81000012204A9052002F034F8B6
:10C148002BE74B4BD3F8483363B11B6853B198477F
:10C1580008F03F038DF810008DF81130022204A971
:10C168000620EBE7FF20F3E703238DF80D30735D1E
:10C178008DF81C300AAB0693E31CDBB2A51DF25CFC
:10C18800231DDBB206A9F35C1B0443EA0223A21CAD
:10C19800D2B20534B25C134364225343E4B20A9327
:10C1A80000230B93335D8DF83030324B93F8480001
:10C1B80002F0A3FEC3B20028EDB28DF80D30FFF6F1
:10C1C800ECAE8DF81030012204A90720B6E7735DA4
:10C1D80003F00F03012B4FF47A7238BF0123534346
:10C1E800244A0234936503F57A73D365E4B20022D6
:10C1F80004A9082062E7735D1E4DC3F340128DF851
:10C20800152095F84800C3F3001205A903F00F03A1
:10C218008DF814208DF8163002F075FE02340130C6
:10C22800E4B23FF44DAFBDF81430134AA5F87C30A2
:10C238009DF816309DF814A0D05CF5F7E7FB0223B3
:10C24800C5F880000AA995F848008DF828308DF8BF
:10C258002AA002F0F7FD95F93930069040B29842CD
:10C26800B8BF184685F83900002204A9092025E737
:10C27800EC1C002028170020333C010803238DF80C
:10C288000D30735D8DF82830E31CDBB2651DF25C60
:10C29800231DDBB20234F35CE4B21B0443EA02233D
:10C2A800325D1343642253430B93644B0AA993F8FA
:10C2B800480002F02EFEC3B20028EDB28DF80D3012
:10C2C800FFF66BAE8DF81030012204A90A2035E77D
:10C2D800092002F0F9F8DFF868B1002849D00921EF
:10C2E800002002F0B7F80023ADF81E30A31CDBB223
:10C2F800F25CE31CDBB216F803A0735D4FEA0A4A4E
:10C308004AEA022A4AEA030A231DDBB2A51D0534BC
:10C31800F35CE4B24AEA036A335D4FF47A7253433A
:10C328000AAC1B122046ADF81C3006F04DFF454BF9
:10C3380053440693DBF83C3300930DF1180A9AE84E
:10C348000600DBF8383308A806F0FBFE099B0093CB
:10C3580094E80600089B504606F0D8FE9AE80300C9
:10C3680006F00AFF01F00AFF0123EDB28BF838341A
:10C3780013E68BF8380410E60C2002F0A5F8002824
:10C388003FF40BAE0C21002002F064F82C4B93F81C
:10C398009034043B012B7FF600AE01F0EBFEFCE588
:10C3A800A31CDBB2725DF15CE31CDBB2651DF35CC0
:10C3B8000434E4B21B04305D43EA012313436421CF
:10C3C800594300F00F0001F0D6FEEDB28DF81000D1
:10C3D800012204A91120B1E60D2002F075F8002809
:10C3E8003FF4DBAD0D21002002F034F8A31CDBB2D2
:10C3F800154AF05C735D1268251D0334E4B243EA04
:10C408000020315DEDB201F0B8FEC6E5725DA31CF7
:10C41800251D0334DBB2E4B2F15C335D1B0443EA4F
:10C42800012313436420584301F0A9FEEDB28DF8AF
:10C438001000012204A9132080E600BF281700205D
:10C44800EC1C0020803DD512BC1000200E4B93F848
:10C458009124920703D593F88F24012A08D90B4910
:10C4680091F81A2122B18A6A501C18BF01328A62D7
:10C478000022A3F8182483F81A24D3F8402322F0C2
:10C488000202C3F840237047EC1C00202817002044
:10C4980070B5184C1848194D06F086FFD4F840338B
:10C4A800D4F89804D5F8906023F02003C4F84033FA
:10C4B80038B106F03FFF864203D2002385F83A30B0
:10C4C80070BD0120FFF766F90028F9D00B28F7D0D6
:10C4D80095F8393084F84234092094F8183484F8EF
:10C4E800453484F8410401F0D7FFBDE87040FFF7F8
:10C4F800ADBF00BFEC1C00205420002028170020EE
:10C50800094BD3F84023012A0AD008490978C907FA
:10C5180008D43AB993F89204013818BF012070473B
:10C528000020704701207047EC1C0020D01000202C
:10C53800034BD3F84003431E58425841704700BF8D
:10C54800EC1C00202DE9F04FA9B0EFF3108272B671
:10C55800DFF8F0B20021DBF80030CBF8001082F3EE
:10C568001088B94C002B00F0E180DAB29B060392E8
:10C5780064D5B64D95F81831022B02D0B44BDB6A5E
:10C588009847EFF3108872B6B24F06F0C9FE3E68BE
:10C59800D4F8B013361A3144AF4806F08DFFAE48D0
:10C5A80006F050FFD4F8B413AC48314406F084FFC9
:10C5B800AA4806F047FF88F3108894F81A34002B2D
:10C5C80000F06B81152312A995F848008DF84830C2
:10C5D80002F038FCD4F8B4130F900144A04806F0D8
:10C5E8006BFF9F4806F02EFF3B6894F81B24EB6214
:10C5F8000DAF38468DF870201D9306F00BFED5F868
:10C608002831009306AE97E80600D5F82431304665
:10C6180006F097FD96E803001FAB83E80300D4F803
:10C628001C341E9395F8303195F84800003B18BF2C
:10C6380001231CA98DF8713002F00DFC039BDF0665
:10C6480048D5824DDFF81CA2D5F8E42004929BF867
:10C658000020BAF90A809AF90C90A4F88C84002377
:10C6680063F300020A9384F84434A4F8223484F86B
:10C678002534C4F82834A4F82C3484F82E34C4F8AB
:10C68800303484F82034C4F8343484F83834C4F8A6
:10C698003C346F4B8BF8002094F89024DB6A84F8C4
:10C6A8008E9484F88F24DAF80470BAF808609847F2
:10C6B80094F88F3413B9694806F076FE3146384647
:10C6C80001F045FD8346002800F0EA80A4F87E8446
:10C6D80084F88094039B19071AD55C4B93F818319A
:10C6E800022B02D05A4BDB6A98470220FEF712FF52
:10C6F80084F8410401F0D0FE94F81A3413B10123F0
:10C7080084F8193494F8913443F0100384F8913480
:10C71800039B5A0703D506210520FEF765FF039BF7
:10C728009B0703D504210320FEF75EFF01F02DFDD2
:10C7380094F89124D7065FD5002384F89234D4F86E
:10C7480040331E0644BF23F08203C4F8403312F07E
:10C75800050F00F0FB820B2001F0B6FE002800F068
:10C76800F58294F89134DD0700F1F082580740F122
:10C778000783D4F8403323F00203C4F84033D4F8D5
:10C78800402382BB94F8915415F001011EBF2B463B
:10C7980062F3000384F8913494F891345E0744BF3F
:10C7A8006FF3820384F89134012384F8923421B121
:10C7B800D4F844332C481B6898476D070BD52B4891
:10C7C80001F08EFE01F0BCFE28B194F8913443F0DC
:10C7D800040384F8913401F0C6FC94F891346FF3A3
:10C7E800041384F89134012384F8923494F8913432
:10C7F80043F0200384F8913494F8913418070AD54B
:10C808006FF3C3031A4984F89134D4F84433A1F17F
:10C818002400DB68984794F8913499070AD56FF398
:10C828004103134984F89134D4F84433A1F16C00DE
:10C838005B68984794F89034022B1BD1FFF722F9D4
:10C8480018E000BFD0100020EC1C002028170020A2
:10C858002C430108CC1000206C20002084200020EC
:10C86800EC200020BC1000202C21002040210020BA
:10C878007821002094F891349A0640F1C4826FF32D
:10C88800451384F89134D4F84033002B40F0BB8230
:10C8980029B0BDE8F04FFFF7ABBA84F84134A3E6FE
:10C8A80095F81831012B0CD101F055FC804668B180
:10C8B800584601F045FC584601F047FC042384F82B
:10C8C8008F347EB9012384F821344FE101F045FC0F
:10C8D8000028F6D0404601F034FC404601F036FC12
:10C8E8000523ECE73B7805935B09013B062B00F237
:10C8F8001782DFE813F00700150295001502920071
:10C9080015020602102EDDD995F830311297F6B2CD
:10C918008DF84C60002BD5D11CA804F055F912AA4B
:10C928001CA9FF2002F09EF89DF85830C3F30303BA
:10C9380007468DF82C3095F8480095F87D308DF82D
:10C948002D3007220BA902F090FA002F5DD10028A4
:10C958005BD09DF853309DF852201599C5F8E41026
:10C968001B0443EA02239DF8512002201343C5F813
:10C97800E03004F037F99DF8583095F8480085F80C
:10C988002E71C3F30212C3F3030385F8703085F8E0
:10C9980078309DF8593085F86920012B38BF01237C
:10C9A8004FF47A725343AB651344EB650DF15A03A8
:10C9B8004FF001081093113E94F81B348DF83C3069
:10C9C8000FA985F868808DF8446002F056FA0223B2
:10C9D800404685F8303101F077FD18B141463846B8
:10C9E80001F038FD94F88F34012B00F2A78194F8F8
:10C9F8001A34002B40F09A8194F8913443F01003D4
:10CA080084F89134FEF786FD64E6012001F05CFDB0
:10CA18000028E7D001210720E2E7012384F8203429
:10CA280095F87D308DF82E3094F824348DF82D301B
:10CA380095F88C3095F848000D330BA98DF82C30FB
:10CA480002F000FAA6F10D031BB2099023EAE37382
:10CA580000B283423FF736AF0B2E7FF633AFBA4BA7
:10CA680025931CA8FF231C978DF874608DF89830C7
:10CA780002F0C4F8074600287FF424AF95F818316F
:10CA8800012B13D101F067FB002872D0384601F062
:10CA980057FB384601F059FB04239DF87C101E987B
:10CAA80084F88F34C1F3001101F06EFB9DF87C30DF
:10CAB8001E99C4F8341413F00F0203D09DF89000A7
:10CAC800002862D19DF89800002861D0002A7FF4E0
:10CAD800F9AE9DF89020002A14BF4FF003084FF0DC
:10CAE800020800220A92D5F8EC2095F8E900914254
:10CAF80051D100284FD0D5F80C1195F8EAB0096843
:10CB08000A9195F81811022902D1032184F88F148B
:10CB1800B8F1030F7FF4D6AE13F0600F7FF4D2AEF6
:10CB28000492012795F82E31BBF1000F36D0BBF1E6
:10CB3800010F13D1012B33D16FF0090646FA08F61D
:10CB480006F00106C6F10206F6B2BDF87E100AAA82
:10CB5800304601F011FE38B3072823D0012384F8AA
:10CB680021340A9BC4F83034C4F86C34FEF720FD35
:10CB7800B0E501F0F2FA002898D0384601F0E1FA61
:10CB8800384601F0E3FA052387E74FF00008A8E7E5
:10CB98004FF00108A5E74FF0010BC3E70426D4E7DF
:10CBA8000326D2E70823DAE71CAB009304990A9B13
:10CBB8003246584601F0A2FE20B1022814BF0B23CA
:10CBC8000A2380E60A9BC4F83034C4F86C349DF814
:10CBD8007C3084F82104C3F3401384F82E3484F89D
:10CBE800443494F88F3484F82274012B9EBF0122B8
:10CBF800A86285F81E21012FC4F8280484F82C04A3
:10CC080084F8410438D1022284F8202495F83A2087
:10CC1800002A4AD19DF87C20D60646D4012B94F8E8
:10CC280040149DF87C2005D8012901D1900601D532
:10CC380001F04CFBB8F1020F94F88F3443D0B8F1EF
:10CC4800030F0AD09DF87C10B8F1010F4A4601F095
:10CC58000F0120A83BD0FFF745F99DF8903084F8E4
:10CC68002334259BC4F828349DF8983084F82C3454
:10CC7800012384F82D3430E0059A02F0E002A02A5E
:10CC88001BD195F82E11012285F83A2009B9279968
:10CC98006963012B84F8202407D9D5F89020C4F8BB
:10CCA8003C24DAF80020C4F8982495F81821002AC2
:10CCB800B4D1012284F82524B0E7002285F83A206F
:10CCC80084F82024A6E79DF8981025984A46FFF78F
:10CCD80009F99DF8903084F823349DF89020E02AD3
:10CCE80008D195F81F312BB984F82324C4F82834C7
:10CCF800A4F82C3494F8913443F0020384F8913466
:10CD080070E6114D013EB2B2791C284604F034F8A1
:10CD18000323A4F82034C4F8285484F82C64E9E7E1
:10CD2800012384F82134FEF743FC5BE694F844348D
:10CD3800002B3FF461AE0020FEF726FC94F88F34F8
:10CD4800022B3FF45FAE57E6241F002094F891347D
:10CD5800590715D5012001F0B7FB60B1012001F09A
:10CD68008BFB08B984F81804D4F8403323F0020385
:10CD7800C4F8403304E0062001F0A6FB0028F3D1F4
:10CD880094F89134DA077FF5FAAC94F840240AB1A4
:10CD9800032A18D11D4A94F8181492F86820914271
:10CDA80005D29B0723D594F88F34012B1FD8184838
:10CDB80006F0FAFAD4F8403323F02003C4F84033DD
:10CDC800FFF744FBDBE4012A11D194F81924002A67
:10CDD8003FF4D5AC0D4A94F8181492F868209142A3
:10CDE800E5D29F0703D594F84434002BDFD194F89B
:10CDF800913400206FF3041384F8913484F81904F3
:10CE0800FFF746FBBBE429B0BDE8F08F28170020E8
:10CE1800542000202DE9F04F89468DB090460746F2
:10CE2800002800F08F81002900F08C810368002B16
:10CE380000F088814368002B00F084818368002B10
:10CE480000F08081C368002B00F07C81104601F05F
:10CE5800F5FF002800F07881BD4CBE4D384601F042
:10CE6800AFFA40F2C4520021204603F099FF40F285
:10CE78001C520021284603F093FFB74BC4F82C310D
:10CE880004F50973089304F50A73002640460993CC
:10CE980008A9B24B84F848800A9384F8186184F88A
:10CEA8008C608DF82C6001F0DBFF0F2306A994F845
:10CEB80048008DF8183001F0C5FF801B18BF01200D
:10CEC8004FF00A0B84F81C0106A994F848008DF865
:10CED80018B001F0B7FF4FF0060A84F8DC0006A985
:10CEE80094F848008DF818A001F0ACFF102384F8DE
:10CEF800DD0006A994F848008DF8183001F0A2FF6B
:10CF08001123C4F89C0006A994F848008DF818303D
:10CF180001F098FF1223C4F8A00006A994F848006D
:10CF28008DF8183001F08EFF1323C4F8A40006A969
:10CF380094F848008DF8183001F084FF1423C4F8E1
:10CF4800A80006A994F848008DF8183001F07AFF77
:10CF58001623C4F8AC0006A994F848008DF81830D8
:10CF680001F070FF172384F8B10006A994F848006F
:10CF78008DF8183001F066FF18230DEB0301C4F893
:10CF8800B400C4F8BC0094F848008DF8183001F0DB
:10CF980059FFC0B21D2384F8B80084F8C00006A960
:10CFA80094F848008DF8183001F04CFF1E2384F8DF
:10CFB800C40006A994F848008DF8183001F042FF23
:10CFC8001F2384F8C50006A994F848008DF8183086
:10CFD80001F038FF2023C4F8C80006A994F84800D7
:10CFE8008DF8183001F02EFF0B23C4F8CC0006A9E9
:10CFF80094F848008DF8183001F024FF0C2306A996
:10D00800A4F8D00094F848008DF8183001F01AFF01
:10D01800D4F89C306365D4F8A030A365D4F8A43064
:10D02800E365D4F8A83023664FF00108D4F8AC3093
:10D038000590A4F8D200636684F8B080C4F894B070
:10D0480084F898A0C4F84CB084F850A084F868809C
:10D0580084F81F81C5F84893FEF7AEFDC5F8447300
:10D06800C4E90B663E4B84F8198185F89164C5F8CC
:10D07800408332464FF0FF31009605F55A7006F0AE
:10D0880035F9384B009632464FF0FF3105F56070A0
:10D0980006F02CF9344B009632464FF0FF3105F577
:10D0A800667006F023F902AF304B009632464FF017
:10D0B800FF3105F5806006F019F9384606F0AAF840
:10D0C80097E8030004F5927383E80300284B294F7F
:10D0D8001E60294BC5F84C33284BC5F85433284BF0
:10D0E800C5F85C33274BC5F85033274BC5F8583380
:10D0F80005F553703B68984704F5A67003F080FB6C
:10D1080020B1112630460DB0BDE8F08F204601F061
:10D1180003FB0028F5D101F039F8B8B91B4801F034
:10D128004DFB06460028ECD17B69984703F002FEC8
:10D13800BB6D94F819019847FB6A9847012385F855
:10D148009234DFE70326DDE70926DBE71326D9E774
:10D1580028170020EC1C002000040001D410002037
:10D1680099C4000861BD0008A9BD000891B5000870
:10D17800D01000202C43010851B7000805B700085B
:10D188004DB50008DDB60008B5B600081018002037
:10D1980008B5034B0020C3F84003FEF7BBF908BDF0
:10D1A800EC1C002010B5FFF7ABF90A4C60B90A4B2C
:10D1B80093F81831022B02D1084BDB6A98470123F8
:10D1C800C4F84033002010BDD4F84003013818BF1C
:10D1D8000120F8E7EC1C0020281700202C43010848
:10D1E80038B5124C204606F0DFF804F1180006F0B6
:10D1F800DBF804F1300006F0D7F804F1980006F0E7
:10D20800D3F800F0AFFF0A4B0025DB6A984744F8D3
:10D21800285CFEF7EDFD0749074840F2C45203F0C9
:10D22800ABFD012344F8283C284638BD5420002093
:10D238002C430108281700206411002070B52E4BDC
:10D248008AB0054693F8DD008DF8090093F8DC00F4
:10D258008DF80A0029489A6A90F818040392002663
:10D268008DF80B0004960C46002940D00692D3F89E
:10D27800882007921A8F93F81A118DF8151052BA50
:10D28800ADF8202093F87C2093F848308DF82430AE
:10D2980003AB8DF822008DF8232000930DF10A02CC
:10D2A8000DF10B030DF1090105A88DF8146000F0CC
:10D2B800D7FE9DF90900FEF74FF9607004A801F048
:10D2C8001BF8B0B9049A0F2A0DD863789A420AD885
:10D2D8001544AB42A3EB02012CBF002001202170B2
:10D2E800C0000AB070BD002323700820F9E70320AE
:10D2F800F7E71320F5E700BF28170020EC1C0020F3
:10D308001FB50446002800F010810378412B00F275
:10D318000781DFE813F0420049004D005100550035
:10D3280059005E000501050105010501050105011A
:10D3380005010501650069006D0078007F00820025
:10D3480085008A0088008C00900093009600990060
:10D358009C009F00AE00B200BA00B600BE00C1003B
:10D36800C500CE00CA00CC000501D20005010501A8
:10D378000501050105010501050105010501050175
:10D3880005010501050105010501DA00DE00E200DD
:10D39800E700EB00EF00F300FC00664B93F8183150
:10D3A8002371002004B010BD624B93F83031F7E7C9
:10D3B800406803F0C3FBF4E7406803F005FCF0E7BE
:10D3C8005C4B93F81A31EBE75A4BD3F8E0306360C3
:10D3D800E7E7584B011D93F8300103F00DFCE0E737
:10D3E800544B93F81931DBE7524B93F88C30D7E75D
:10D3F8001C238DF808304F4B02A993F8480001F020
:10D4080021FD6060CDE74C4B043493E8030084E8C9
:10D418000300C6E7494B0434F7E7494B0434F4E703
:10D42800484B0434F1E71A23E3E71923E1E7414BBA
:10D4380093F86830B4E73F4B5B6DC8E73D4B9B6D95
:10D44800C5E73C4BDB6DC2E73A4B1B6EBFE7394B78
:10D458005B6EBCE702238DF80830364B02A993F8BF
:10D468007C2093F848008DF80A2001F0EBFC20712D
:10D4780097E7304B93F8DD3092E72E4B93F839302D
:10D488008EE72C4B93F8DC308AE72A4B93F8383038
:10D4980086E7284BDB6C9AE7264B93F850307FE7FA
:10D4A800244BD3F8843063607BE7224B8FE7264B0D
:10D4B8008DE7204BD3F8CC30F5E71E4BD3F82C3151
:10D4C800436001F04DFDA0606BE71A4BD3F8903034
:10D4D8007DE7184B93F81F3162E7164BB3F8883095
:10D4E800A3805EE7134BB3F88A30F9E7114BB3F822
:10D4F800D030F5E70F4BB3F8D230F1E70D4B93F886
:10D5080048200AB1062A12D1B3F8A035E8E7094B3A
:10D5180093F848200AB1062A09D1D3F8A43556E76A
:10D5280004B0BDE8104000F021BE03203AE71820FF
:10D5380038E700BF2817002094170020DC170020C8
:10D548009C170020E4170020641100207FB50446D2
:10D5580010B9032004B070BDA34DD5F840339A0725
:10D5680000F16F820278412A00F26882DFE812F047
:10D578004200470055005B005F00640069007600C8
:10D58800810087008D00930099009F00A500AB00E3
:10D59800B5006602BA00DC00EF0016013801290167
:10D5A80042014B014F01530157015B0166025F01C4
:10D5B800710199018701AB01B101B801BD01C20137
:10D5C8006602280266026602660266026602660251
:10D5D8006602660266026602660266026602660203
:10D5E80066026602340239023E02430248024D02D4
:10D5F80052025C020079FEF773FA30B1AAE70379A8
:10D60800022BA6D0794A82F8303195F8913443F04C
:10D61800200385F8913400209CE7406803F080FAE5
:10D628000028F2D095E7406803F0BEFAF8E76F4BA0
:10D63800027983F81A21E8E76C4B4268C3F8E020C6
:10D64800E3E76A4E416896F8300103F0CBFA002808
:10D658007FF47FAF6368C6F8E430D6E741680029F5
:10D668003FF477AF002001F0DDF90028CDD011207C
:10D6780070E7416800293FF46CAF0120F3E7416887
:10D6880000293FF466AF0820EDE7416800293FF420
:10D6980060AF0920E7E7416800293FF45AAF0C2042
:10D6A800E1E7416800293FF454AF0D20DBE741680A
:10D6B80000293FF44EAF0E20D5E7416800293FF41A
:10D6C80048AF0F20CFE74A4C484B007983F819013F
:10D6D800A36D9847E36A984797E7444B027983F824
:10D6E8008C2092E7414E037A8DF8043096F8480072
:10D6F80096F87D308DF80530072201A901F0B5FBB9
:10D7080000283FF426AF636896F84800019300228A
:10D7180001A901F0AAFB00283FF41BAF6C36D4E93D
:10D72800010186E8030070E7304E037A8DF8043073
:10D7380096F8480096F87D308DF80530072201A943
:10D7480001F093FB00283FF404AFB436E7E7274E17
:10D75800037A8DF8043096F8480096F87D308DF8F5
:10D768000530072201A901F080FB00283FF4F1AE43
:10D77800D4E9010106F1740383E8030096F818312F
:10D78800022B7FF442AF96F83031002B3FF43DAFC7
:10D79800174BDB6A9847FEF775F936E7134E037A9D
:10D7A8008DF8043096F8480096F87D308DF80530ED
:10D7B800072201A901F059FB00283FF4CAAEBC3684
:10D7C800ADE74368029301238DF80C30074B02A99B
:10D7D80093F8480001F056FB00287FF416AFB8E62E
:10D7E800436802930023EFE7EC1C00202817002071
:10D7F8002C43010803795A1E0E2A3FF6AAAE934A13
:10D8080082F8683001E7914B42685A65FDE68F4B14
:10D8180042689A65F9E68D4B4268DA65F5E68B4B06
:10D8280042681A66F1E6894B42685A66EDE6874C0B
:10D83800037994F848008DF80430062201A901F014
:10D8480014FB00283FF485AE9DF8043084F8DD30E1
:10D85800DBE67E4C03798DF8043094F8480094F8A0
:10D868007C308DF80630052201A901F0FEFA002867
:10D878003FF46FAE9DF8043084F83930C5E6734C38
:10D88800037994F848008DF804300A2201A901F0C0
:10D89800ECFA00283FF45DAE9DF8043084F8DC30E3
:10D8A800B3E66A4C037994F848008DF804300922ED
:10D8B80001A901F0DAFA00283FF44BAE9DF80430D4
:10D8C80084F83830A1E6614B4268C3F89420DA64E2
:10D8D8009BE65E4B027983F8982083F8502094E603
:10D8E8005A4B4268C3F884208FE6584B4268C3F805
:10D8F800CC208AE6012B40F0A480554C24212046F8
:10D9080003F050FA636A984201D0172022E61C21DE
:10D9180004F1280003F046FA636C9842F5D14FF4FD
:10D92800807104F1480003F03DFAD4F84831984278
:10D93800EBD1D42104F5A67003F034FAD4F82032E0
:10D948009842E2D1002104F5097003F02BFAD4F8CB
:10D9580024329842D9D14FF4607104F50A7003F06B
:10D9680021FAD4F8A8359842CFD1142104F2AC504A
:10D9780003F018FAD4F8C0359842C6D1334E214680
:10D98800304640F2C45203F0F7F9204640F2C45240
:10D99800002103F005FA95F81B3485F8E833736F16
:10D9A800C5F8EC3396F87D3085F8F83340F201235A
:10D9B800A5F8FA33274B96F819019B6D984724E68A
:10D9C8008379012B3FF6C5AD204B42684068C3F808
:10D9D8002C2100F0BDFE48E61C4B4268C3F890209D
:10D9E80013E61A4B027983F81F210EE6174B82883B
:10D9F800A3F8882009E6154B8288A3F88A2004E654
:10DA0800124B8288A3F8D020FFE5104B8288A3F838
:10DA1800D220FAE50D4B93F848200AB1062A12D114
:10DA2800A288A3F8A025F0E5084B93F848200AB18E
:10DA3800062A08D16268C3F8A425E6E500F098FB39
:10DA4800DBE5012086E5182084E500BF28170020C3
:10DA5800641100202C4301082DE9F04387B000230E
:10DA6800ADF800300646002800F0EE800361FEF7AE
:10DA780047FD20B10124204607B0BDE8F08300F03F
:10DA880065FD0028F6D100F05BFD014618B96F4826
:10DA9800142203F085F96E4D95F89134012243F074
:10DAA800040385F8552485F8913433788DF80430CB
:10DAB8000021013B8DF80520ADF806100C2B00F273
:10DAC800BB80DFE803F007B9B9B97982B9B990B971
:10DAD800AD9AA900D5F8407317F02007CAD196F877
:10DAE8000480B8F1020F46D1DFF868815A4CFEF77E
:10DAF80063F896F9051098F848003A4601F00FFACD
:10DB080088F83900B37988F83830384607238DF813
:10DB18000530FDF7E5FFFF2304F58670A5F80C3105
:10DB2800C5F8084185F8047103F04EF804F58A70C9
:10DB380003F004F83846FDF72DFE0446002839D0D6
:10DB480096F9051098F84800012201F0E8F988F8DC
:10DB58003900D5F894343361002C71D000F0F0FC12
:10DB6800002888D195F8913485F81A0460F3820367
:10DB780085F891347FE7B8F1010F4FF00204E8D13E
:10DB8800DFF8D0908DF8144099F8480089F81D7195
:10DB980002A901F065F9337989F830318DF80570FB
:10DBA8008DF80680FDF7C4FC95F8913443F0100316
:10DBB80085F891340024CCE700226946022000F061
:10DBC800F3FA0028F6D01324C3E7244BB288DB6BA2
:10DBD80096F90C10B0689847D5F8403343F0020323
:10DBE800C5F84033E6E702A90D2000F053FB0028F2
:10DBF800E0D0002269460D20E1E7164B93F8183172
:10DC0800D3B9347904F0070000F0ABFA8DF800407E
:10DC1800012269461020D2E7002269461220CEE789
:10DC28008DF8072000F08EFA044638B900F087FA1C
:10DC3800204600F089FABDE702248AE7012488E734
:10DC480001A800F0D1FB16E7032414E740210020C7
:10DC5800EC1C002028170020EE1C00202C43010893
:10DC68002DE9F04F99B08046059118B9032019B0F5
:10DC7800BDE8F08F00230361FEF742FC044600284C
:10DC880040F0A58046460FCE0EAD0FC5142252486F
:10DC980098F800A0B8F80C7098F90EB04F4E2146CD
:10DCA80003F07EF84E4B012283F8412496F8302188
:10DCB800022A25460BD196F81821022A07D196F890
:10DCC8001E2122B9BAF1010F38BF4FF0010ABAF18B
:10DCD800010F2BD0BAF1030F2AD0BAF1000F33D1BC
:10DCE80002229DF83C30DDF84090029362F347151C
:10DCF800012496F87C108DF8321002220CA996F8AF
:10DD080048008DF8302001F09DF896F81A3196F801
:10DD180030C196F81D1140B2002B63D0BCF1010F41
:10DD280057D1002955D1002C61D153E00422D8E7FE
:10DD38000023DDF83C90BDF840709DF942B0029395
:10DD480065F01F050124D4E74FF0000BD946CDF844
:10DD580008B0CEE74FF0010084F81A04D2E005F2CB
:10DD68009A420BA900F0D4FA002800F0158113207C
:10DD7800049B33871A4B002283F81A2423E105F207
:10DD88009A452A460BA900F0C3FA0028EFD10B9B4D
:10DD980084F82801C4F82C5184F83031FCE0B9F13A
:10DDA800000F00F0F980002A00F0F6804946E01CD8
:10DDB80002F0E2FF94F8373201332380ECE01220BE
:10DDC800D6E70220D4E70720D4E71320D2E70120C2
:10DDD8004DE7FCB90220F6E02C210020281700208E
:10DDE800EC1C0020002CF5D05845B8BF584696F8D2
:10DDF8007C308DF82000052296F848008DF82230F6
:10DE080008A901F032F800283FF430AF9DF820301F
:10DE180086F839306F4A704BD2F89804D3F890409E
:10DE280038B105F087FA6C4B84423CBF002283F876
:10DE38003A20198F1A8F93F830010491996A099141
:10DE480052BA0028BFD093F81B0100B9186393F8A1
:10DE58001801ADF85820013893F87C2093F81A413E
:10DE68001491D0F1000BD3F888108DF85B204BEBA0
:10DE7800000B93F8482093F83A0093F868308DF82F
:10DE88005A3009AB0093554B03904FF001008DF8C1
:10DE98004C0015918DF85C20A3F12F01A3F13002FD
:10DEA80013A88DF84D4000F0DBF8039B4FEA0B1BDD
:10DEB8004BEA431B00264BEA801B4BEAC413B145CF
:10DEC800444C039308BF37463A46494604F59C70CC
:10DED800CDE90A669B46268084F81A6402F04CFF56
:10DEE800E9B2A570C5F34215FAB2042D3A4E039B68
:10DEF80084F837223FF42EAF072D3FF450AF022DA0
:10DF08007FF45FAF364D84F80D110420029984F830
:10DF18000401FF2084F80C0184F8281184F81431D6
:10DF2800D6F8E410C4F8085105F59B730AA8C4F89C
:10DF3800101184F83021C4F82C3100F011FC0028AD
:10DF48007FF43DAF0A9BA4F844040BA8A4F816314B
:10DF5800C4F84C3400F0D0F900287FF408AF0B9BCC
:10DF6800D3B196F93900FDF7F7FA94F83732002B58
:10DF78003FF405AF0B9B0F2B3FF6F1AE05F58B7207
:10DF88000BA90F2000F0C4F900287FF4F0AE0B9B1A
:10DF980063F3030B84F814B10598FDF7FBFB002825
:10DFA8007FF4E6AE099B86F83A00B36200F080F988
:10DFB80000287FF40AAF94F8913484F840A443F021
:10DFC800010384F89134034BD3F89434C8F8103023
:10DFD8004DE600BFEC1C00202817002090170020F9
:10DFE800EE1C002037B50B4D8DF8040004460F22B7
:10DFF80095F8480001A900F038FF40B1064A85F8B5
:10E008001C4192F8913443F0200382F8913403B014
:10E0180030BD00BF28170020EC1C002010B5FFF70A
:10E02800C1F8044688B90A4805F0BEF9094805F060
:10E03800BBF9094805F0B8F900F094F8FDF7BCFD04
:10E04800064BDB6A9847204610BD0124FBE700BF5A
:10E05800542000206C200020842000202C4301083C
:10E068002DE9F04F8BB047780093149B90F90C8002
:10E0780090F90D6090F80EB08A4641681960044620
:10E088009146002F58D002238DF8103004A9C37B85
:10E09800007C8DF8123000F0D5FEB4F808C0618914
:10E0A80043B26068984545466144B8BF1D4660451F
:10E0B80034BF00270127884209D30A218DF81010A0
:10E0C800207C019304A900F0BDFE019B46B2B4F880
:10E0D80008C0608961680CEB400E714519D3A1EB4B
:10E0E8000C01B1FBF0FC00FB1C1191B9984503DC55
:10E0F8002378CBB94FF0010B21238DF81030207C09
:10E10800E37B8DF8115004A98DF8123000F09AFEC7
:10E1180045B2009B8AF80050384689F8006083F8B9
:10E1280000B00BB0BDE8F08F0223207C8DF82430BE
:10E1380006A900F095FEDDE74546EAE77047704717
:10E14800704770470020704770477047704700203D
:10E15800704700207047002070470020704700205B
:10E168007047704770477047022070470220704719
:10E1780002207047704700207047704770470020A2
:10E1880070470020704770477047704710B5054CBE
:10E198004FF403722046002102F002FE0020C4E979
:10E1A800000010BD082200202DE9F8438146904662
:10E1B80000293CD01F4C2023224604F1100012F8FD
:10E1C800017F6FBB8242FAD11B4E3368013403B919
:10E1D8003460736803B11C6000252560C4F80880AA
:10E1E80074601FFA88F284F80490601D02F0C4FD80
:10E1F800B9F1110F4FF0000398BF104D6373D6F8B3
:10E20800083298BF25FA09F503F1010398BF05F014
:10E21800010543442573C6F808323846BDE8F8833B
:10E22800013B13F0FF030446C6D10227F5E7012797
:10E23800F3E700BF0F220020082200202007020079
:10E2480010B518B3124A1368984204D103681360D2
:10E25800002305E00B46002BFAD019688842F9D153
:10E268005168884208BF53600BB101681960D2F841
:10E2780008328168013B00245B1A04602146C2F819
:10E288000832102202F08CFD204610BD0120FCE768
:10E2980008220020054B1B6813B11A798242FAD173
:10E2A800002B0B600CBF03200020704708220020C1
:10E2B80010B5054B186800B910BD037B04680BB98D
:10E2C800FFF7BEFF2046F6E70822002038B5084BC6
:10E2D800084C186800B938BD03790568112B05D8B2
:10E2E80024FA03F3DB0701D5FFF7AAFF2846F1E775
:10E2F800082200202007020028B1044BD3F8083276
:10E308000360002070470120704700BF08220020EA
:10E318002DE9F04107460E46154642B339B3154B71
:10E328001C6800232CB93046FFF7E6FF0020BDE843
:10E33800F081A268F91A0132914215D32279EA5480
:10E34800581C22895FFA80F8611D55FA80F002F0A6
:10E3580013FDA368246898445FFA88F3E2E720462F
:10E368002568FFF76DFF2C46002CF8D1DBE701206C
:10E37800DDE700BF082200200238C0B211289ABF8A
:10E38800014B185C00207047433C010830B50B4B2B
:10E3980093F820200446084672B100211C33057802
:10E3A800A54208D001319842CDB214BF04301038CC
:10E3B800AA42F4D8002030BD1046FCE714240020FF
:10E3C80010B5084C00232060142204F10C00FF2132
:10E3D80084F82030C4E9010002F0E2FC012384F84B
:10E3E800213010BD1424002010B50E4A92F82010D8
:10E3F800042915D8936804781C7044785C70C47834
:10E40800807898700131DC7082F8201002F11C01CC
:10E418008B4214BF043302F10C039360012010BD3A
:10E428000020FCE714240020094B93F8200068B171
:10E438005A6803F11C018A4200F1FF3014BF04320C
:10E4480003F10C0283F820005A600120704700BFD6
:10E458001424002010B5074B93F8202004460846E2
:10E4680032B15968FFF792FF10B1012344708370ED
:10E4780010BD00BF1424002008B5064B93F82020D7
:10E488002AB15968FFF782FF08B1407808BD01201A
:10E49800FCE700BF1424002030B50A4A92F8201087
:10E4A800536882F8210061B1916801241C32DD783B
:10E4B800587005B99C70934214BF0433103B9942BD
:10E4C800F5D130BD1424002008B5044B5968FFF776
:10E4D8005DFF003818BF012008BD00BF14240020CC
:10E4E800F7B50422154E044600210DEB020096F8FC
:10E4F800207002F055FC0025EBB29F4201D803B012
:10E50800F0BD7368197821705A786270987838B1BC
:10E51800336820469B689847FFF786FF0135EBE78D
:10E52800DB788DF804108DF805208DF80730FFF79B
:10E538007BFF01A8FFF758FFF0E700BF1424002075
:10E54800014B93F82000704714240020034B93F8E4
:10E558002000042894BF00200120704714240020C4
:10E568001FB50024CDE90244C41F8DF800408DF882
:10E5780001100C0AADF80420090C120C8DF80310D8
:10E588008DF806208DF8073002461B0A01216846DF
:10E598008DF802408DF8083002F05DFA002818BFA7
:10E5A8000E2004B010BD2DE9F04188B090460D460C
:10E5B8000F9A0746002847D000240121CDE90444DA
:10E5C8008DF810109DF838108DF81510ADF816302C
:10E5D800190CCDE900441B0ECDE902448DF8193021
:10E5E800ADF81A20130C120E07948DF818108DF838
:10E5F8001C308DF81D20E3B21E01002DF6B203DC9D
:10E60800002008B0BDE8F081013310218DF81F30DB
:10E6180042466B460DEB010002F0B3F90346A8B978
:10E62800102D28463E44A8BF10206946327811F8BC
:10E6380001CB013382EA0C02984206F8012BF5DC83
:10E64800103D2DB20134D6E70920DAE70E20D8E7CD
:10E658000138032815D8DFE800F002080C100A4B2F
:10E668001B681B690B6000207047074B1B685B69C0
:10E67800F8E7054B1B689B69F4E7034B1B68DB69EC
:10E68800F0E70520704700BF382400202DE9F0414D
:10E69800C4B00C464A9E17461D468046B8B3B1F52D
:10E6A800807F36D84FF488720021684602F078FBE4
:10E6B800492300934FF48073ADF804302B0C8DF888
:10E6C8000830330CADF80650ADF80A608DF80C3000
:10E6D80022460023414604A82D0E360E8DF80E3032
:10E6E8008DF809508DF80D608DF80F4002F044FB4D
:10E6F80004F110014B9A3B4689B2684602F02BF9A7
:10E7080010B1012818BF0E2044B0BDE8F0810920DF
:10E71800FAE70D20F8E7000010B590B10A4C28225E
:10E728000021206002F03CFB2368084A1A600020A0
:10E738004FF0FF32C3E90302C3E90522C3E9072208
:10E7480010BD0820FCE700BF3824002000010101AB
:10E75800024B1B6818600020704700BF3824002057
:10E7680030B1044B1B68DB6801330360002070473D
:10E77800092070473824002013B500230C46019364
:10E78800CAB101A9FFF764FF18B9019B591C02D14E
:10E79800146002B010BD99B2611A002901DD5C183D
:10E7A800F6E702D113600720F3E71B0C1B0403F5FF
:10E7B80080331C44ECE70920EBE7000028B1044B48
:10E7C8001B681C334362002070470920704700BF54
:10E7D800382400201FB5044600B3002303A8039380
:10E7E80002F090F9104ABDF80C3012682046938068
:10E7F800E38200F05EFA98B904F1180300932168E7
:10E808000123132202F09CF860B9204600F051FA67
:10E81800003818BF0120000104B010BD0920FBE733
:10E828001020F9E70E20F7E738240020F0B5054658
:10E8380087B01C4613B9092007B0F0BD2E4E3368C7
:10E84800DB68834255D894F82020002A0CBF0822A0
:10E858000922834205D3204600F05FFA68B11020F0
:10E86800EAE7002301900093A36894F82810606AEF
:10E87800FFF799FE0028EED0DEE723792168B4F887
:10E8880008C0A768043B9AB20029D4D0B2F5807FAB
:10E898002DD8ADF80EC08DF817304FEA174C04F19B
:10E8A8002C033F0E8DF8117000932F0C08234FF0A6
:10E8B800490EADF80C008DF814708DF816002F0E67
:10E8C8000DEB0300CDF808E08DF810C0ADF812503C
:10E8D8008DF8157002F034F808B10E20ACE7204628
:10E8E80000F01BFA0028BAD13368DD60A4E70D20D8
:10E8F800A2E70620A0E700BF382400202DE9FF4149
:10E908000A9D80460F4616461C46002D5AD0002305
:10E9180003A910460393FFF79BFE18B1062004B025
:10E92800BDE8F081039B9C4201D80133F6D128460B
:10E9380000F064F9002847D1264B1A78424503D0E5
:10E948001A79424542D10120AA68BA4240D103EB64
:10E958008002EB6A92F801802979CDE900430439F5
:10E96800927828683B4689B2FFF790FE0028D6D1F6
:10E9780095F820300194002B4FF00103009314BF49
:10E988004246082295F82810686A3B46FFF70BFEB6
:10E998000028C4D1013E032EC1D8DFE806F00207E3
:10E9A8000B0F0D4B1B681C611C62B8E70A4B1B68F8
:10E9B8005C61F9E7084B1B689C61F5E7064B1B682F
:10E9C800DC61ACE70920AAE70F20A8E70B20A6E73F
:10E9D8000220A4E7A4080020382400201FB50B2932
:10E9E8004FF00003CDE90033CDE902330A4607D0E2
:10E9F8000C2914D00A2910D00A2005B05DF804FBB0
:10EA0800012802D120238DF800300021684602F049
:10EA180022F8002818BF0E20EFE73023F3E70B2178
:10EA2800F4E7000038B5054602F010F8044610B1C6
:10EA38000E24204638BD002DFBD1094B1B680B2145
:10EA48009878FFF7CBFF0028F2D10C21FFF7C6FF1B
:10EA58000028EDD10A21FFF7C1FF0028E9D0E7E738
:10EA6800382400202DE9F04380468FB00C46174625
:10EA7800002A6BD0002969D0002529461D2206A846
:10EA8800059504F0A7FE8DF81350344D2B680DF151
:10EA980014099E88CDF804900DF1130302933B7975
:10EAA80000933B6832462146404601F0F0FF0028BB
:10EAB8004ED138683A79494602F05EF9384600F096
:10EAC8004FF8002846D13C7AFA79BB79240444EA05
:10EAD80002241C432B689A6894423DD99C609DF897
:10EAE80013000B21FFF77AFF034658BB0C21FFF7F1
:10EAF80075FF034630BB0A21FFF770FF034608BBCA
:10EB08007B7ABA7AFF7A3F0447EA02271F433A46DC
:10EB1800334621460920FFF723FD034690B93346C3
:10EB28003A4621460820FFF71BFD034650B92A68DC
:10EB38009DF8131091700021D1604FF0FF31C2E9A8
:10EB48000411916118460FB0BDE8F0830923F9E775
:10EB58000E23F7E70F23F5E70323F3E73824002014
:10EB680010B50446002845D00168002942D011F8A4
:10EB7800013B43710322063002F0FEF820460322CF
:10EB880050F8091B043102F0F7F82168CB79E360EB
:10EB98000A7A43EA0223E3604A7A43EA0243E360DB
:10EBA8008A7A43EA0263E360CB7A23740B7B63744B
:10EBB8002379212B1AD110220D3104F1120002F011
:10EBC800DBF81D222168501C8B5C6362085C43EAF9
:10EBD8000023901C6362085C033243EA00436362CB
:10EBE8008A5C43EA02636362002010BD112B03DCD8
:10EBF8000D22E7E70220F8E70120F6E710B5044602
:10EC0800002854D00168002951D00B7843714B7803
:10EC180083608A7843EA02238360CA7843EA02431E
:10EC280083600A7943EA026383604B7903738B79C3
:10EC3800C381CA7943EA0223027BC38102F00F022F
:10EC48000831103002F098F8237B002203F00F03FC
:10EC580084F8202084F82820227903F10800111A6A
:10EC680004290DDD21680933043AD21A085C84F8B6
:10EC78002000D2B2606A84F82820194402F07CF897
:10EC8800237922681A44002012F8043CE36212F83F
:10EC9800031C43EA0123E36212F8021C43EA01431E
:10ECA800E36212F8012C43EA0263E36210BD02201A
:10ECB800FCE710B5044660B3036853B30279162A1B
:10ECC80029D942791A700146082251F8060B0130F9
:10ECD80002F05CF82146082251F80E0B093002F0C8
:10ECE80055F82368E28A5A74E38A22681B0A9374E7
:10ECF8002368A269DA74A36922681B0A137523685A
:10ED0800628B5A752368E27E9A7517232371002057
:10ED180010BD0120FCE70220FAE738B504460028B8
:10ED280063D00168002960D0037B90F8282003F0A5
:10ED38000F03002A57D1083320790432134498422C
:10ED480055D363790B702368A2685A70A368226848
:10ED58001B0A937023686289DA702368E27A1A7151
:10ED68002368227B5A712368E2899A71E3892268B1
:10ED78001B0A2146D371227B51F8100B02F00F02B7
:10ED8800083001F0F9FF237B94F8282003F00F03E3
:10ED980003F108052AB1226894F82010515503F1AF
:10EDA8000905206894F82820616A284401F0E4FFE6
:10EDB80094F828302268E16A2B44D1545A1CE16A3D
:10EDC800206892B2090A81549A1C2168E08D92B297
:10EDD8008854DA1C216894F82F0092B204338854BE
:10EDE8002371002038BD0933A6E70120FAE7022085
:10EDF800F8E70000024B1A8810431880704700BFDC
:10EE08003C24002008B5074B1B883BB1FEF7CAF924
:10EE1800002814BF6FF00200002008BD6FF0010049
:10EE2800FBE700BF3C24002010B5034B00241C80E6
:10EE3800FEF7AEF9204610BD3C240020B0FA80F061
:10EE48004009704782B018B9084602B000F0CAB845
:10EE5800002002B0704710B9084600F077B9704733
:10EE680010B9084600F08EB97047034608461146A7
:10EE78000BB900F0E5B90020704710B9084600F05A
:10EE88006DBD704710B9084600F006BA00207047FB
:10EE980010B40446084611461A46019B14B910BC22
:10EEA80000F014BA10BC70470346084611460BB967
:10EEB80000F03EBA0020704710B4044608461146D8
:10EEC8001A4614B910BC00F0ABBA002010BC704749
:10EED80030B40546084611461A46DDE902341DB924
:10EEE800029430BC00F02ABB002030BC704710B937
:10EEF800084600F0DBBB0020704710B9084600F058
:10EF08006BBD0020704710B9084600F0EABB00202E
:10EF1800704710B9084600F0E7BB00207047034669
:10EF2800084611460BB900F001BC0020704710B428
:10EF38000446084611461A46019B14B910BC00F055
:10EF4800F7BB092010BC704710B4044608461146A8
:10EF58001A4614B910BC00F061BDC8B210BC7047A5
:10EF68000048704701000102064B10B51B6A0446B1
:10EF7800984730B10448054B204498428CBF002084
:10EF8800012010BD2C43010840C220C980B92A00C5
:10EF9800F0B5114B85B00C4610491F56054601F0D7
:10EFA8004BF80F4BE4B25E6A072D4FF00103CDE931
:10EFB800024301460AD105220023CDE900234FF47C
:10EFC8007A727A431846B04705B0F0BD082200208F
:10EFD800CDE900203A46F5E7103D0108F03C01086C
:10EFE8002C4301081FB5002300930378013B372BFE
:10EFF80021D8DFE803F01C242020201E2020202018
:10F008004143454E2055585B5E6164206C1E6E730B
:10F01800787A20207D812620202020202020202072
:10F028002020202083858A2020838A208C90C37802
:10F038000BB102230093009805B05DF804FB8378B8
:10F04800F6E743788DF8043005238DF8053083788A
:10F05800003B18BF01235B008DF8063010238DF8A4
:10F068000730304B1B6801A803F55872CDE902231D
:10F0780000F0C2FF0090DEE74023DBE72023D9E75A
:10F08800827890F9013012B9274AD35CD2E7274A2F
:10F09800FBE7827890F90130002AF8D1244AF4E796
:10F0A80040F6B833C6E74FF47A73C3E74FF4FA6310
:10F0B800C0E741F28833BDE741F27073BAE71D48F3
:10F0C8004FF47A7101F03CFE00F5FA60D2E71A4B72
:10F0D800B0E7144B1B6803F55873ABE7114B1B687B
:10F0E80003F55B73A6E71023A4E70E4B1B68A1E7A3
:10F0F8004FF0834300939EE7104BFBE7104B99E7D3
:10F1080040F21113ADF8003095E7032392E790F928
:10F1180001300C4AB9E70C4990F9010000F08CFF66
:10F12800A8E700BF44240020E53C0108D53C0108BD
:10F13800DD3C010818FCFFFF00EA06379A990940F0
:10F1480040F70937103D0108F03C010837B50B4B73
:10F1580002781B680C2101FB02335B7A03EB430442
:10F16800074B1D6803690093C3684278816805EB03
:10F17800C40000F0DDFC03B030BD00BF4424002013
:10F188004024002070B586B0027B6423ADF80030BF
:10F19800012A4FF00003CDE90133CDE903338DF89F
:10F1A80002308DF8143030D0022A39D05ABB0368A7
:10F1B8004BB343683BB31F4D80682B601E4B18222E
:10F1C8006946186001F0D8FD1C4B2C6893E80700CD
:10F1D8000C3384E8070093E8070004F10C060323C6
:10F1E80086E80700A4F86C33012204F55B7104F586
:10F1F800587000F08EFC2B684FF6B072A3F8782395
:10F208000522C3F87C2306B070BD0A49086843602C
:10F21800036100F55B7100F5587000F07AFCF2E7C5
:10F22800044B1B68B3F86023B3F86C130A43A3F8C4
:10F238006023E8E74424002040240020C83901085E
:10F2480008B503460A2924D8DFE801F0062323235A
:10F25800230B161B23212100BDE808400068FFF797
:10F2680083BE90F900009978052271B900F011FC6D
:10F27800003818BF012008BD052293F900000021BD
:10F28800F4E790F900005978EEE70221EEE707224B
:10F29800F3E70020EFE7000008B502791AB1012A68
:10F2A8000BD0002008BD084B01681B68012203F53C
:10F2B800587000F02EFC0120F4E7034B01681B682E
:10F2C80003F55B70F5E700BF44240020F7B5052877
:10F2D800144D1C46A8BF052058700E4629461746EF
:10F2E80000F0AAFE94F90130A070072B13D1322048
:10F2F80000F0A2FD0C4BDB6D0546984704F10C02AB
:10F3080008340346019200943A463146284600F0F4
:10F3180098FD03B0F0BD054A55F82310D05C00F005
:10F3280083FDE7E7F03C01082C430108103D010884
:10F338002DE9F04F344F90F901607B68D0F80490C4
:10F348008BB00446884698470546002859D1E37C87
:10F3580073B92E4A2378126803EB4303990002EB32
:10F368008303D3F80490B9F1000F01D152F801904A
:10F37800274B484613F906B0FB689847A37C2289B7
:10F38800D7F818A00993072E28D100230121CDE929
:10F398000223204A0693CDE90431CDE9073305213C
:10F3A800CDE900214FF47A7202FB0BF24CF2503196
:10F3B8001846D047637C13B3174B995D7B6D0D31AD
:10F3C800C9B228469847E07C3246494600F046FED6
:10F3D80088F8006001200BB0BDE8F08F00210125FE
:10F3E8000823CDE90013CDE90715CDE90511CDE9CD
:10F3F80003110292A1782B465A462846D9E7074BB3
:10F40800DBE70020E7E700BF2C4301084424002085
:10F41800103D010885450100DD3C0108E53C010877
:10F428002DE9F04F8DB090F90130DFF8FCA0DFF83E
:10F43800FC90CDE90A123E4A12F903B00278DAF8D4
:10F4480000300C2505FB02333A4A5B7A126803EB5D
:10F45800430302EBC303044693F9021090F9020038
:10F4680000F0E5FD3449064694F9010000F0E4FD9A
:10F47800A26861688046304600F00BFD2178DAF812
:10F488000020D9F80C306943074650589847D9F8F6
:10F498001C309C4694F901300025072B4FF47A6301
:10F4A800CDE90753CDE905552DD10123CDE9035306
:10F4B8000523CDE901534FF47A7303FB0BF3009353
:10F4C8003946434646F2A81228466746B847237885
:10F4D800DAF800200C214B4394F90110D05800F0C1
:10F4E800DFFDA18994F90100FFF752FD0B9B217BF9
:10F4F8001860D9F85430284698470A9B01201E7096
:10F508000DB0BDE8F08F01200823CDE90350CDE907
:10F5180001032A46CDF800B0654643463946A84758
:10F5280001200546D3E700BF442400202C430108EE
:10F53800103D010840240020F03C01082DE9F04F5F
:10F548008FB0002405468A46914698460494ADF843
:10F558001440ADF8024007264FF0010B2B7AA34266
:10F5680006D9686804A9204400F0F6FB00285ED19B
:10F5780002238DF8083002A86B7A8DF80A30FFF75D
:10F5880031FDAB7A8DF81D309DF811308DF81E30A5
:10F598009DF812308DF81F309DF810308DF820300E
:10F5A800EB7A8DF821302B7B8DF822306B7B8DF830
:10F5B800233010238DF81C608DF824303A4E8DF8D6
:10F5C8002C000DF102030A9305238DF82D303368C2
:10F5D8000C930723ADF834302B6806930DF1120213
:10F5E80004AB0DF1110106A800F0D0FB0728054671
:10F5F8000BD130680C22002100F5587001F0D0FBC7
:10F608003368BDF80220A3F860239DF811308AF80A
:10F6180000309DF8123089F800309DF8103088F8D5
:10F628000030189B28461C700FB0BDE8F08F9DF87D
:10F638001330BDF81470ADF802702044C4B2F3B9A9
:10F6480017B3194A00201168072602464FF00C0C20
:10F65800062B1BD10CFB00FE51F80EE0BEF1000F8B
:10F6680004D00BFA00F23A4397B201220130102875
:10F67800EED1002A3FF472AFADF802706EE75A1E61
:10F68800042A01D9062BDCD0062667E747FA00FED4
:10F698001EF0010FEAD00CFB00FE51F80EE0BEF19F
:10F6A800000F08BF0626E1E74424002038B50546C8
:10F6B8004068FFF759FC0522841D002195F90000D8
:10F6C800E4B200F0E6F908B904F0FD0495F9010088
:10F6D8000722002100F0DDF908B904F0FB042046F8
:10F6E80038BD00207047000010B503780F2B044682
:10F6F80018D84068FFF738FC22780B4902EB420221
:10F708000968831C01EB820051F82220DBB21AB988
:10F7180003F0FD0358B210BD032B06BF62684260B8
:10F728000223F7E70020F6E7442400200220704770
:10F738002DE9F04FDFF838810446D8F8000099B079
:10F748008946174600211E460122032300F55870FA
:10F75800CDE90611CDE908118DF814108DF81510B2
:10F76800ADF8163000F0B7F938B9D8F80020B2F87B
:10F77800603343F00303A2F86033D8F80020637ABB
:10F788008DF8283002F55871CDE90B12394A94F9F1
:10F79800083012680D920DF116020F92226810922D
:10F7A80062681192D4E90301A27A8DF848200122F7
:10F7B8008DF8492013AA82E803001025227DE18AEA
:10F7C8008DF8293018468DF85420ADF83850FFF7D9
:10F7D800DFFB0AAB17930DF1150316900093314622
:10F7E800019705AB06AA10A800F0C2FB064698BB15
:10F7F8009DF81410204F013901F0A2FA1F4B1B6924
:10F808000393C4B24FF00C0B04F160036B44D8F8B7
:10F81800000013F848AC9DF814300BFB0AFC0134C7
:10F828003946B4FBF3F203FB1244D0F87C33B0F949
:10F83800782350F80C00DDF80CC0E4B2E04728B19A
:10F8480089F800A0304619B0BDE8F08F013D15F0E9
:10F85800FF05D9D10D26F5E70C2801BFD8F80020FF
:10F86800B2F8603343F00303A2F86033EAE700BF5D
:10F878004424002040240020400D03002C430108AC
:10F88800F8B50679012E054648D90F2E48D80368E1
:10F89800187A40F303000522002140B200F0F9F87D
:10F8A8002B680446187A40F303100522002140B261
:10F8B80000F0EFF8B8B1B4FA84F4640929680B7A57
:10F8C800086843F3030243F303135BB252B29A424C
:10F8D800C8BF0124FFF748FB80F00103DBB224B165
:10F8E8000533D8B2F8BD0124E8E7DBB90E4F296823
:10F8F8003B6806EB460003EB80000C2201F03CFA63
:10F908003A680C2303FB062320465C72B2F86013A6
:10F918000123B3400B43A2F86033E3E70620E1E795
:10F928000320DFE70420DDE74424002010B4017839
:10F9380001290ED9084B18680C234B43C418002220
:10F94800C250C4E9012200F5587010BC102200F022
:10F95800A9B8002010BC7047442400202DE9F041CC
:10F9680086B050238DF81430037A102B074630D117
:10F978004368DD7B6DBB0224A8466426062C14D898
:10F988007A68535D03932A44517843EA0123039329
:10F99800927843EA02437343CDE9033863B9684672
:10F9A8008DF80040FFF7C2FF0DE0CDF80C808DF810
:10F9B8001480CDF81080F2E703AB01A801938DF80D
:10F9C8000840FFF75DFF0134E4B2102C05F1030590
:10F9D800D4D106B0BDE8F0811FB50268037911687B
:10F9E80049B901A88DF80430FFF7A0FF78B10320CA
:10F9F80005B05DF804FB02A802928DF80C30FFF701
:10FA08003FFF042805D0052805D00028EFD00020A6
:10FA1800EEE70220ECE70120EAE70000C90020B980
:10FA2800034B0B449856C0B27047024BF9E700BF2E
:10FA3800953C0108553C0108F0B59A42069D03DB48
:10FA48009DF914309A4220DD0020F0BD03EB4303FA
:10FA580031F814C005EB830300264CFA06F7FF07BC
:10FA680007D51F7A07F00F0E964502DCB2EB171F79
:10FA78000DDD0136102E03F10C03EED10134E4B292
:10FA88002301DBB29842E1D8DEE70024F8E7012041
:10FA9800DBE7884204DB9042CCBF0020012070479E
:10FAA8000020704710B51409B4EB111F03464FEA44
:10FAB80011100ED391420CD202B201F00F0133F8AB
:10FAC8001240012000FA01F124EA010123F8121082
:10FAD80010BD0020FCE7F0B528B100EB4105012777
:10FAE8000020914200D3F0BD002435F802CB234614
:10FAF80007FA04F636EA0C0608BF013304F10104DC
:10FB080008BFDBB2102CF3D118440131C0B2C9B21E
:10FB1800E7E710B500B149B910BD31F8134020F836
:10FB280013400133DCB2A242F7D8F5E70023F9E726
:10FB380082B030B504880493D2B9B3F5616F15D398
:10FB480049F6AF2542F21072AB4298BF4FF47A7271
:10FB5800944238BF14466143BDE83040C3688B42C5
:10FB68008CBF5B1A0023C36002B070476422EFE7C2
:10FB7800012C38BF0124EEE72DE9F04F8FB0154670
:10FB8800199F03939DF8603007930C46804603F055
:10FB9800C7FB6A4A0590A7F5F633303BB3FBF2F38F
:10FBA800534303F5F63B0493182313FB05430BF16A
:10FBB800300B069300254FF0FF3A069B9C4207D175
:10FBC800002D14BF50464FF0FF300FB0BDE8F08F46
:10FBD800BDF96830ADF82430099919973846089767
:10FBE80003F02EFB2688B8F1000F5FD1B7F5616FDF
:10FBF8005AD349F6AF2242F21073974298BF4FF496
:10FC08007A739E4238BF1E46642E59D1DFF8309170
:10FC1800A060A1680CA803F035FB0D9B0093DDE9FB
:10FC280008120C9B0AA803F08CFA039A0A9B0AB9DB
:10FC3800079A2AB122694A4502D1424A93420ED90B
:10FC4800414BC4F80C909F4209D90023ADF82C30E1
:10FC58000B99CDF828B0584603F0F2FAA060606816
:10FC680008B9C4F80C90C4F81090B8F1000F04D08B
:10FC780003F060FBE3680344E360D4E90332934292
:10FC8800059B88BFE26063601B9BE16873439942F0
:10FC980004D20398E8B9B8F1000F1AD001231D4423
:10FCA8002375EDB2183488E76423AAE7039B0BB9E0
:10FCB800234BE360012EDFF8889038BF0126CEE79A
:10FCC800B6F57A7F0ABFDFF88490DFF88490A060E9
:10FCD8009FE700209342207506D85B1A9A4505F1E4
:10FCE800010528BF9A46EDB2B8F1000FDAD1642EAB
:10FCF800184AADF82C801DD049F6B023B6F57A7FA6
:10FD080018BF1346974281BF049A02F5A83202F53C
:10FD1800C0729B180A931A9B00930AAE96E80600D5
:10FD2800199B304603F00DFA96E8030003F088FAB1
:10FD38008246B7E74FF46163E4E700BF80510100F2
:10FD480040771B007F5101002FEC010080A81201B1
:10FD5800002E930230EC01000378032B14D1437872
:10FD680003F00F021B098A704B7083788B80C2786E
:10FD780043EA02238B800379C3F3021203F00F03D3
:10FD8800CA700B7005207047002070472DE9F347B3
:10FD98009A464379057990F907609146044690F9A7
:10FDA80006208846D3B190F90870002D37D00F2A65
:10FDB8001BD194F909200F2E27D194F90A00072D99
:10FDC80002D1002F08BF012788F8002089F8000019
:10FDD80028468AF8007002B0BDE8F08790F90B70E9
:10FDE80090F9092090F90A60DFE7A369019394F973
:10FDF8001530009394F914302169207BFFF71CFE1D
:10FE08000028D8D105F0FD05D5E794F91D00B042CA
:10FE1800D5DC94F91C30B34203DA05F0FB05304613
:10FE2800D2E73046CBE70000024B03FA00F0B0FB04
:10FE3800F1F0704740420F004FF4FA53B3FBF0F073
:10FE4800704730B54FF47A750C1F6A4300FB0422E3
:10FE580052001EBF00F1FF341219B2FBF0F29142BA
:10FE680038BF1146039A1160820048431CBF013015
:10FE780040084FF47A71121A01FB1323002BCABFF2
:10FE880003F2E73393FBF1F1B3FBF1F1049B196043
:10FE980030BD38B5400014460D46F1F7B7FD0146B0
:10FEA8002846F1F701FD2146F1F7FEFCF1F7F0FBDA
:10FEB80003F0DEFCF1F7CCFC40B238BD2DE9F74F7A
:10FEC800019300239C469E46048A1E01F6B2B44262
:10FED80046D906EB46054FEA4309AD0000244768BA
:10FEE80037F809702741FF0729D5876807EB050A06
:10FEF8007F5927B3077837B9476927B137F80970A9
:10FF08002741FF071BD59AF8087090F901B047F30D
:10FF180003084FFA88F8D84511DC47F303177FB276
:10FF28005F450CDB9AF8097007EB4708C76807EBD1
:10FF3800C8073F7D5FB90CF1010C5FFA8CFC0134F6
:10FF4800102C05F10C05CAD10133DBB2BCE70EF168
:10FF5800010706EB040801F80E805FFA87FEEEE75A
:10FF6800019B82F800E083F800C003B0BDE8F08F81
:10FF78002DE9FF4704464068DDE90C671D468A46BF
:10FF8800914603F0D7F923681B1A3B604FF000082D
:10FF98000123337085F80080636813B123688342B6
:10FFA80024D8D4F81CC0CAF80080A3699CF800E0E3
:10FFB8000393D4E9030101AB83E80300237D009395
:10FFC800DCF80C10237A627A7046FFF7D5FD3346C9
:10FFD80038602A46E0694946FFF770FF2B782BB155
:10FFE800C7F80080002004B0BDE8F0873378002B04
:08FFF8000CBF0C200B20F6E702
:020000040801F1
:1000000037B590F9002090F90250954204460FD080
:10001000013A52B295420BD0A368019394F9013092
:1000200000936168E0782B46FFF70AFD0028EFD0C7
:10003000104603B030BD8842B8BF08467047000084
:1000400051F82000054B984205D0054BC31A584281
:100050005841400070470120704700BF90D0030016
:1000600020A1070005281FB50ED80C4B53F82030EF
:100070000093CDE901120A4B01220021022002F077
:100080006BFE05B05DF804FBCDE90012054B0122C3
:100090000021022002F060FEF3E700BF843D01086A
:1000A000183D0108373D010807B5054BCDE90001B2
:1000B00001220021022002F04FFE03B05DF804FB94
:1000C000533D010810B5102204460021F13000F024
:1000D0006BFE0021C4F814112046F022BDE8104048
:1000E00000F062BE02460846102100F0A5B92DE9D5
:1000F000F0430446D0F8140185B00E46154604F2CC
:10010000011988B3C0F110089045474628BF17462B
:10011000BAB2484400F034FED4F814313B440F2BFB
:10012000C4F814312DD9A8452BD204F1F00304F5FD
:10013000807113F8012F187C8B4282EA00021A703A
:10014000F7D104F1F10810224146684600F018FE8C
:1001500022466946684600F0F1F910226946404699
:1001600000F00EFE3E44ED1B04F5807804F1F1072B
:10017000102D09D8AAB23146484600F001FEC4F855
:10018000145105B0BDE8F08304F1F003711E13F8BB
:10019000012F11F8010F434582EA00021A70F6D1CF
:1001A00010223946684600F0EBFD22466946684653
:1001B00000F0C4F910226946384600F0E1FD10361F
:1001C000103DD5E7F0B589B00C4610220021054658
:1001D000684600F0E9FD22466946684600F0AEF93F
:1001E0009DF90030002B6A464FF0000143DA137886
:1001F00012F8010F01315B0043EAD0130F2902F816
:10020000013CF4D19DF80F305B0083F08703D4F8F4
:100210001401DBB210288DF80F303BD104F5807348
:10022000694604F5887013F8016F11F8012B9842A4
:1002300082EA06021A70F6D104F1F00304F5807127
:1002400013F8012F187C8B4282EA00021A70F7D152
:1002500010220DEB020004F1F10100F091FD2246A5
:10026000294604A800F06AF910220021684600F02F
:100270009BFD09B0F0BD137812F8010F01315B004E
:1002800043EAD0130F2902F8013CF4D19DF80F3056
:100290005B00BCE79DF90030002B6A464FF000017F
:1002A00037DA137812F8016F01315B0043EAD61395
:1002B0000F2902F8013CF4D19DF80F305B0083F068
:1002C0008703471CDBB28DF80F30102F04EB0003BF
:1002D000C0F10F064FF0800288BF002600F5817044
:1002E00083F801210021324620443E4403F076FA8F
:1002F000C4F8146104F58073694604F5887013F836
:10030000016F11F8012B984282EA06021A70F6D1A9
:1003100092E7137812F8016F01315B0043EAD613BC
:100320000F2902F8013CF4D19DF80F305B00C8E7BB
:100330000A780378534003704A78437853404370F7
:100340008A78837853408370CA78C3785340C370E7
:100350000A790379534003714A79437953404371D1
:100360008A79837953408371CA79C3795340C371C1
:100370000A7A037A534003724A7A437A53404372AB
:100380008A7A837A53408372CA7AC37A5340C3729B
:100390000A7B037B534003734A7B437B5340437385
:1003A0008A7B837B53408373CA7BC37B5340C37375
:1003B000704710B50B7814786340037054784B780D
:1003C0006340437094788B7863408370D478CB78A3
:1003D0006340C37014790B796340037154794B798E
:1003E0006340437194798B7963408371D479CB797D
:1003F0006340C371147A0B7A63400372547A4B7A68
:10040000634043728B7A947A63408372D47ACB7A56
:100410006340C372147B0B7B63400373547B4B7B41
:1004200063404373947B8B7B63408373CB7BD27B32
:100430005340C37310BD0000A1F11003DBB2102BB9
:100440002DE9F047044604D83A4820FA03F3DB07C5
:1004500005D4002382F8F030FF20BDE8F087561E57
:10046000254615F8013B06F8013F631B0B4413F0CA
:10047000FF00F6D101F11C039B005FFA83FCC3F37C
:100480000313013BDFF8B09082F8F0308846531830
:100490004FF0010EB8FBF1FA01FB1A8A1AF0FF0ABD
:1004A00013F8047C13F8036C13F8025C13F8014C86
:1004B00030D119F806A019F8056019F8045019F898
:1004C00007404FEADE1707EB47078EEA0A0A07EBF9
:1004D000C7074FEA4E0EFFB25FFA8EFE87EA0E0E96
:1004E000574692F800A087EA0A071F7057787E40A7
:1004F0005E70967875409D70D57808F104085FFAB3
:1005000088F86C40C445DC7002F1040203F1040376
:10051000C0D8A2E71829E4D9BAF1100FE1D1DFF869
:1005200018A01AF807701AF806601AF805501AF899
:100530000440D6E7010101009C3F01082DE9F04F7E
:10054000A3B092F8F0301D911B920193002B00F0A4
:10055000538101461EA8FFF72CFF1B9BA74CA84DFB
:10056000A84E10330293002303939DF87C0004905F
:100570009DF886000590205C06909DF87B00079012
:10058000205C089004989DF881C0205C099014F8C4
:100590000C000A909DF880000B909DF885009DF856
:1005A00078809DF87DE09DF882A09DF887900C9062
:1005B0009DF87A00029B1C9314F80A2014F8093065
:1005C00014F8081014F80E700D90205C0E909DF831
:1005D0007F000F90205C10900B98205C11900C987D
:1005E000205C12909DF8840013909DF8790014907F
:1005F0009DF87E001590205C16909DF88300179062
:10060000205C18901398205C19901498205C1A9024
:100610000398013003900298DDF804B01030029086
:100620009DF80C00834536D88DF878108DF87A2027
:1006300009990E9A8DF87C108DF882201199069AEE
:100640008DF880108DF87E201999169A8DF88410F7
:100650008DF886200A99189A8DF87D108DF88720DC
:100660001299109A8DF87B301B9B8DF881108DF8B4
:1006700083201A99089A1D988DF885108DF87F208F
:100680001EA903EB0B128DF87970FFF792FE002084
:1006900023B0BDE8F08F15F808B082EA03008BEABA
:1006A000000016F80EB080EA0B008DF8780015F8FF
:1006B0000E004B40434016F80A0043408DF8793055
:1006C00081EA070315F80A10594016F80930594015
:1006D00016F808308DF87A107A40534015F8092042
:1006E00053408DF87B30089A069B5340049AAA5CCD
:1006F000534016F80C2053408DF87C30DDE9083269
:100700005A4015F80C305340059AB25C53408DF8AE
:100710007D30DDE909325A40059BEB5C5340079A76
:10072000B25C53408DF87E30069B0A9A5340049A7F
:10073000B25C5A40079BEB5C5A408DF87F200E9BC1
:10074000109A53400B9AAA5C53400C9AB25C5340E7
:100750008DF88030DDE910325A400C9BEB5C534041
:100760000D9AB25C53408DF88130DDE911325A4068
:100770000D9BEB5C53400F9AB25C53408DF8823076
:10078000129A0E9B53400B9AB25C5A400F9BEB5C43
:100790001C995A408DF88320169B189A5340139A3F
:1007A000AA5C5340149AB25C53408DF88430DDE962
:1007B00018325A40149BEB5C5340159AB25C53407C
:1007C0008DF88530DDE919325A40159BEB5C5340BA
:1007D000179AB25C53408DF886301A9A169B534094
:1007E000139AB25C5340179AAA5C1EA853408DF826
:1007F0008730FFF79DFDB8E6FF2049E79C3F0108E1
:100800009C3E01089C3D010808B538B1044A0549E1
:100810001060D82200F0B4FA002008BD0220FCE7E6
:1008200048240020CC4401080A4B1A6870B5002304
:1008300002F1180503EB03142E5D864204D118342F
:1008400022440A60002070BD01330B2BF2D103203B
:10085000F9E700BF482400202DE9F041CCB006465E
:10086000DDF8488117461C460D4631B3B8F1000F3C
:1008700023D006A8FFF726FC204601A9FFF7D4FFE6
:100880000446B0B9019906A80131FFF72BFC26B147
:100890001022314606A8FFF72AFC3A46294606A848
:1008A000FFF725FC06A902A8FFF78CFC029BC8F8FD
:1008B000003020464CB0BDE8F0810224F9E700008A
:1008C00030B595B013A90446FFF7AEFF002830D12C
:1008D0001B4B0C2101FB00F2D5189A5CA2422AD1D5
:1008E000139B1A7C1092DA7B0F929A7B0E925A7BA2
:1008F0000D921A7B0C92DA7A0B929A7A0A925A7AB1
:1009000009921A7A0892DA7907929A7906925A79B4
:1009100005921A790492DA7803929A7802925B78B7
:1009200001930022AB6800931146064B022002F0AF
:1009300013FA15B030BD01300B28CBD1F9E700BF59
:10094000144201089C40010810B40B2B019C03D8F1
:10095000019410BCFFF780BF032010BC704730B576
:100960000D4685B01446014668B103AA00200092E6
:100970002A460390FFF770FF18B90398001B18BFB1
:10098000012005B030BD0220FBE72DE9F0430D4604
:10099000BFB014469946804620B31BB311F00F0137
:1009A00022D1F02201A800F0FFF920466946FFF7A6
:1009B0003BFF044648B9009801AA10210130FFF717
:1009C0003BFD2E46AF1BFFB21EB920463FB0BDE82F
:1009D000F08301AA09EB070108EB0700FFF7AEFD62
:1009E000103EEFE70224F0E70524EEE7F0B5184EDD
:1009F0003468024685B00846002304F1180103EB71
:100A000003154F5D97421ED10D2A05F1190513D12B
:100A10000023CDE90033CDE902330C2210216B46CF
:100A2000FFF7B3FF0446306810226946284400F0FF
:100A3000A7F9204605B0F0BD01461022601900F06C
:100A40009FF90024F5E701330B2BD8D10324F0E7FD
:100A50004824002009B1FFF7C9BF022070471FB525
:100A60001446A0B10C2A01D10B2912D10023CDE9E3
:100A70000033CDE902330A466B461021FFF785FFAC
:100A800018B969462046FFF7B1FF04B010BD022037
:100A9000FBE70320F9E7F8B51E46DDE907479DF8B7
:100AA00018505BB354B34FB3212D29D819462A46A9
:100AB000204600F065F90122631C691EB018FFF79B
:100AC00064FFF8B9E37ADB093B70EBB963192046A0
:100AD00013F8012C13F8021C120642EA014213F823
:100AE000041C0A4313F8031C012342EA0122291FB4
:100AF000FFF735FF003818BF0120F8BD0220FCE7E2
:100B00000520FAE70720F8E70420F6E710B50446C9
:100B100028B1044B5B6998472060002010BD02207B
:100B2000FCE700BF2C43010808B5014630B1044B77
:100B30000822186800F024F9002008BD0220FCE714
:100B40004824002008B530B1044B0822196800F091
:100B500017F9002008BD0220FCE700BF4824002050
:100B60007FB5124E0023044602A801930D46FFF7FD
:100B7000E9FF33685B6901936CB102AA082312F89C
:100B8000011B41B9013B13F0FF03F8D102A8A047B4
:100B900002A8FFF7C9FF35B1019B23B901A8A847F7
:100BA0003368019A5A61002004B070BD48240020C7
:100BB00008B5014638B1054B18680822104400F00A
:100BC000DFF8002008BD0220FCE700BF4824002019
:100BD00008B538B1044B19680822114400F0D0F868
:100BE000002008BD0220FCE748240020034B1B68BE
:100BF00002280CBF19615961002070474824002069
:100C000049B1064B1B68D3E90423022808BF1346E9
:100C10000B60002070470220704700BF482400206E
:100C200030B58FB0002405460CA80994FFF78AFF61
:100C30009DF8373007939DF8363006939DF8353090
:100C400005939DF8343004939DF8333003939DF859
:100C5000323002939DF8313001939DF8303000938B
:100C6000224621461E4B022002F076F80AA8FFF722
:100C7000AFFF9DF82F3007939DF82E3006939DF817
:100C80002D3005939DF82C3004939DF82B30039361
:100C90009DF82A3002939DF8293001939DF8283061
:100CA000009322460F4B2146022002F055F809A975
:100CB0002846FFF7A5FF9DF8243003939DF82530C3
:100CC00002939DF8263001939DF827300093224629
:100CD000054B2146022002F03FF80FB030BD00BFA7
:100CE000F8400108364101087441010808B50020A8
:100CF000FFF7E6FD0120FFF7E3FD0920FFF7E0FD28
:100D00000820FFF7DDFD0020FFF78AFF002008BD67
:100D100010B504460B20FFF7D3FD0C20FFF7D0FDE4
:100D20000920FFF7CDFD0820FFF7CAFD0A20FFF7D5
:100D3000C7FD2046FFF774FF002010BD014B18606F
:100D4000704700BFAC0800200B4A30B514680B4D4B
:100D500043F2390305FB04331360091A6FF00042B4
:100D6000B3FBF2F2C2EBC27201319B1A93FBF1F2B8
:100D700001FB1233184430BDAC0800206D4EC64153
:100D800001380A44914200D1704711F8013B00F844
:100D9000013FF7E710440A44914200D1704711F82F
:100DA000013B00F8013DF7E702F018BD30B530B166
:100DB0000A4D01444FF0FF33814201D1D84330BD89
:100DC00010F8012B5340082243F30004013A2C4051
:100DD00092B284EA5303002AF6D1EDE72083B8EDFE
:100DE00001207047054B4FF400529A62044B1B6878
:100DF00013B15B6803B11847704700BF0004004897
:100E0000D8240020054B4FF480529A62044B1B6893
:100E100013B1DB6803B11847704700BF00040048F6
:100E2000D8240020012070470120704701F03EB90E
:100E300001F02CB910B501F00FFE0E21044640F66A
:100E40001F1001F023F92046012101F0EFFDBDE85C
:100E5000104001F0CDBA000070B50C4E01EB40031C
:100E60000D46B3654FF6FF71002304461A46084647
:100E700001F054FB96F85600002101F0D7FD2946F9
:100E80002046BDE8704001F08BBA00BF7C240020F2
:100E900010B5044601F0A0FE01281CD101F0A4FE0B
:100EA00034B11248214602F00BFB104802F0CEFA92
:100EB0000F4C104B00214FF48052A1659A6194F8B9
:100EC000560001F0B3FD63786BB16FF07F40BDE871
:100ED000104001F049BA002340F262211A46084648
:100EE00001F01CFBDCE7A0688001F0E74C24002047
:100EF0007C24002000040048002001F0B5B9000067
:100F000008B501F0BDF80438C0B2032896BF024B03
:100F10000020185C08BD00BFF642010808B501F0CA
:100F2000B0FD033008BD01F03FB901F0FFB808B5CE
:100F300001F0F6FC08BD000038B50D46144601F07E
:100F400053FB284601F088FD0E21054640F61F1090
:100F500001F09CF828460121074D01F067FD01F0E2
:100F600047FA4FF47A716143284602F0A9FA2846FD
:100F7000BDE8384002F06ABA6424002001F034BBB6
:100F800008B5084B002193F8560001F04FFD0023EF
:100F90004FF4C0711A46084601F0C0FABDE8084097
:100FA00001F01ABA7C24002010B5044601F014FEAA
:100FB00001281CD101F018FE34B11248214602F07C
:100FC0007FFA104802F042FA0F4C104B00214FF408
:100FD0008052A1659A6194F8560001F027FD63786C
:100FE0006BB16FF07F40BDE8104001F073B9002392
:100FF00040F262211A46084601F090FADCE7A06848
:101000008001F0E74C2400207C24002000040048EC
:1010100008B54FF0040001F00DF9BDE808400220CA
:10102000F1F744BD08B500231A461946184601F0E9
:1010300075FABDE8084001F063B900001D4B73B5B7
:101040001D4D186000241D486C70C5E90144AC6555
:1010500001F08EFAAC8101F0F9F92146204601F049
:1010600041FC21460422012001F0F2FA144E154DF4
:101070004FF6FF7123462246084601F04FFAFFF76C
:10108000C7FF2246104B00944FF0FF31304602F06C
:1010900031F90E4B009422464FF0FF31284602F002
:1010A00029F9304602F084F9284602B0BDE87040C4
:1010B00002F07EB9D82400207C2400207120010891
:1010C000642400204C240020E50D0108050E0108D1
:1010D0000128084805D1084BC17719700E3001F07E
:1010E0009DBB437D012B03D1034B81751970F5E73F
:1010F000704700BF7C240020B00800200D4B10B5C5
:10110000044618735873012000F016F85CB13421BE
:101110004FF4E86000F0BAFF4421BDE8104040F20F
:10112000417000F0B3BF14214FF4E86000F0AEFF4F
:101130002421F2E77C24002038B5114C05462070AC
:1011400001F057FD052D04D8DFE805F0090B031762
:101150001709032001F066FA0023637338BD0020ED
:10116000F8E7012001F05EFA207B637B8342F5D033
:101170006073BDE83840FFF7C1BF0220EAE700BF57
:101180007C2400202DE9F0431E4687B0002305464D
:10119000CDE901330C46174601F01DFD032D5BD848
:1011A000DFE815F07A00C1000C010400A27C082AD7
:1011B00069D8A16801A801F0D5FE2168002962D094
:1011C00042F210729142E37C874D50D80322AA73F9
:1011D00085F83820E96385F844304FF002086368E9
:1011E000A17DDB002B820423AB74A37CDB00EB74BA
:1011F00002294FF000032B75637D02D0227D022A65
:1012000046D103F10F02D2B2012A01D9012B3AD102
:10121000764B774A196803944FF0010903A88DF8BB
:10122000149001F0D5FC70BB287685F8179068758E
:10123000FFF762FE4046FFF77FFF6E4801F082FA3B
:101240006D4801F0EBFA01A800F080FF208A00F061
:1012500051FFA08900F096FF384601F0FDFB624C7B
:1012600084F8560001F0BCFC666000200DE04FF0F1
:101270000008E963890885F80E8085F8388085F8CC
:1012800044302964ABE74FF0FF3007B0BDE8F0838E
:10129000EB7529766A75CBE72368002BF3D0A27C27
:1012A000082AF0D8504DA16801A801F05BFE002388
:1012B00085F838302268EA63E27C85F84420A26928
:1012C000AB732A646268D2002A820422AA74A27CC8
:1012D0002B75D200EA74A27D022A02D0237D022B54
:1012E0001CD1627D02F10F03DBB2012B01D9012A6F
:1012F000C9D13E4B3E4A196803944FF0010803A838
:101300008DF8148001F064FC0028BCD1287685F8A3
:1013100017806875FFF7F0FD00208CE7617DE975A7
:101320002A766B75F6E7304D012185F83810227862
:1013300085F85020637885F85130A37885F85230CD
:10134000E3788B4202D0022B03D03BB985F85330AF
:1013500004E00B3A012A29D885F853104FF0010810
:1013600085F80E80A388AB83A379AB77E37985F802
:101370002030237A85F82130FFF7BEFD4046FFF785
:10138000DBFE1C4801F0DEF91B4801F047FA95F836
:101390005130062B40F689000AD100F087FE00F09C
:1013A000FB0140F6890000F071FE55E70023CDE710
:1013B00000F07CFE40F00401C9B2F2E72368013B73
:1013C000B3F57A7FBFF45FAF0320FFF7B5FE0648A1
:1013D000022380F8383023688364162380F84C3069
:1013E000383001F0AFF937E77C240020D824002002
:1013F00064240020B42400208A240020F0B51E4676
:1014000087B00023CDE90133144607460D4601F0AD
:10141000E2FB002C724C16BF0123002300266370F0
:1014200027B1012F7AD0002007B0F0BDAB68002BA8
:1014300000F0D280EB68002B00F0CE80AA7F082A53
:1014400000F2CA80296901A801F08CFD28680038E3
:1014500018BF012000F0D6FF84F83870AB68E36352
:1014600095F8203084F84430686801F057FBA77382
:1014700084F84500EB68DB002382EB7FA374AB7F2D
:10148000DB00E37495F82130237595F82230002BAA
:101490003ED12A7D95F82410A275022995F82320C3
:1014A00001D0022B36D102F10F03DBB2012B02D99E
:1014B000012A40F0918000238DF81430494B4A4AAC
:1014C0001968049503A801F083FB002840F084808C
:1014D00001232076E3756075FFF70EFD0020FFF70E
:1014E0002BFE424801F02EF9414801F097F901A87E
:1014F00000F02CFEA88B00F0FDFD288B00F042FED2
:101500004FF4FA53AA687343B3FBF2F3A3608AE77C
:10151000FF22BFE7E27521766375DDE72B8E002B96
:101520005AD095F83230A86A012B0CBF2F7DFF27C7
:10153000003818BF012000F065FFF0B200F06EFF28
:10154000012184F8381095F82C2084F8502095F863
:101550002D3084F8513095F82E3084F8523095F8BB
:101560002F308B4202D0022B03D03BB984F853308A
:1015700004E00B3A012A27D884F853102B8EA3835A
:1015800095F83230A3770126AB8E2384A673E777D4
:10159000FFF7B2FC3046FFF7CFFD144801F0D2F858
:1015A000134801F03BF994F82130B34240F2367011
:1015B0000CD100F07BFD00F0FB0140F2367000F032
:1015C00065FD4FF6FF73A1E70023CFE700F06EFD46
:1015D00040F00401C9B2F0E74FF0FF3024E700BF4C
:1015E0007C240020D82400204C240020B424002097
:1015F0008A2400202DE9F04F85B082460E9DBDF86B
:1016000040809DF844709DF84890019193461E4695
:1016100001F0E1FABAF1010F524C54D0BAF1040FC3
:1016200000F09180BAF1000F3AD10B22304684F8D5
:10163000442084F838A0E56301F070FA4FEAC8034B
:10164000B9F1000F238241F6040363820CBF01232A
:10165000F223E37587F001070123237684F8450020
:10166000C4F840B084F80EA084F814A06775FFF7A2
:1016700043FC5046FFF760FD04F1380001F062F8CA
:1016800004F10E0001F0CAF8374A1068516802AB45
:1016900003C302A800F05AFD40F2FF1000F02AFD3B
:1016A000019801F0D9F90E2184F8560040F61F1078
:1016B00000F0ECFC94F8560001F092FA169B63607F
:1016C00005B0BDE8F08F294984F838A0EAB2895DF9
:1016D00084F8502076BB0B3D012D8CBF00250125E1
:1016E000053A012A04D8B8F10C0F38BF4FF00C08A6
:1016F0001F4B9DF83C201B7884F85350E37701255D
:101700009DF8543084F8511084F8522084F8213028
:10171000A573A4F81C80A77784F82090FFF7ECFB52
:101720002846FFF709FD134801F00CF8124801F0B4
:1017300075F8B5E7012E04D1A5F10C035D425D41BA
:10174000CEE70025CCE75046FFF7F6FC022384F8ED
:10175000383004F138001623A56484F84C3000F0CA
:10176000F1FF9DE77C240020E039010828430108AF
:10177000B0080020B42400208A2400202DE9F04F76
:1017800087B0DFF8B4B29DF864A09DF84C90029346
:1017900014469DF854309DF85020BDF848800392BF
:1017A00005468BF801A0BDF8446001930F4601F097
:1017B00012FABAF1000F18BF4FF00008DFF87CA250
:1017C000039AB9F1000F08BFFF22012D8AF800200B
:1017D00000F0C880052D48D0002D40F0C08028467C
:1017E00000F010FE0B2238468BF844208BF838505E
:1017F000CBF83C4001F092F9019B8BF8450041F693
:101800000402002BABF812209AF800208BF8162067
:101810000CBF0122F2228BF81720F600012289F07A
:1018200001098BF818208BF80E50ABF810608BF87C
:1018300014508BF81590FFF75FFB2846FFF77CFCF0
:101840000BF1380000F07EFF0BF10E0000F0E6FF18
:101850007B490868496804AA03C204A800F076FC22
:1018600040F2FF1000F046FC71E0012000F0CAFDDC
:1018700009224FF000098BF8442038464FF4487293
:10188000CBF840208BF83890CBF83C4001F046F97B
:101890004FF48052ABF812209AF800208BF84500E4
:1018A0008BF8162028460122F6008BF817208BF8BB
:1018B0000E90ABF81060ABF814908BF81890FFF70F
:1018C0003BFC0BF1380000F03DFF0BF10E0000F087
:1018D000A5FF5B498868C96804AA03C204A800F090
:1018E00035FC40F2FF1000F005FC40F6B80000F0B7
:1018F000DDFB00F0EF0140F6B80000F0C7FB04216B
:1019000040F6B90000F0C2FB40F69B0000F0CEFBB1
:1019100000F0E30141F0080140F69B0000F0B6FB47
:1019200040F2D16000F0C2FB40F01801C9B240F2B1
:10193000D16000F0ABFB40F2AC6000F0B7FB00F010
:101940008F0141F0500140F2AC6000F09FFB4FF47A
:10195000FA5202FB08F2B2FBF4F2CBF8082007B00F
:10196000BDE8F08F002000F04DFD36498BF838506F
:10197000E2B2C95D8BF85020002F4DD10B3C012CF9
:101980008CBF00240124053A012A02D80C2E38BF4E
:101990000C26029B9AF800208BF852308BF85340AB
:1019A000019B8BF81F2001249DF860208BF82120DB
:1019B0008BF851108BF820308BF80E40ABF81C6080
:1019C0008BF81E90FFF798FA2046FFF7B5FB1E48EC
:1019D00000F0B8FE1D4800F021FF5FFA88F000F02B
:1019E0001DFD40F6A30000F061FB00EA040140F693
:1019F000A30000F04BFB9BF82120A24240F236707E
:101A000013D100F053FB00F0FB0140F2367000F000
:101A10003DFB4FF6FF72A0E7012F04D1A4F10C03A8
:101A20005C425C41AFE70024ADE700F03FFB40F0D3
:101A30000401C9B2E9E700BF7C240020B0080020FF
:101A4000E039010828430108B42400208A2400203A
:101A5000F0B58BB00D46044617461E46FFF74CFA0C
:101A60000020FFF769FB204600F0BEFD00240123A3
:101A7000CDE9084303234FF4167229462046CDE9E9
:101A80000644CDE90444CDE90244CDE900532346A0
:101A9000FFF774FE2046FFF787FAFFF73FFAF1F7EA
:101AA00005F801F041FC0446204601F047FCB04235
:101AB00005D30124FFF720FA20460BB0F0BD00F05B
:101AC0002FFF8742F0DA0024F4E70000F7B5002387
:101AD0000C4640F201211A460646084600F01EFD5B
:101AE000644B654D4FF400529A6195F85600012100
:101AF00000F09CFF2B78012B40F6890013D195F85C
:101B00005130062B0FD100F0D1FA00F0FB0140F666
:101B1000890000F0BBFA2B78042B6CD8DFE803F0C7
:101B2000524B527F090000F0C1FA40F00401C9B2E3
:101B3000EDE7524A731E1046C6F101074FF0000C44
:101B4000F9188C426FDC0022E7001346BA4271D1CB
:101B50009A0142EAC3125B0183F020031343661C1F
:101B60000355F6B202234648AB73AE7600F056FE3C
:101B70000021F12000F08AFA0021F02000F086FA1E
:101B8000AB6C642B70D17021F32000F07FFA1D2123
:101B9000F22000F07BFAE1008C1CF420090A00F02E
:101BA00075FA04F0FE01F52000F070FA33486FF08A
:101BB0007F4231461DE0EC77314800F02FFE0022D5
:101BC000214615E001F008F80128074625D12146F5
:101BD0000DF10702304601F004F80446A0B99DF863
:101BE00007302748AB7500F019FE9DF80710224614
:101BF000304600F065FB6968224801F061FC21482D
